:100000000C94AA200C94C7200C94C7200C94C720F1
:100010000C94C7200C94C7200C94C7200C94909586
:100020000C94C7200C94C7200C94C7200C94A08B70
:100030000C94C7200C94C7200C94C7200C949F43A9
:100040000C94C7200C94BEB90C9422340C945134F7
:100050000C9484340C945A2A0C9457480C94C7205E
:100060000C9441780C9484930C94C7200C94C72072
:100070000C94C7200C94C7200C94C7200C94C72064
:0C0080000C94C7200C94C7200C94C720DF
:100100005A5A5A5A5A5A5A5A5A5A5A5A5A5A5A5A4F
:100110005A5A5A5A5A5A5A5A5A5A5A5A5A5A5A5A3F
:100120005A5A5A5A5A5A5A5A5A5A5A5A5A5A5A5A2F
:100130005A5A5A5A5A5A5A5A5A5A5A5A5A5A5A5B1E
:100140005B5B5B5B5B5B5C5C5C5C5C5C5C5D5D5DF2
:100150005D5D5D5D5D5E5E5E5E5E5E5E5F5F5F5FC0
:100160005F5F5F5F60606060606060606061616190
:100170006161616161626262626262626263636361
:100180006363636363636464646464646464656533
:100190006565656565656666666666666666676703
:1001A00067676767676767686868686868686969D4
:1001B00069696969696A6A6A6A6A6A6A6B6B6B6BA0
:1001C0006B6B6C6C6C6C6C6C6D6D6D6D6D6E6E6E66
:1001D0006E6E6E6F6F6F6F70707070717171717223
:1001E00072727273737374747475757676767777CA
:1001F0007878797A7A7B7C7D7D7D7D7D7D7D7D7D46
:10020000FFFFFFFFFFFFFFFFFFFFFFFFFFFFFEFA04
:10021000F6F2EEEBE7E4E1DFDCDAD7D5D2D0CECCF4
:10022000CAC9C7C5C3C1C0BEBDBBBAB8B7B6B4B3EF
:10023000B2B0AFAEADABAAA9A8A7A6A5A4A3A2A130
:10024000A09F9E9D9C9B9A99989797969594939220
:100250009291908F8F8E8D8C8B8B8A8988888786E0
:100260008585848383828181807F7F7E7D7C7C7B8A
:100270007A7A797878777776757574737372717125
:10028000706F6F6E6E6D6C6C6B6A6A6968686766BA
:1002900066656464636362616160605F5E5E5D5D4C
:1002A0005C5B5B5A5A5958585756565554535352DB
:1002B0005151504F4F4E4D4D4C4B4B4A4949484878
:1002C0004746454444434241403F3F3E3D3C3B3B23
:1002D0003A393837373635343332312F2E2D2C2BEF
:1002E0002A29282726242322201F1D1B1A18161509
:1002F00013110F0C0A0704020000000000000000A8
:10030000FFFFFFFFFFFFFFFFFFFFFFFFFFFFFEFA03
:10031000F6F2EEEBE7E4E1DFDCDAD7D5D2D0CECCF3
:10032000CAC9C7C5C3C1C0BEBDBBBAB8B7B6B4B3EE
:10033000B2B0AFAEADABAAA9A8A7A6A5A4A3A2A12F
:10034000A09F9E9D9C9B9A9998979796959493921F
:100350009291908F8F8E8D8C8B8B8A8988888786DF
:100360008585848383828181807F7F7E7D7C7C7B89
:100370007A7A797878777776757574737372717124
:10038000706F6F6E6E6D6C6C6B6A6A6968686766B9
:1003900066656464636362616160605F5E5E5D5D4B
:1003A0005C5B5B5A5A5958585756565554535352DA
:1003B0005151504F4F4E4D4D4C4B4B4A4949484877
:1003C0004746454444434241403F3F3E3D3C3B3B22
:1003D0003A393837373635343332312F2E2D2C2BEE
:1003E0002A29282726242322201F1D1B1A18161508
:1003F00013110F0C0A0704020000000000000000A7
:10040000062B032B2A2B272BF42A242BF72A212B0C
:10041000302BF42AF72AFA2A2D2BF72AFA2AF42A63
:10042000002B1E2B1B2B182B122B0F2B092B7B2D7C
:10043000772D772D6B2D582D832D7F2D8D2D3B2DD9
:10044000472D3F2D4B2DB42CAC2CA42C9E2C862C50
:10045000F52CF12CD72CD32CC72CC22CBE2CB82CAD
:10046000112D0B2DFF2CF92C2F2D1D2D232D802C24
:10047000682C5C2C742C502C442C342C242CF12B08
:10048000ED2BE92BE52BE12BDD2BD92BA42B752BA9
:10049000083233323732C331C331C331C3315B32F7
:1004A000C3316232C331BD31C33167326C32C331C3
:1004B0007132C3319532B932C331C331C331C33123
:1004C000C331C331C331C331C331C331C331C3318C
:1004D000C331C331C331C331C331C331C331BE3280
:1004E000C331F132C3311E33C3314B337833EC3275
:1004F000C331C331C331D033C331A333FD33499A40
:10050000219A109A289AED99B49AA89A659A5D9AB8
:100510002E9C3D9AB49BCC99189C549C489C3B9B28
:100520001F9BF59AEA9AC099DB9AC99A3A9C359C26
:10053000119B039B979A8B9A559A879D839D7F9DCC
:1005400031AA31AA31AA31AA7B9D31AA31AA779D5D
:1005500031AA31AA31AA31AA259D31AA219D1D9D1A
:1005600031AA199DC79CC39C31AA31AA31AA31AACC
:1005700031AA31AA31AA31AA31AA31AA31AA31AAA3
:1005800031AA31AA31AA31AA31AABE9C31AA31AA14
:1005900031AA31AA31AAB99CB49CAF9C31AA31AA24
:1005A00031AA31AA31AA31AA31AA31AA31AA31AA73
:1005B00031AA31AA31AA31AA31AA31AA31AA31AA63
:1005C00031AA31AA31AA31AA31AA31AA31AA31AA53
:1005D00031AA31AA31AA31AA31AA31AA31AA31AA43
:1005E00031AA31AA31AA31AA31AA31AA31AA31AA33
:1005F00031AA31AA31AA31AA31AA31AA31AA31AA23
:1006000031AA31AA31AA31AA31AA31AA31AA31AA12
:1006100031AA31AA31AA31AA31AA31AA31AA31AA02
:1006200031AA31AA31AA31AA31AA31AA31AA31AAF2
:1006300031AA31AA31AA31AA31AA31AA31AA31AAE2
:1006400031AA31AA31AA31AA31AA31AA31AA31AAD2
:1006500031AA31AA31AA31AA31AA31AAA79C31AA5A
:1006600031AA31AA31AA31AA31AA31AA979C979D01
:10067000C39DAD9D939D259E0A9EF29D939DDB9DFE
:100680009A9E839E7A9E639E939D139FB19E4C9EDD
:10069000939D369E939D939D61A00BA0939DA99FD2
:1006A000939D939D939D939D939D939D939D939DCA
:1006B000939D879F939D939D939D939D939D7D9FD8
:1006C000939D939D939D939D939D719F649F509F38
:1006D000939D939D939D939D939D939D939D939D9A
:1006E000939D939D939D939D939D939D939D939D8A
:1006F000939D939D939D939D939D939D939D939D7A
:10070000939D939D939D939D939D939D939D939D69
:10071000939D939D939D939D939D939D939D939D59
:10072000939D939D939D939D939D939D939D939D49
:10073000939D939D939D939D939D939D939D939D39
:10074000939D939D939D939D939D939D939D939D29
:10075000939D939D939D939D939D939D939D939D19
:10076000939D939D939D939D939D939D939D939D09
:10077000939D939D939D939D939D939D939D939DF9
:10078000939D939D939D939D939D939DF2A0DEA039
:10079000CAA0B6A011A1FDA03C9F289F61A14DA1B8
:1007A00039A125A10EC2F9C1F9C1F9C109C2F5C12A
:1007B00027C2F5C1FCC1F5C122C2F5C1FCC1F5C11A
:1007C00001C2F5C134C230C22CC215C211C21DC251
:1007D000F5C1FCC1F5C119C2F9C1FFFFFFFF0080DF
:1007E000555500403333AB2A92240020721C9A19CD
:1007F00046175515B1134912111100100F0F390E7C
:10080000790DCD0C310CA30B210BAB0A3D0AD90994
:100810007B092509D408890842080008C20788070F
:1008200050071C07EB06BD06900666063E06180636
:10083000F405D105B00591057205550539051F056B
:100840000505EC04D504BE04A80492047E046A04E1
:10085000570444043204210410040004F003E103AB
:10086000D203C403B603A8039B038E03820376035B
:100870006A035E03530348033E03330329031F0344
:1008800016030C030303FA02F102E902E002D802A4
:10089000D002C802C102B902B202AB02A4029D0298
:1008A00096028F02890283027C02760270026A023B
:1008B00064025F02590254024E02490244023F029E
:1008C0003A02350230022B02270222021E021902CE
:1008D000150211020C02080204020002FC01F801D8
:1008E000F401F001ED01E901E501E201DE01DB01C6
:1008F000D701D401D101CE01CA01C701C401C10190
:10090000BE01BB01B801B501B201AF01AC01AA0142
:10091000A701A401A1019F019C019A0197019501E2
:10092000920190018D018B01880186018401820171
:100930007F017D017B0179017601740172017001F3
:100940006E016C016A016801660164016201600167
:100950005E015D015B0159015701550154015201CE
:1009600050014E014D014B0149014801460144012E
:100970004301410140013E013D013B013A01380183
:10098000370135013401320131012F012E012D01D2
:100990002B012A012901270126012501230122011A
:1009A00021011F011E011D011C011A01190118015D
:1009B00017011601150113011201110110010F0198
:1009C0000E010D010B010A010901080107010601D1
:1009D00005010401030102010101FF1814009090B8
:1009E000909022069E031A062206D6046605210769
:1009F000660556454D532047656E626F61726420EF
:100A000076332C200071185D185918551846184176
:100A1000182F182A18191800000000000000000004
:100A20000000000000000000000E180000000000A0
:100A300000000000000000000000000000FD17F4AE
:100A400017EC17E217DA17D217CB17C317B917A786
:100A500017A017981790178B17000078176D1700BD
:100A60000000000000671700000000000058174F4A
:100A70001748173F173117231713170017F616E8F3
:100A800016DF16D616CD16C416BB16AF16A916A1BC
:100A90001698168F1686167A166D16641656164810
:100AA000163516221615160816F515E215CF15B7C8
:100AB00015AD15A6159F1598158D1576155F154959
:100AC000153C152D1516150A150000000000000034
:100AD0000000000000000000000000FA14EC14DE2A
:100AE00014C814B314A11498149014841479146EB7
:100AF00014631458144D143E142F14241419140F95
:100B0000140414F513E413D613C713B713A9139CD5
:100B1000138913771368135313411330131D130AEA
:100B200013F712E012CF12BE12AD1298127F127498
:100B3000125E124D1241122F121E1212120012F0EA
:100B400011DE11CD11B811A611931180116C115F36
:100B500011521141112E111B110811F510E110D283
:100B600010C310B510AE10A41096108D1081106F28
:100B7000105D104C103C102A101E101010FA0FEDD2
:100B80000FD90FC50FAF0F990F840F770F6B0F6041
:100B90000F4E0F460F3D0F2C0F1C0F0B0FFB0EE6D9
:100BA0000ED10EC30EB40EA60E9B0E8D0E7D0E6DD5
:100BB0000E5D0E4D0E3D0E2D0E1C0E0C0EFC0DECA2
:100BC0000DDC0DCC0DBC0DAB0D9F0D8F0D830D738A
:100BD0000D6A0D5A0D4F0D3E0D2C0D1F0D120D05FA
:100BE0000DF40CE60CD60CC90CBC0CAC0C990C89A1
:100BF0000C780C680C580C4B0C3E0C300C1F0C1174
:100C00000C050C0000736F667472706D5F72706D0E
:100C10000073686966746375745F74696D650073E9
:100C2000686966746375745F6368616E6E656C0095
:100C300073686966746375745F636F6E6600746170
:100C400063685F6469766964657200746163685F94
:100C50006368616E6E656C006675656C6375745F64
:100C60006D61785F6B7061006675656C6375745F4C
:100C70006D696E5F6B706100746F6F746872656C24
:100C80005F6D697373696E6700746F6F7468726506
:100C90006C5F6E6F726D616C0077617465725F700E
:100CA000756D705F6368616E6E656C007761746509
:100CB000725F70756D705F687973740068796272C5
:100CC00069645F72706D5F6D006879627269645FFC
:100CD00072706D5F610077617465725F70756D70C1
:100CE0005F74656D7000626F6F73745F6368616ECF
:100CF0006E656C00626F6F73745F7069645F696CBE
:100D0000696D697400626F6F73745F7069645F6BA3
:100D10006400626F6F73745F7069645F6B69006217
:100D20006F6F73745F7069645F6B7000626F6F7375
:100D3000745F6D696E707265737375726500626F52
:100D40006F73745F7461726765746F666673006257
:100D50006F6F73745F636F6E6600616C735F746B4B
:100D6000735F6368616E6E656C00656774315F63A5
:100D7000616C006163745F72706D5F6368616E6E59
:100D8000656C006163745F72706D5F72706D00619D
:100D900063745F776F745F6368616E6E656C00612A
:100DA00063745F776F745F72706D006D6973633227
:100DB0006F75745F6368616E6E656C006D697363F7
:100DC000326F75745F6D61786D6170006D6973630A
:100DD000326F75745F6D696E6D6170006D697363FC
:100DE000326F75745F6D6178747073006D697363D1
:100DF000326F75745F6D696E747073006D697363C3
:100E0000326F75745F6D617872706D006D697363B8
:100E1000326F75745F6D696E72706D006D697363AA
:100E2000316F75745F6368616E6E656C006D6973B8
:100E300063316F75745F6D61786D6170006D69739A
:100E400063316F75745F6D696E6D6170006D69738C
:100E500063316F75745F6D6178747073006D697361
:100E600063316F75745F6D696E747073006D697353
:100E700063316F75745F6D617872706D006D697349
:100E800063316F75745F6D696E72706D00616C7344
:100E90005F7265765F6C696D697400616C735F7217
:100EA000657461726400616C735F64656163745F33
:100EB00065677400616C735F64656163745F746916
:100EC0006D6500616C735F64656163745F72706D02
:100ED00000696E6A5F7374616765325F7374617213
:100EE000745F6D617000696E6A5F7374616765320B
:100EF0005F73746172745F74707300696E6A5F739C
:100F000074616765325F72617465006675656C70E7
:100F1000756D705F6368616E6E656C0070756D7085
:100F20005F6F6E5F6D696E74696D6500656E676990
:100F30006E655F6F66665F64656C61790069676E98
:100F400063686D61780069676E5F6F7574006967CB
:100F50006E5F6372616E6B5F616476616E63650084
:100F600069676E5F6477656C6C360069676E5F6495
:100F700077656C6C31340069676E5F7464636465B7
:100F80006C61790072657365745F656E6770686126
:100F900073655F61667465720063616D5F73796E1E
:100FA000635F665F656467655F7068617365006352
:100FB000616D5F73796E635F725F656467655F70B3
:100FC0006861736500746F6F74685F776865656CDE
:100FD0005F7477696474683200746F6F74685F77E8
:100FE0006865656C5F747769647468310063726109
:100FF0006E6B5F6D696E70657200616E6F746865AF
:10100000725F747269676765725F746F6F7468008E
:10101000747269676765725F746F6F746800746F6C
:101020006F74685F776865656C007365636F6E6485
:101030006172795F74726967676572007072696D59
:101040006172795F74726967676572006C63645F6F
:1010500064656661756C745F7669657700616C7351
:101060005F7265746172645F6D6178747073006142
:101070006C735F7265746172645F6D696E747073B6
:101080000069676E5F62616C616E6365006B7061C1
:101090005F636F6E66006C63645F6261636B6C6953
:1010A000676874006C63645F64656C6179006C638D
:1010B000645F63300076655F6C6561726E5F636F5D
:1010C0006E660076655F6C6561726E5F6C696D69F6
:1010D000740076655F6C6561726E5F7370656564E0
:1010E0000076655F6C6561726E5F6D696E5F7765D6
:1010F000696768740076655F6C6561726E5F6567CD
:101100006F5F7363616C650076655F6C6561726EBD
:101110005F6B70615F7363616C650076655F6C65C2
:1011200061726E5F72706D5F7363616C650076658E
:101130005F6C6561726E5F6D61785F706F7765720D
:101140000076655F6C6561726E5F636F6F6C616E78
:1011500074006B6E6F636B5F6D617872706D006BA6
:101160006E6F636B5F6D696E72706D006B6E6F6337
:101170006B5F616476616E63655F64656C61790065
:101180006B6E6F636B5F616476616E63655F7374D2
:101190006570006B6E6F636B5F7265746172645F24
:1011A00064656C6179006B6E6F636B5F726574610F
:1011B00072645F73746570006B6E6F636B5F646500
:1011C0006661756C745F726574617264006B6E6FDA
:1011D000636B5F6D61785F726574617264006B6EE2
:1011E0006F636B5F6E6F6973655F7363616C6500DE
:1011F0006B6E6F636B5F7468726573686F6C6400AD
:101200006B6E6F636B325F696E7465677261746F6A
:1012100072006B6E6F636B325F6761696E006B6E3D
:101220006F636B325F6672657175656E6379006BB3
:101230006E6F636B315F696E7465677261746F7234
:10124000006B6E6F636B315F6761696E006B6E6F11
:10125000636B315F6672657175656E6379006B6E85
:101260006F636B5F73616D706C696E675F77696EDA
:10127000646F77006B6E6F636B5F636F6E66007792
:10128000626F325F72695F636F6E666964656E6319
:10129000655F7363616C650077626F325F70756D57
:1012A000705F7069645F696C696D69740077626F03
:1012B000325F70756D705F7069645F6B6400776238
:1012C0006F325F70756D705F7069645F6B69007716
:1012D000626F325F70756D705F7069645F6B700014
:1012E00077626F325F6865617465725F7069645FB1
:1012F000696C696D69740077626F325F68656174EB
:1013000065725F7069645F6B640077626F325F68FB
:1013100065617465725F7069645F6B690077626FA5
:10132000325F6865617465725F7069645F6B7000DD
:1013300077626F325F63616C6962726174696F6E4C
:101340000077626F325F70756D705F70775F7A657E
:10135000726F0077626F325F6E65726E7374646372
:101360005F7461726765740077626F325F72695F84
:101370007461726765740077626F325F6564676578
:1013800074696D655F6D696E0077626F325F656469
:10139000676574696D655F636F72720077626F3243
:1013A0005F72657472795F740077626F325F666135
:1013B0006C6C6261636B0077626F325F6C696D6940
:1013C000745F6D6178740077626F325F6162735F22
:1013D0006C696D697400616C735F72656163745FE1
:1013E0007470730077626F325F7761726D75705FD2
:1013F00072616D700065676F5F7069645F77696EB9
:10140000646F770065676F5F74617267657400650C
:10141000676F5F64656C746100616C735F656E72A9
:101420006963680065676F5F7069645F6B70006512
:10143000676F5F726963685F6C696D697400656787
:101440006F5F6C65616E5F6C696D69740065676F75
:101450005F7761726D75700065676F5F6D6178723F
:10146000706D0065676F5F6D696E72706D006567A6
:101470006F5F6D61786D61700065676F5F6D61783A
:101480007470730065676F5F636F6F6C616E74007B
:1014900065676F5F6C61670065676F5F636F6E663E
:1014A000006961635F69676E5F7468726573686F16
:1014B0006C64006961635F69676E5F726574617215
:1014C000645F6C696D6974006961635F69676E5F11
:1014D000616476616E63655F6C696D697400736FDA
:1014E000667472706D5F72616E6765006961635FDB
:1014F00069676E5F736C6F7065006961635F736FBE
:101500006C5F6368616E6E656C006961635F7265D4
:10151000665F706F73006961635F6F766572636C9D
:101520006F73655F696E74657276616C00616C7370
:101530005F6375745F6D6178747073006961635F78
:101540006465616462616E64006961635F696E74A1
:10155000656772616C5F6465616462616E64006995
:1015600061635F696E74656772616C5F6C696D69F8
:10157000745F696E63006961635F696E7465677249
:10158000616C5F6C696D69745F646563006C617543
:101590006E63685F72706D006961635F6B640069A0
:1015A00061635F6B69006961635F6B7000696163B0
:1015B0005F7370656564006961635F61667465721D
:1015C00073746172745F6475726174696F6E0069BF
:1015D00061635F616674657273746172745F727067
:1015E0006D006961635F7761726D5F7374617274BE
:1015F0005F706F73006961635F636F6C645F7374C6
:101600006172745F706F73006961635F7761726D9F
:101610005F72706D006961635F636F6C645F7270AD
:101620006D006961635F7761726D5F69646C655FAE
:1016300074656D70006961635F636F6C645F69649A
:101640006C655F74656D70006961635F7470735F72
:101650007468726573006961635F6D61785F73744C
:10166000657073006961635F636F6E6600696163D3
:101670005F737465705F7365710066616E5F636848
:10168000616E6E656C0066616E5F6879737400668A
:10169000616E5F74656D70007470735F6869676810
:1016A000007470735F6C6F7700646261726F0061C9
:1016B0006C735F6D61785F637574006661737469E4
:1016C000646C6500626174745F63616C00636F6E6B
:1016D000666967313300636F6E6669673132006334
:1016E0006F6E66696731310061697264656E5F694A
:1016F000676E6F7265007265765F6C696D69740004
:101700006F76657272756E5F6675656C72657375FE
:101710006D65006F76657272756E5F6675656C6378
:101720007574006C61756E63685F72657461726474
:10173000006C61756E63685F656E726963680074E2
:10174000707361636F6C640061636D756C740074B9
:1017500070736173796E6300616C735F6375745F3E
:101760006D696E747073007470736171007470735E
:10177000646F747261746500747073646F745F6B0E
:101780007061646F745F636F6E660072706D6B0082
:10179000696E6A70776D3600696E6A70776D740075
:1017A000696E6A70776D00696E6A72616D707570CE
:1017B0005F6261747466616300696E6A6F63667507
:1017C000656C006B70616F666673006B706166615B
:1017D00063006261747466616300696E6A6F70654C
:1017E0006E00616C7465726E61746500646976691F
:1017F000646572007265715F6675656C0077617211
:101800006D75705F72706D5F7363616C6500776199
:10181000726D75705F636C74007761726D75705F67
:10182000636C745F72616E67650061776563006108
:101830007765765F74656D705F7363616C696E6701
:101840000061776576006372616E6B696E675F74C5
:1018500068726573006377680063776C0070726903
:101860006D65705F74656D705F7363616C696E67E1
:10187000007072696D657000004E6676838D969E6D
:10188000A5ABB1B6BBBFC3C7CBCED1D4D7DADCDEF4
:10189000E1E3E5E6E8EAEBEDEEF0F1F2F3F4F5F67C
:1018A000F7F8F9F9FAFBFBFCFCFDFDFDFEFEFEFF7F
:1018B000FFFFFFFFFFFFFFFF03040506804020102E
:1018C0000804020130313233343536373839414279
:1018D00043444546003F3F00457272002E723F73FD
:1018E00091769B76F274CD75A876CC713E70CE70F1
:1018F0000C7131719B71C171C8766577961A8C1A1B
:10190000801A721A641A5E1A521A441A321A2A1A61
:10191000261A1C1A101A041AF819E819E219DA1909
:10192000D019CC19C019BA19B419AE199E19901949
:10193000881980197819701968195E19AC1AA81AD3
:10194000A81AA81A56194E19A81AA81A00005C86D7
:101950004E80538000001A861F864E860000ED845C
:101960002584087ED5830000A384FF7DC17E00000E
:10197000C383FF7DCC830000A983FF7DB683000075
:10198000C582FF7D1D8300009F82FF7D04830000D0
:101990007A827F82FF7D9682FF7D697E00003D8294
:1019A0004282FF7D6682FF7DD57DDA7D00006A85FB
:1019B000FF7D00004F858D8500003685B2850000D3
:1019C0003D824282FF7D7A827F820000D6810000C4
:1019D000B481BF81C881D181000063817581A581F7
:1019E00000003F8144810000F081FF7D9C80FF7DED
:1019F0002481FF7DF1800000FC80FF7D0781FF7D59
:101A000012810000D080FF7DDB80FF7DE68000003A
:101A1000BC80C180FF7DDA7D8B800000A384FF7DC8
:101A2000BC7EC17E000050840000FF8312842584A8
:101A30000000D57DDA7DFF7D29833983FF7D9D7E82
:101A4000A27E0000F081FF7DBC809C808B80FF7DAA
:101A500000001E802380037E3D8242820000DE85DE
:101A6000C4850000D57DDA7DFF7D298331833983EC
:101A70000000F081FF7D6D8672868B808380000080
:101A80001E802380037E4E8061800000097F187FC6
:101A9000FF7DDF7F0000D57DDA7DFF7D167E417EF4
:101AA000FF7D9D7EA27E0000FF7D00006D86728618
:101AB0000000E43DAA3D823D5A3D3D3D093DCC3C00
:101AC000AF3C7F3C00000000000000000000000070
:101AD000000000000000503C00000000000000007A
:101AE00000000000000000000000103CF73BDB3B62
:101AF0009F3B793B543B2B3BFD3ACC3A9E3A643AB0
:101B00002E3AF039B53900008839643900000000F8
:101B100000002E390000000000001F39FF38C838CF
:101B20008B386C3843380A38CD37B2377D373B377E
:101B30000A37D836B6368B367F3659364636333680
:101B40001436FC35DE35B3356C3553352A35013561
:101B5000D834BA349C347F34623432340834DB33C2
:101B6000CF33C333B733AC338F33723335331F3393
:101B70000F33EE32CC320000000000000000000005
:101B80000000000000000000B93292327B32543273
:101B90002F32FB31DC319B316A3141311D31F6305E
:101BA000CE30B7307430513029301A30FA2FDF2F51
:101BB000BA2F942F822F562F2A2FFE2EDD2EB52ED0
:101BC000852E572E382E072EEC2DD82DC42DB02D56
:101BD000902D7E2D6C2D5A2D3C2D072DD92CA42C0B
:101BE000822C752C532C312C242C022CF12BD72B2E
:101BF000AF2B832B5A2B362B0C2BE72ACF2AB72A55
:101C00007D2A382A092ADA29AB297B295029132968
:101C1000DA28992859283B280828C127AF279D276B
:101C200083273C27F526CB2696266C264626222699
:101C3000F625BA257D256525422529250925DD249A
:101C400097246D243B240424EC23BB238D235623AB
:101C50003A232123FF22DC22B82299227A225C2215
:101C60003E221B22F821D721B82199217B215D2119
:101C70003A211721F620D020B620902076205B2034
:101C80004420FD1FC61FA51F911F7D1F691F491FEF
:101C9000241F061FDE1EB01E991E7E1E4E1E1B1E1A
:101CA000E71DA81D8D1D701D361D111DEB1CDB1CB5
:101CB000B41C00004E6F206D6F72652076617269F2
:101CC00061626C652C20676F206261636B2C2064FD
:101CD0006F6E277420746F7563680049676E2053B8
:101CE0006F667472706D2052504D0069676E637537
:101CF000742074696D6520616674657220696E7008
:101D0000757470756C7365205B34206D7365635DED
:101D1000007368696674637574206D637033323064
:101D200038206368616E6E656C2C20646973616233
:101D30006C653A464600626974343A736869667441
:101D4000637574206675656C2C20626974313A7312
:101D50006869667463757420737061726B20626960
:101D600074303A72657663757420737061726B00BB
:101D700064697669646520746865207461636820AD
:101D80007369676E616C206279205820007461630A
:101D900068207369676E616C206F7574707574204C
:101DA0006368616E6E656C0063757420746865208D
:101DB0006675656C2069662074686520656E676964
:101DC0006E65206B7061206578636565647320744F
:101DD0006869732076616C756520307846463D648D
:101DE000697361626C65006675656C637574206209
:101DF000656C6F772074686973204D4150202830DE
:101E0000303A64697361626C653B203130207265E1
:101E1000636F6D6D656E64656429006D6178206126
:101E20006C6C6F776564202B2F2D206D697373693F
:101E30006E6720746F6F74682064657669616E6385
:101E400065205B312F385D2042352F3030006D61C9
:101E50007820616C6C6F776564202B2F2D206E6F5E
:101E6000726D616C20746F6F74682064657669614F
:101E70006E6365205B312F31365D20373600776128
:101E80007465722070756D702C206F757470757428
:101E9000206368616E6E656C007761746572207096
:101EA000756D702C20687973746572657369730041
:101EB0005645206D6F64653A73706565642064658E
:101EC0006E7369747920284D4150292061626F76C4
:101ED00065205B2A3130305D2052504D2000564540
:101EE000206D6F64653A616C7068612D6E202854B6
:101EF0005053292062656C6F77205B2A3130305D4A
:101F00002052504D200077617465722070756D709D
:101F10002C2073746172742074656D7065726174C5
:101F200075726500626F6F7374636F6E74726F6C3D
:101F300020736F6C656E6F6964206F757470757453
:101F4000206368616E6E656C00626F6F7374636F9F
:101F50006E74726F6C2070696420696E746567724C
:101F6000616C206C696D697400626F6F7374636F6C
:101F70006E74726F6C20706964206B6400626F6FA6
:101F80007374636F6E74726F6C20706964206B6918
:101F900000626F6F7374636F6E74726F6C20706920
:101FA00064206B70006163747561746F72204F46BA
:101FB000462062656C6F7720746869732070726563
:101FC000737375726500626F6F7374636F6E747292
:101FD0006F6C20746172676574206F6666736574D8
:101FE000206170706C69656420616674657220623E
:101FF0005B52504D5D2A745B5450535D00626F6FAD
:102000007374636F6E74726F6C20626974373A34E4
:102010002050574D20706572696F64205B386D7376
:1020200065635D3B20626974333A62697432207281
:102030006566706F733B206269743020303A626F5E
:102040006F737400414C5320544B53206F75747060
:102050007574206368616E6E656C0045475420633B
:10206000616C6962726174696F6E206D756C746900
:10207000706C6965720052504D20737769746368A3
:10208000206F7574707574206368616E6E656C0086
:1020900052504D207377697463682052504D2074FC
:1020A00068726573686F6C64202846463D64697386
:1020B00061626C652900574F5420737769746368B7
:1020C000206F7574707574206368616E6E656C0046
:1020D000574F54207377697463682052504D2074B1
:1020E00068726573686F6C64202846463D64697346
:1020F00061626C6529006D697363326F75742C6F52
:102100007574707574206368616E6E656C2073659C
:102110006C6563746F72006D697363326F75742CD4
:102120006D6178696D756D206D616E69666F6C6447
:10213000207072657373757265006D697363326FB9
:1021400075742C6D696E696D756D206D616E696653
:102150006F6C64207072657373757265006D69735E
:1021600063326F75742C6D6178696D756D20747054
:102170007320706F736974696F6E006D6973633279
:102180006F75742C6D696E696D756D207470732038
:10219000706F736974696F6E006D697363326F7508
:1021A000742C6D6178696D756D2072706D205B3176
:1021B00030302072706D5D006D697363326F7574BD
:1021C0002C6D696E696D756D2072706D205B31309C
:1021D000302072706D5D006D697363316F75742CA2
:1021E0006F7574707574206368616E6E656C2073B2
:1021F000656C6563746F72006D697363316F7574BC
:102200002C6D6178696D756D206D616E69666F6C9E
:1022100064207072657373757265006D69736331E4
:102220006F75742C6D696E696D756D206D616E6969
:10223000666F6C64207072657373757265006D698A
:102240007363316F75742C6D6178696D756D207471
:10225000707320706F736974696F6E006D6973635A
:10226000316F75742C6D696E696D756D2074707346
:1022700020706F736974696F6E006D697363316F7D
:1022800075742C6D6178696D756D2072706D205B51
:102290003130302072706D5D006D697363316F7520
:1022A000742C6D696E696D756D2072706D205B3177
:1022B00030302072706D5D00526576206C696D69FA
:1022C00074207768656E20414C5320616374697691
:1022D00065205B3130302072706D5D00616C732C55
:1022E0006D61782069676E2E20726574617264205A
:1022F0005B312F34206372616E6B6465675D0061D2
:102300006C732C7377697463686F66662065677495
:10231000205B35206465672063656C736975735D48
:1023200000616C732C7377697463686F66662074E0
:10233000696D65205B7365635D00616C732C7377F9
:10234000697463686F66662072706D205B3130302F
:102350002072706D5D007365636F6E6461727920C9
:10236000696E6A6563746F7273206F70656E206149
:10237000626F766520676976656E206D616E69664D
:102380006F6C64207072657373757265007365633A
:102390006F6E6461727920696E6A6563746F7273BF
:1023A000206F70656E2061626F7665206769766563
:1023B0006E207468726F74746C65007365636F6E01
:1023C0006461727920696E6A6563746F72732072DA
:1023D00061746520746F2063616C63756C617465F2
:1023E00064207077205B302E34255D006675656C47
:1023F00070756D70206F7574707574206368616E90
:102400006E656C006D696E696D756D2074696D65C2
:1024100020746F206C65617665206675656C7075DB
:102420006D70206F6E2061742073746172747570AA
:10243000205B3236326D7365635D007475726E2099
:102440006F6666206675656C70756D702061667468
:10245000657220696E616374697669747920746944
:102460006D65205B3236326D7365635D00685B328B
:102470005D206D6178696E64657820666F72206991
:10248000676E6974696F6E206368616E6E656C203B
:102490006C6F6F6B757000454449533A3078303F2C
:1024A0002064756D6D793A203078373F2064697308
:1024B00061626C653A3078666620626974313A20F0
:1024C00069676E5F6475616C5F6F757420626974B3
:1024D000303A20696E766572746F75740069676E44
:1024E0006974696F6E20616476616E6365206174E2
:1024F000206372616E6B696E67205B302E323563CC
:1025000072616E6B6465675D00616464656420641C
:1025100077656C6C2074696D652061742036562077
:102520002832377573656329006477656C6C2061A8
:10253000626F7665203134562028363475736563B2
:1025400029005444432061667465722074686520D4
:102550007472696767657228302E356372616E6BBD
:102560006465672900656E6770686173652C207704
:1025700068656E20746F2072657365740063616DA9
:102580002073796E632C2066616C6C696E672065C0
:102590006467652C20656E67696E6520706861737D
:1025A00065206174206E657874207072696D617247
:1025B0007920747269676765720063616D20737951
:1025C0006E632C20726973696E6720656467652C81
:1025D00020656E67696E652070686173652061743F
:1025E000206E657874207072696D617279207472E2
:1025F000696767657200746F6F74682077686565D6
:102600006C2C20616E67756C6172207769647468E8
:10261000206F66206D697373696E6720746F6F74C5
:102620006800746F6F746820776865656C2C206132
:102630006E67756C6172207769647468206F6620BC
:10264000746F6F7468004372616E6B74696767655D
:102650007220706572696F64206D696E696D756D49
:1026600020282A313620757365632900746F6F74D2
:102670006820776865656C2C20646566696E6520E6
:10268000616E6F7468657220747269676765722025
:10269000746F6F746800746F6F7468207768656515
:1026A0006C2C206163746976652074726967676554
:1026B0007220746F6F7468202830303A6D697373BC
:1026C000696E6720746F6F74682900746F6F746827
:1026D00020776865656C2C206E756D626572206F61
:1026E00066207465657468206F6E20746865207755
:1026F0006865656C0074726967676572322C206268
:1027000069743020303A66616C6C696E672F313ABB
:10271000726973696E672C206269743120303A6582
:102720006E61626C652F313A64697361626C652C0D
:10273000206269743220313A66696C00747269678C
:10274000676572312C206269743020303A66616CA2
:102750006C696E672F313A726973696E672C2062FB
:1027600069743120303A746F6F7468776865656C8E
:102770002F313A636F696C2C206269743220303AD1
:102780006E6F004C43442C2064656661756C742048
:1027900072756E74696D65207669657700414C537A
:1027A00020726574617264206D6178747073004189
:1027B0004C5320726574617264206D696E7470731D
:1027C0000069676E6974696F6E2062616C616E6327
:1027D00065205B302E32356372616E6B6465675DB8
:1027E0002C2064656475637465642066726F6D2067
:1027F000616476616E636520746F206D6F7665200D
:102800007A65726F20706F00626974372D343A20D8
:102810006B70616661635F756E69742C20626974A8
:10282000332D303A206B70615F636F6E6669675F4E
:102830007265736F6C7574696F6E004C43442062EF
:1028400061636B6C696768743A204646206973203F
:1028500066756C6C79206F6E004C43442D63616229
:102860006C656C656E6774682064656C6179732053
:1028700048696768657268616C663A6265666F721E
:1028800065454E61626C65204C6F77657248616C7E
:10289000663A454E61626C65004C434420666C614B
:1028A000677320343A207377206272696768746EA8
:1028B00065737320333A7265696E697420313A6CBE
:1028C00063645F65617379676F746F20303A627516
:1028D0007379706F6C6C656420005645206C65617F
:1028E000726E2C20636F6E6669672C20626974308B
:1028F0003A656E61626C6520626974313A73696D24
:10290000756C61746520626974323A203278326283
:102910006F78005645206C6561726E2C206D617871
:1029200020646576696174696F6E20282B2F2D20D5
:102930005B302E34255D292066726F6D20726566CE
:102940006572656E6365205645207461626C650032
:102950005645206C6561726E2C207370656564202D
:102960006F66206368616E67657320746F2074689A
:1029700065205645207461626C65005645206C6583
:1029800061726E2C206D696E696D756D2077656959
:1029900067687420666F72206D6F64696679696E0E
:1029A0006720564520656E747279005645206C6527
:1029B00061726E2C2065676F207363616C696E674E
:1029C00020666163746F722028735E32203C20326F
:1029D00035352F7363616C6529005645206C656140
:1029E000726E2C206B7061207363616C696E67205E
:1029F000666163746F722028735E32203C2032352A
:102A0000352F7363616C6529005645206C656172D2
:102A10006E2C2072706D207363616C696E67206626
:102A20006163746F722028735E32203C203235352A
:102A30002F7363616C6529005645206C6561726E69
:102A40002C206175746F206D6F64696669636174B1
:102A5000696F6E206F6620564520656E747279200E
:102A60006F6E6C792062656C6F7720706F7765721E
:102A70003D6D61702A72706D2F32353600564520DB
:102A80006C6561726E2C206D696E20636F6F6C6176
:102A90006E7420666F72206175746F206D6F64694B
:102AA0006669636174696F6E206F662056452065A4
:102AB0006E7472696573006B6E6F636B2C206D6151
:102AC000782072706D205B31303072706D5D006BFC
:102AD0006E6F636B2C206D696E2072706D205B31A0
:102AE000303072706D5D006B6E6F636B2C206967A8
:102AF0006E6974696F6E20616476616E63652064CF
:102B0000656C6179205B31356D735D006B6E6F6351
:102B10006B2C2069676E6974696F6E2061647661E1
:102B20006E63652073746570205B312F342064659B
:102B3000677265655D006B6E6F636B2C2069676EF5
:102B40006974696F6E207265746172642064656C6B
:102B50006179205B31356D735D006B6E6F636B2C3B
:102B60002069676E6974696F6E2072657461726442
:102B70002073746570205B312F3420646567726543
:102B8000655D006B6E6F636B2C2064656661756CB0
:102B9000742069676E6974696F6E20726574617202
:102BA00064205B312F34206465677265655D006B5E
:102BB0006E6F636B2C206D61782069676E69746934
:102BC0006F6E20726574617264205B312F342064F3
:102BD00065677265655D006B6E6F636B2C206E6F51
:102BE000697365207363616C6520666163746F72DD
:102BF000006B6E6F636B2C207468726573686F6C0A
:102C000064006B6E6F636B322C20696E7465677243
:102C10006174696F6E2074696D6520636F6E737483
:102C2000616E74006B6E6F636B322C206761696E2E
:102C3000006B6E6F636B322C2062616E6470617327
:102C4000732063656E746572206672657175656E5A
:102C50006379006B6E6F636B312C20696E746567EE
:102C6000726174696F6E2074696D6520636F6E7335
:102C700074616E74006B6E6F636B312C20676169D9
:102C80006E006B6E6F636B312C2062616E647061DD
:102C900073732063656E7465722066726571756505
:102CA0006E6379006B6E6F636B2C2073616D706C5B
:102CB000696E672077696E646F77205B3420646586
:102CC000677265655D206C656E6774683A737461E0
:102CD0007274284154444329006B6E6F636B2C203F
:102CE000636F6E6669672E206269743020313A65C1
:102CF0006E61626C6520626974313A20303A6368B3
:102D0000616E6E656C300077626F322C20526920E4
:102D1000636F6E666964656E6365207363616C6979
:102D20006E6720666163746F722028735E32203C88
:102D3000203235352F7363616C65290077626F32FD
:102D40002C2070756D702070696420696E746567E1
:102D500072616C206C696D69740077626F322C202F
:102D600070756D7020706964206B640077626F32DB
:102D70002C2070756D7020706964206B690077621B
:102D80006F322C2070756D7020706964206B70003C
:102D900077626F322C206865617465722070696497
:102DA00020696E74656772616C206C696D6974006E
:102DB00077626F322C206865617465722070696477
:102DC000206B640077626F322C20686561746572D5
:102DD00020706964206B690077626F322C2068650F
:102DE0006174657220706964206B700077626F3265
:102DF0002C2063616C6962726174696F6E20636F0D
:102E00006E7374616E740077626F322C2070756D12
:102E100070207A65726F20647574796379636C656C
:102E2000202864656661756C743A20363629205B0B
:102E300035562F3235365D0077626F322C20746143
:102E400072676574206E65726E73744443205B35DF
:102E5000562F3235365D0077626F322C20746172E6
:102E6000676574205269202870756C736520616DE8
:102E7000706C69747564653A4333295B35562F3439
:102E80003039365D0077626F322C20736D616C6C67
:102E90006572206564676574696D6573206172652C
:102EA000206E65676C6563746564205B302E3575D4
:102EB0007365635D0077626F322C206564676574AB
:102EC000696D6520636F7272656374696F6E2063EC
:102ED0006F6E7374616E7420432F52200077626F9F
:102EE000322C20726574727920636F6E74726F6C0D
:102EF000206166746572205B347365635D00776280
:102F00006F322C2066616C6C6261636B20562061AD
:102F100066746572206D617874205B31633D313079
:102F2000562066663D3330565D0077626F322C2046
:102F30006D61782074696D65207370656E742061B1
:102F400074206162735F6C696D6974205B32363224
:102F50006D7365635D0077626F322C206865617404
:102F60006572206162736F6C757465206C696D6940
:102F700074205B32613D3132562066663D333056F7
:102F80005D00414C532074707320746872657368DF
:102F90006F6C640077626F322C207761726D757090
:102FA0002072616D70207370656564205B33663DCF
:102FB000302E32562F7365635D0065676F2C206D70
:102FC000696E696D756D2077696E646F7720666FC5
:102FD000722070696420746F20726561637400658B
:102FE000676F2C2074617267657420766F6C7461F2
:102FF000676520284E424F32290065676F2C207389
:103000007465702073697A65202870657263656ED7
:103010007429205B302E34255D00414C5320656EB1
:10302000726963686D656E740065676F2C20696EE8
:103030006372656469626C65207370656564206C99
:10304000696D697420286F7220706964206B702923
:103050000065676F2C206D61782070657263656E06
:103060007420746F2072696368206166725B302E11
:1030700034255D0065676F2C206D61782070657266
:1030800063656E7420746F206C65616E206166727A
:103090005B302E34255D28696E2053494E474C45E0
:1030A0005F544152474554206D6F646520726963D7
:1030B0006820746F6F290065676F2C207761726DCF
:1030C00075702074696D65205B7365635D0065676D
:1030D0006F2C206D61782072706D20666F72204FAA
:1030E0003220636F7272656374696F6E205B31307A
:1030F0003072706D5D0065676F2C206D696E207297
:10310000706D20666F722065676F20656E61626CFE
:10311000696E67205B31303072706D5D0065676F7E
:103120002C206D6178206D617020666F72204F32A7
:1031300020636F7272656374696F6E5B6B50615D63
:103140000065676F2C206D61782074707320706F3C
:10315000736974696F6E20666F722065676F206394
:103160006F7272656374696F6E0065676F2C206D96
:10317000696E20636F6F6C616E742074656D70652D
:1031800072617475726520666F722065676F206565
:103190006E61626C696E675B465D0065676F2C20CF
:1031A00074696D65636F6E7374616E742028656EEB
:1031B00067696E65206379636C65732920666F7239
:1031C000206368616E67696E6720636F7272656302
:1031D00074696F6E20666163746F720065676F2C2F
:1031E00020626974353A4E424F325F616463372022
:1031F000626974303A5049442020006961632C2090
:103200007468726573686F6C6420666F72206163A6
:103210007469766174696E672061697220636F6E8C
:1032200074726F6C205B302E32356465675D0069A7
:1032300061632C2069676E6974696F6E20726574B2
:10324000617264206C696D6974205B302E32356464
:1032500065675D006961632C2069676E6974696FD9
:103260006E20616476616E6365206C696D6974209F
:103270005B302E32356465675D200049676E697486
:10328000696F6E20536F667452504D2072616E6785
:1032900065006961632C2069676E6974696F6E20CF
:1032A000616476616E6365205B302E3235646567DC
:1032B0002F32353672706D5D00696163206F7574F1
:1032C000707574206368616E6E656C006961632C53
:1032D000207265666572656E636520706F736974D0
:1032E000696F6E2028666E2074656D7029006961B3
:1032F000632C207365636F6E6473206265747765F9
:10330000656E206F766572636C6F73696E670069B6
:1033100061632C20637574206D617874707300692B
:1033200061632C206465616462616E64205B31209E
:1033300072706D5D006961632C20696E74656772DF
:10334000616C206465616462616E64205B3120722F
:10335000706D5D20286265696E67207465737465A1
:103360006420666F722075736566756C6E65737325
:1033700029006961632C20696E74656772616C2035
:10338000696E637265617365206C696D697400694B
:1033900061632C20696E74656772616C206465637B
:1033A0007265617365206C696D6974004C61756E3E
:1033B00063682052504D006961632C20442D746570
:1033C000726D006961632C20492D7465726D00690E
:1033D00061632C20502D7465726D006961632C202F
:1033E0006163747561746F722061646A7573746D62
:1033F000656E742073706565642F70776D206672DA
:10340000657175656E6379006961632C20647572FE
:103410006174696F6E206F66206166746572737483
:103420006172742072706D205B302E312073656381
:103430005D006961632C20616674657273746172EA
:10344000742072706D205B31302072706D5D2C20A5
:10345000616464656420746F2069646C65207270B7
:103460006D006961632C206372616E6B20706F73F5
:103470006974696F6E2061742031373020460069AD
:1034800061632C206372616E6B20706F7369746965
:103490006F6E206174202D34302046006961632CEA
:1034A0002069646C652072706D20287761726D29C7
:1034B000205B31302072706D5D006961632C206982
:1034C000646C652072706D2028636F6C6429205BCA
:1034D00031302072706D5D006961632C206D696E02
:1034E0002074656D706572617475726520666F72A7
:1034F000207761726D2069646C6520737065656406
:10350000006961632C206D61782074656D7065724F
:10351000617475726520666F7220636F6C642069D8
:10352000646C65207370656564006961632C206557
:103530006E67696E652E7470732076616C75652098
:10354000666F722069646C65207468726573686F59
:103550006C64006961632C206D6178207374657000
:103560007320746F20657874656E64006961632CE4
:1035700020626974373A736F667469646C6520629F
:103580006974363A6173796D20626974353A64758D
:10359000616C736F6C20626974343D313A69676E97
:1035A000616476204F4E2C20626974333A707265E4
:1035B0006369006961632C207374657070696E675C
:1035C0002073657175656E63652028646566696E34
:1035D000652069616320776972696E672900636F8E
:1035E0006F6C616E742066616E2C206F75747075DF
:1035F000742073656C656374696F6E00636F6F6CC4
:10360000616E742066616E2C2068797374657265D2
:1036100073697300636F6F6C616E742066616E2CEA
:103620002073746172742074656D70657261747555
:103630007265007470732C206D6178206164632D55
:10364000636F756E74007470732C206D696E2061E9
:1036500064632D636F756E74006D617820646966B4
:10366000666572656E636520696E206261726F6D5A
:103670006574726963207072657373757265004159
:103680004C53206D617820637574004661737469D2
:10369000646C652076616C7665206F666620616279
:1036A0006F766520746869732054656D705B2E2E8B
:1036B000462D34305D0056426174742063616C693C
:1036C00062726174696F6E20617070722E42433D48
:1036D00064656661756C74006331332C20626974B3
:1036E000333A6261726F20626974323A616C706859
:1036F000616E20626974313A57424F3220626974B8
:10370000303A6F646466697265006331322C2062FE
:103710006974372D343A696E6A6E756D206269740A
:10372000332D323A4D415474797065206269743199
:103730002D303A434C5474797065006331312C203C
:10374000626974372D343A6E63796C2D3120626969
:1037500074333A54424920626974323A3273747253
:103760006F6B6520626974303A303D6D707834312A
:1037700031352F313D6D7078343235300046616B14
:10378000652061697264656E73697479206C6F7706
:10379000206C696D697420286C6F772072706D20C1
:1037A0006F6E6C79292C20303D3D64697361626CC9
:1037B0006500526576206C696D69742028686172B5
:1037C0006429205B3130302072706D5D004F76656A
:1037D0007272756E206675656C726573756D652C99
:1037E00020696E6A6563746F7273207265656E61BD
:1037F000626C65642062656C6F7720746869732001
:103800005B3130302072706D5D004F76657272757D
:103810006E206675656C6375742C20696E6A6563CD
:10382000746F72732064697361626C656420616295
:103830006F76652074686973205B31303020727058
:103840006D5D006C61756E63682C206669786564D7
:103850002069676E2E20726574617264205B312F5F
:1038600034206372616E6B6465675D006C61756EB8
:1038700063682C206675656C20656E726963686D7F
:10388000656E74205B302E34255D00436F6C6420C0
:10389000616363656C65726174696F6E20616464F5
:1038A000656420616D6F756E7420286174202D34FD
:1038B000302046206465677265657329205B31306E
:1038C0003020757365635D00416363656C6572618B
:1038D00074696F6E20636F6C64206D756C746970B1
:1038E0006C69636174696F6E20666163746F722CBA
:1038F0002062696173656420617420313030004159
:103900006363656C65726174696F6E206475726162
:1039100074696F6E205B302E31207365635D0041EA
:103920004C5320637574206D696E7470730054502D
:10393000532F4D4150444F5420616363656C657251
:103940006174696F6E20616D6F756E742028666E8C
:1039500020545053444F5429205B3130302075732C
:1039600065635D005450532F4D4150444F542061C6
:103970006363656C65726174696F6E2062696E73F2
:103980002C2064762F647400303A20545053444FF6
:10399000542C20313A204D4150444F5420616363F0
:1039A000656C65726174696F6E20656E72696368BB
:1039B0006D656E7400436F6E7374616E7420666F14
:1039C000722063616C63756C6174696E672C207220
:1039D000706D203D2031322C3030302F6E63796C89
:1039E0002028303A20686967682062797465290068
:1039F000616464656420496E6A6563746F72205007
:103A0000574D2064757479206379636C6520647503
:103A100072696E67206C6F77206261747465727969
:103A200020766F6C74616765202836562900496ED0
:103A30006A6563746F722050574D2074696D6520FC
:103A4000617420776869636820746F2061637469AA
:103A5000766174652070776D205B3130302075732E
:103A600065635D00496E6A6563746F722050574DDF
:103A70002064757479206379636C652028776865A4
:103A80006E2063757272656E74206C696D697469FD
:103A90006E67206973206163746976652900696EB9
:103AA0006A6563746F722072616D70757020736CDB
:103AB0006F706520626174746572792064657065E9
:103AC0006E64656E6365202846462900696E6A65E6
:103AD00063746F72206F70656E696E6720656666CD
:103AE0006563746976652072616D707570207469A4
:103AF0006D65205B323420757365635D004D415008
:103B0000207369676E616C206F66667365742065EB
:103B1000672E30784138202D33322E2E2B33326BE6
:103B20005061205B32353050615D004D4150207254
:103B3000616E6765205B326B50615D20303A2075A5
:103B4000736520412F42206C6F6F6B75702074611C
:103B5000626C6500426174746572792067616D6D95
:103B60006120666163746F72205B31362075736506
:103B7000632062617365645D00496E6A6563746F9A
:103B800072206F70656E2074696D652061742031DC
:103B9000332E3256205B313620757365635D0041EC
:103BA0006C7465726E61746520696E6A6563746FAA
:103BB0007220647269766572732C20626974342095
:103BC000313A62617463682066697265207768655E
:103BD0006E206372616E6B696E670049525120649A
:103BE000697669646520666163746F7220666F72BE
:103BF0002070756C7365004675656C20636F6E731D
:103C000074616E7420287265715F6675656C290039
:103C10005761726D757020656E726963686D656E4F
:103C200074207363616C65722061742068696768D1
:103C30006573742072706D2062696E3A2046463D4D
:103C400072706D20696E646570656E64656E740077
:103C50005761726D757020656E726963686D656E0F
:103C6000742062696E7328666E2074656D70292CED
:103C700020626961736564206174203130300057BF
:103C800061726D75702074656D70657261747572A6
:103C9000652072616E6765206F662062696E7320B1
:103CA000282B34302046206F6666736574290041E6
:103CB0006674657273746172742074696D6520280E
:103CC00036206372616E6B72657629004166746599
:103CD000727374617274207761726D757020736392
:103CE000616C696E67206174203137304620283856
:103CF000303D68616C662C2066663D73616D6520A1
:103D0000617320636F6C642900416674657273741B
:103D1000617274207761726D757020656E7269636F
:103D2000686D656E74202870657263656E742C20F2
:103D300061646465642076616C7565290043726115
:103D40006E6B696E67207468726573686F6C64204F
:103D50005B3130302072706D5D004372616E6B6953
:103D60006E672070756C73657769647468205B3169
:103D7000303020757365635D2061742031373020E9
:103D800046004372616E6B696E672070756C736577
:103D90007769647468205B31303020757365635DCA
:103DA000206174202D34302046005072696D696E98
:103DB000672070756C7365207363616C696E672032
:103DC0006174203137302046202838303D68616CDE
:103DD000662C2066663D73616D6520617320636F9C
:103DE0006C6429005072696D696E672070756C7320
:103DF00065206174202D34302046205B3130302026
:103E0000757365635D00562E452E4D2E532E00466C
:103E100069726D776172653A2000312E302E33362B
:103E200000205570646174696E67204669726D7711
:103E3000617265200052504D3A0020200020202061
:103E4000202000540050004F32253D003F3F2E3FC0
:103E5000004C613A004F323A302E0065676F433AAA
:103E60000065676F433A00636C743A0020747073A6
:103E70003A0070773A006D617800706F733A2000F5
:103E80006469723A20006961633A00206163746971
:103E900076650020202020202020005645206C65DB
:103EA00061726E3A002061637469766500207369FF
:103EB0006D0064633A006164763A003F3F006477C6
:103EC000656C6C3A00446164763A20200044647763
:103ED000656C6C3A0052693A004E65726E73743AC2
:103EE00000486561743A0050756D703A00204F4E7D
:103EF000004F4646004146523D004146523D005368
:103F00003A00204C3A00443A00523A00206B613AA1
:103F10000020643A200020433A0047616D65206F1D
:103F20007665722C20696E73657274203120457538
:103F3000726F20746F20706C617920746865202224
:103F400074756E652D7468652D656E67696E652084
:103F500067616D652220616761696E2E2E2E006299
:103F60006F6F7374205467742000204D41500065BA
:103F700067743A0074630020706F733D00207661AF
:103F80006C3D0000F900F5F3F1F2FC00FAF8F6F4EC
:103F900009A70000A20000A151210000005A5341CE
:103FA0005722000043584445A4230000205646549D
:103FB000522500004E42484759260000004D4A5500
:103FC0002F2800003B4B494F3D2900003A5F4CD859
:103FD000503F000000C600C560000000000D5E00FC
:103FE0002A0000003E0000000008000031003437C5
:103FF000000000302C323536380100FB2B332D2ADF
:1040000039000000F900F5F3F1F2FC00FAF8F6F4DB
:10401000097C0000A20000A171310000007A7361E8
:10402000773200006378646534330000207666746C
:10403000723500006E62686779360000006D6A753F
:10404000373800002C6B696F303900002E2D6CF86A
:10405000702B000000E600E55C000000000DA800E9
:10406000270000003C000000000800003100343749
:10407000000000302C323536380100FB2B332D2A5E
:10408000390000312E302E33360A004D6F6E204637
:1040900065622032372031313A31393A35342043A4
:1040A000455420323030360A0048656C6C6F3E0D46
:1040B0000A004F4B0D0A004F4B0D0A004D454E555F
:1040C0005F63616E004279650D0A005965732C20AB
:1040D0006D656E7520616E6420636F6D6D20776F06
:1040E00072780D0A004F4B0D0A004F4B0D0A004429
:1040F0004BB045E240B23C0539C335DB323F30E5D9
:104100002DC22BD02909286626E5248023362202D9
:104110002100376C9ECDFAFBFBFCFCFDFDFEFEFF93
:10412000FFA728AC29AF2AB42BBF2CD52DFD2E40DC
:1041300030AA314633283561370B3A423D2941E9EF
:1041400045B34BC052555B0000003F02103B032DAE
:104150001502020011241FBECFEFD0E1DEBFCDBF9C
:1041600011E0A0E0B1E0E8E8FCE801E00BBF02C02C
:1041700007900D92AA33B107D9F71AE0AAE3B1E08C
:1041800001C01D92AB3DB107E1F70C94B8220C942D
:1041900000000F931F93CF9380911E07C0911D07BE
:1041A000883010F4C23030F4809164038B778093B0
:1041B000640387C0E82FFF27EE0FFF1FE85AF54F73
:1041C000008111810E949DB98091640399278370B9
:1041D0009070039779F080916403992783709070B1
:1041E0000297A1F10058114008F46BC0809164035C
:1041F0008360DDCF0F3F110508F063C08091640339
:104200008150809364032C2F332721FF05C0009138
:10421000640304600093640324FF05C010916403E9
:10422000106810936403E0915108F09152087E2FBA
:104230006627A0914F08B09150082B2F3327622B8F
:10424000732B70931102609310023BC030911F07D3
:10425000432F5527FA01EE0FFF1FEE0FFF1FA0910E
:104260005108B09152083A2F222760914F0870915F
:104270005008872F9927282B392B80911002909175
:104280001102B901681B790B6E177F07D0F0440F3C
:10429000551F440F551F440F551F4617570750F41D
:1042A00030931102209310024091640348774093A9
:1042B000640398CF8E0F9F1F90931102809310027A
:1042C000F3CFCF911F910F91089580910A0283FF40
:1042D00011C085B38F70806B85BB9798979A20919A
:1042E0000A0224FF11C085B38F70806A85BB97983E
:1042F000979A089585B38F70806385BB9798979A36
:1043000020910A0224FDEFCF85B38F70806285BBB8
:104310009798979A08959FEF9BBB9ABBA1E0A8BB83
:1043200077EF77BB64E065BB94BB50EE52BB4BEEBE
:1043300041BB13B83AE332B91092620010926100A7
:104340002CE1209365008FE1809364008998919A15
:104350008898909A8091E90680FF8DC050E840913E
:10436000EA064F5F01F181FD88C04150E42FFF272D
:10437000E256FC4F8089F5B3FF709927829592959C
:10438000907F9827807F9827852BF82BF5BBE091AD
:104390006500EB7FE0936500B0916500B460B09379
:1043A0006500442311F70E945D6C6EE179E080E0C6
:1043B0000E945A8B10920A020E949B430E94AA7983
:1043C0000E94103460E08EE199E00E9499998CE49B
:1043D00099E00E9437AA89E299E00E9437AA0E94D8
:1043E000D14480E00E940C448091D9069927880F1F
:1043F000991F880F991F8093E2080E94102A0E943B
:10440000CE3C0E94FB3B10923B0334E130933C03D3
:1044100010923D0310924B034FEF5FEF6FEF7FEF72
:1044200040934703509348036093490370934A03B2
:1044300010924E0310924D0321E0209361031092DD
:1044400062031092510380914D0680FF4EC020916F
:104450003F03309140038091D50699278F7090706B
:10446000029709F44CC083E02C3F380708F440C0A1
:104470008FEF90E04CC050E072CF4150E42FFF2707
:10448000E256FC4FA089E5B3EF708A2F99278295F9
:104490009295907F9827807F9827852BE82BE5BB06
:1044A000F0916500FB7FF0936500B0916500B4600A
:1044B000B0936500A15075B37F708A2F99278295BC
:1044C0009295907F9827807F9827852B782B75BBB6
:1044D000609165006B7F60936500909165009460CA
:1044E00090936500442349F65ECF809145030FC049
:1044F0003695279536952795822F992708C03695AA
:1045000027953695279536952795822F992780935D
:1045100046034091E806409352030E9436BA2BE0CE
:10452000209384010E942B2A0E9415B10E94DA3444
:104530000E9422AC0E94235F0E94A0400E94FA9435
:1045400063E083E199E00E9499990E9444950E945A
:1045500005B80E9416B80E9463B90E9441BA8AE069
:104560008093140251E0509313020E948BBF089570
:10457000CFEFD0E1DEBFCDBF0E94F77A0E948B2142
:104580000E94CB3F0E9492BF0E949C7978940E9427
:10459000FB3B0E9469480E94A2490E94DB4A80912D
:1045A0000A0283FF15C285B38F70806B85BB979815
:1045B000979A00910A0204FF15C285B38F70806A32
:1045C00085BB9798979A10913C0310FD15C20E94E5
:1045D00049350E94E84E30914B03332321F140913D
:1045E0003C0344FF07C090914B0350912606591796
:1045F00008F0A2C360913B0361FD67C37091840121
:10460000713009F469C30E943E4D80911E07C0912C
:104610001D07883018F4C23008F06BC38091640322
:104620008B77809364030E946A350E948F3D0E94BD
:10463000294F0E94FD390E945D3B0E944DBD0E94A2
:10464000B9BB10911802112309F0F7C20E9474B18E
:104650008091170281FF23C08D7F80931702909174
:10466000620691FFEDC20E94AF7C70913B0370FF28
:1046700007C080918401823018F0815080938401BA
:10468000F894E0913C03E5FF09C0B0915103BF3FAE
:1046900029F0C0915103CF5FC09351037894F894EF
:1046A00000914F08109150084CB55DB550935008DB
:1046B00040934F084017510748F48091510890915A
:1046C000520801969093520880935108CA01789439
:1046D0002091850130918601821B930B61E6883A17
:1046E000960708F4AFC08155934C08F400C250936C
:1046F0008601409385010E94803620914503F09108
:10470000A306F21710F0819B04C0F8941092510395
:10471000789460915108709152089B014427552765
:104720008091550890915608A0915708B09158086B
:10473000CD01AA27BB27281B390B4A0B5B0B8091A5
:10474000EB069927AA27BB2782179307A407B5076B
:1047500098F58091EC0699278617970768F5F894E5
:104760008091E90680FF64C250E84091EA064F5FFD
:1047700001F181FD4BC14150E42FFF27E256FC4F70
:10478000808915B31F70992782959295907F9827FD
:10479000807F9827852B182B15BBA0916500AB7FD8
:1047A000A093650060916500646060936500442398
:1047B00011F70E94BA41789480911402815009F057
:1047C0009DC13AE030931402809115029091160237
:1047D0000196909316028093150240911702426051
:1047E0004093170250916D0653FF07C08091D30884
:1047F000882309F40CC20E944B5C90913B0390FF0C
:1048000004C07091D10670FD94C280913A018F5F0F
:10481000843009F450C280933A01F894C0910A029E
:10482000C860C0930A0278948091CE0A8F3F31F01D
:10483000882309F45BC281508093CE0A40914F08CF
:104840005091500880910A078823F1F09927969596
:104850008795782F7877E52FFF272E2F60910D020F
:10486000261B271788F03327A72FBB27AA0FBB1FAC
:10487000A217B3070CF0D8C1E0930D020E943DBE11
:1048800040914F0850915008452F5527842F209173
:104890003D02821B8F30B8F099274F970CF4AAC1C4
:1048A00040933D020E94ACBB0091D60800FD07C0BA
:1048B000F091E807FF2309F4B4C10E94D66C0E946E
:1048C000864B0E94624C0E9438486CE479E08EE18D
:1048D00099E00E94D0AA6EE179E089E299E00E9415
:1048E00004AB0E94B0972091E807222309F4A2C1EB
:1048F00060916D0662FDC2C010917806212F3327AA
:104900002F7330702C5F3F4F3695322F222737950B
:104910002795F894E0914F08F09150086CB57DB55B
:104920007093500860934F086E177F0748F480918A
:104930005108909152080196909352088093510823
:10494000AB017894E0913702F09138024E1B5F0B77
:104950004217530788F08901000F111F041715072C
:1049600008F058C170933802609337020E949A6031
:1049700060914F0870915008472F5527842F209140
:104980001202821B873078F099270F970CF4B9C078
:10499000409312023091620631FFBAC05091530326
:1049A000543009F4BCC080919A0890919B080196FC
:1049B00090939B0880939A080E94FB3B0E94694851
:1049C0000E94A2490E94DB4A80910A0283FDEBCD3E
:1049D00085B38F70806385BB9798979A00910A0280
:1049E00004FDEBCD85B38F70806285BB9798979A55
:1049F00010913C0310FFEBCDF89420913C032E7FE7
:104A000020933C0378940E94103FE1CD4150E42F65
:104A1000FF27E256FC4F108905B30F70812F9927AD
:104A200082959295907F9827807F9827852B082BD9
:104A300005BB209165002B7F2093650030916500B8
:104A4000346030936500115065B36F70812F9927E2
:104A500082959295907F9827807F9827852B682B49
:104A600065BBF0916500FB7FF0936500C091650028
:104A7000C460C0936500442349F69BCE80917806BC
:104A800099278F7390700196F82FEE27F894409134
:104A90004F08509150086CB57DB5709350086093E5
:104AA0004F086417750748F4A0915108B091520857
:104AB0001196B0935208A09351089B0178944091AD
:104AC000370250913802241B350B2E173F0708F48C
:104AD00053CFCF01880F991F8217930708F08EC01C
:104AE00070933802609337020E94A25F41CF28552D
:104AF0003E493093860120938501FDCD80931402B9
:104B000071CE295F209312023091620631FD46CFAB
:104B10000E9490AC50915303543009F044CF20913F
:104B20004703309148034091490350914A03BB2702
:104B3000A52F942F832F8F3F41F1803408F033CF7E
:104B400060914F0870915008E0915F03F09160030D
:104B50006E1B7F0B9B014427552780914703909143
:104B60004803A0914903B0914A03880F991FAA1FD7
:104B7000BB1F82179307A407B50708F014CF072FB0
:104B800011270038110508F00ECFF8948091E9063E
:104B900080FFD5C050E84091EA064F5F01F181FDEA
:104BA00052C04150E42FFF27E256FC4F8089B5B335
:104BB000BF70992782959295907F9827807F98273C
:104BC000852BB82BB5BB709165007B7F709365001A
:104BD00090916500946090936500442311F7789458
:104BE000A091C208B091C3081196B093C308A093D6
:104BF000C208D9CE215F20933D0254CE4E0F5F1FD5
:104C000050933802409337020E94A25FB1CE0E94B7
:104C1000705CF3CDE20FF31FF0933802E09337029C
:104C2000A5CE0E9482864BCE670F60930D0226CEE2
:104C300050E09BCD0E944A675BCE0E94A94306CDFF
:104C40000E942DAC10CD4150E42FFF27E256FC4FBF
:104C5000A089F5B3FF708A2F992782959295907F4E
:104C60009827807F9827852BF82BF5BBC09165008E
:104C7000CB7FC09365008091650084608093650060
:104C8000A150B5B3BF708A2F992782959295907FD6
:104C90009827807F9827852BB82BB5BB709165002E
:104CA0007B7F7093650090916500946090936500A0
:104CB000442349F694CF10923A01F894B0910A0235
:104CC000B77FB0930A027894AFCD0E9453357091AC
:104CD0008401713009F097CC10928401F894A0916E
:104CE0003C03AF7EA0933C0378948DCC0E949ABF86
:104CF000A5CDE82FFF27EE0FFF1FE85AF54F0081E3
:104D000011810E949DB980916403992783709070EE
:104D10000397B9F08091640399278370907002978C
:104D2000E1F10058114008F47ECC80916403836067
:104D300078CC0E94D45969CD0E94C23F64CC50E027
:104D40002ACF0F3F110508F06ECCB0916403B1502B
:104D5000B09364032C2F332721FF05C0C091640357
:104D6000C460C093640324FF05C0F0916403F0683D
:104D7000F09364036091510870915208962F882730
:104D800020914F0830915008032F1127802B912B31
:104D9000909311028093100246CC30911F07632F2D
:104DA0007727FB01EE0FFF1FEE0FFF1FA0915108A9
:104DB000B09152083A2F222780914F0890915008C5
:104DC000492F5527242B352B8091100290911102E9
:104DD000A901481B590B4E175F0708F424CC660F36
:104DE000771F660F771F660F771F6417750750F4DC
:104DF000309311022093100250916403587750931E
:104E000064038FCF8E0F9F1F909311028093100227
:104E1000F3CF0F93CF93DF93801730F5061718F079
:104E2000822F99272CC0681B081BE62FFF27EE0F47
:104E3000FF1FE652F84F65917491FF27EE27609FA0
:104E4000E001709FD00DE11D11248D2F9E2FAF2FFB
:104E5000BB27082F421758F0842F821B809FD00158
:104E600011248B2F9927481B842F992708C0241BB6
:104E7000289FE00111248D2F9927840F9927DF9116
:104E8000CF910F9108950F93CF93DF93742F522FEB
:104E9000302F681728F0801740F0272F332768C07D
:104EA000601760F1252F332763C00617D8F7681BFA
:104EB000381BE62FFF27EE0FFF1FE652F84FA59194
:104EC000B491FF27EE27A39FE001B39FD00DE11D12
:104ED0001124CE01DF01892F9A2FAB2FBB27082F7A
:104EE000421708F43CC0842F821B809F900111243C
:104EF000832F9927781B272F33273AC0081708F0EC
:104F0000CCCF861B361BE82FFF27EE0FFF1FE65284
:104F1000F84FA591B491FF27EE27A39FE001B39F1F
:104F2000D00DE11D1124CE01DF01892F9A2FAB2F67
:104F3000BB27082F241748F0822F841B809F9001E5
:104F40001124832F9927581BADCF721B789FE00146
:104F500011248D2F9927820F282F332709C0541B26
:104F6000589FE00111248D2F9927840F282F332774
:104F7000822F9927DF91CF910F910895CF92DF92E1
:104F8000EF92FF920F931F93CF93DF93EA01A90152
:104F9000801710F09E014BC0061708F048C0681B30
:104FA000081BE62FFF27EE0FFF1FE652F84F8591F3
:104FB0009491FF24EE24809F6001909FD00CE11C0F
:104FC0001124D701C6019601C417D507D0F06E0190
:104FD000C41AD50A44279D9D80018C9D70019C9D1B
:104FE000F00C011D141F8D9DF00C011D141F1124C8
:104FF000A8019701CA01AA27BB279E01281B390BCC
:1050000016C04C1B5D0B8827359F7001249F6001E3
:10501000349FD00CE11CF81E259FD00CE11CF81E1B
:105020001124C701AA27BB279C012C0F3D1FC901D2
:10503000DF91CF911F910F91FF90EF90DF90CF9074
:105040000895CF93DF93841718F080E090E01CC0A0
:105050004617C0F4681BE62FFF27EE0FFF1FE6522E
:10506000F84F65917491481BFF27EE27649FE0017C
:10507000749FD00DE11D11248D2F9E2FAF2FBB27C4
:10508000992702C08FEF90E0DF91CF910895CF93E1
:10509000DF93DC01E90191E020E0822F261780F404
:1050A000282FFD01E80FF11D8081481708F490E0DA
:1050B000822F8F5F861710F4992391F7222319F41A
:1050C0002983288304C0215028832F5F2983DF91FF
:1050D000CF9108959B0199E2899FD0011124EE2779
:1050E000B39FB001A29FA001B29F500D611D7E1F12
:1050F000A39F500D611D7E1F1124529562957295DC
:1051000040EF7627742376276527642365279B0164
:10511000C90108959B019DEC899FC0011124EE27D0
:10512000939FB001829FA001929F500D611D7E1F31
:10513000839F500D611D7E1F1124DB01CA013BE0DE
:10514000B695A795979587953A95D1F70895CF93FA
:10515000DF93FB0169E255274427869F9001969FC4
:10516000300D411D1124232F342F452F5527BB27E8
:10517000AA27E69FC001F69F900DA11D1124892F3B
:105180009A2FAB2FBB276627399FF001289FE0019C
:10519000389FD00DE11DF61F299FD00DE11DF61F90
:1051A00011248D2F9E2FAF2FBB27DF91CF91089514
:1051B000CF93DF9320E8FF27EE27829FE001929FA5
:1051C000D00DE11D1124CE01DF01292F3A2F4B2FE5
:1051D00055275CEDFF27EE27659FE001759FD00DF9
:1051E000E11D1124AE01BF01BB27A72F962F852FEC
:1051F0006627399FF001289FE001389FD00DE11DFF
:10520000F61F299FD00DE11DF61F1124CE01DF01ED
:10521000892F9A2FAB2FBB27DF91CF910895CF9382
:10522000DF9320E1FF27EE27829FE001929FD00DC0
:10523000E11D11242D2F3E2F4F2F552749E2FF2727
:10524000EE27649FE001749FD00DE11D11248D2F86
:105250009E2FAF2FBB276627399FF001289FE001C3
:10526000389FD00DE11DF61F299FD00DE11DF61FBF
:1052700011248D2F9E2FAF2FBB27DF91CF91089543
:10528000FC0131813283208121836083261740F421
:10529000862F321740F4622F861740F4992708951D
:1052A000822F3217C0F3632F8617C0F3862F9927FA
:1052B000089508956817790714F4AB0104C08417A2
:1052C00095070CF0AC01CA01089568172CF4862FDD
:1052D000992787FD9095089584172CF4842F99279A
:1052E00087FD90950895992787FD909508950895D5
:1052F000681718F4862F99270895841718F4842FB7
:1053000099270895992708950895861710F49927E5
:105310000895862F992708950895681710F49927FE
:105320000895862F992708950895CF93DF93EC0170
:10533000942F4F7092959F70E92FFF279F012F5F49
:105340003F4FA62FBB272A173B072CF0AC0FBD1FE2
:1053500011978C911DC0EC0FFD1F5081252F332715
:10536000C0E1D0E0C41BD1092C9FD0012D9FB00D0E
:105370003C9FB00D1124CD012181249FB001112447
:10538000860F971F929582958F7089279F70892726
:105390009927DF91CF910895CF93DF93EC01942F5C
:1053A0004F71929596959770E92FFF279F012F5F78
:1053B0003F4FA62FBB272A173B072CF0AC0FBD1F72
:1053C00011978C911FC0EC0FFD1F5081252F3327A3
:1053D000C0E2D0E0C41BD1092C9FD0012D9FB00D9D
:1053E0003C9FB00D1124CD012181249FB0011124D7
:1053F000860F971F96958795929582958F7089272E
:105400009F7089279927DF91CF91089587708064D5
:1054100087B9369A349BFECF349A84B195B10895FA
:1054200087E886B920E0322F3770306437B9369A72
:10543000349BFECF349A44B155B1E22FFF27EE0FD3
:10544000FF1FE15CFD4F440F551F408351832F5FC9
:10545000283048F3089510923E0220E427B987EFE0
:1054600086B908958770806487B9349A0895E82FC3
:1054700086B19927929582958F7089279F70892789
:105480009C012170307080FF12C0FF27EE0FFF1FBC
:10549000E15CFD4F808191819695879524B135B16E
:1054A000820F931F8083918381E090E00895C9016A
:1054B000089508951F920F920FB60F9211242F9303
:1054C0003F934F938F939F93AF93BF93CF93DF936C
:1054D000EF93FF932091BB09E22FFF27DF01A8572D
:1054E000B64F34B5ED013AA3EE0FFF1FE857F64F64
:1054F00084B195B1808391832F3021F0203140F029
:10550000339806C040913E024770406447B9349AD0
:105510002F5F2093BB09FF91EF91DF91CF91BF9156
:10552000AF919F918F914F913F912F910F900FBE0F
:105530000F901F901895883008F080E08093CE0877
:105540000895DC0120912403422F55274F5F5F4FC0
:105550009A0141505040F901E07FF1702E1B3F0B42
:10556000809191022817B1F0FA01EE0FFF1FEE0FA4
:10557000FF1FEE0FFF1FE40FF51FEE56FD4FA08338
:10558000B18362831382148215822093240380E006
:1055900090E008958FEF90E008950895823138F4F7
:1055A000E82FFF27EE50F64F8491992708958251F6
:1055B000863038F4E82FFF27E050FF4F808199278D
:1055C000089580E090E0089508959927AA27BB27C1
:1055D0008731910590F4FC01E050FE4FEE0FFF1F64
:1055E0000590F491E02D099480E290E0089581E324
:1055F00090E0089582E390E0089586E590E00895B4
:105600008BE690E0089585E490E0089586E590E0CB
:1056100008958091D5060E946D63992708958CE2C4
:1056200090E008958091D5060E94646399270895BB
:105630008DE390E0089581E690E0089580E790E0A2
:1056400008958EE290E0089586E790E0089583E55E
:1056500090E008958DE490E0089588E790E0089543
:1056600080E390E0089508958091150299270895A8
:1056700020E0883078F4E82FFF27EE0FFF1FE85A6C
:10568000F54F808191813FEF8F3F930719F0892F6C
:105690009927282F822F99270895CF93C0E088302B
:1056A00080F4E82FFF27EE0FFF1FE85AF54F019017
:1056B000F081E02D9FEFEF3FF90709F0CE2F0E9418
:1056C0009DB98C2F9927CF910895CF939927AA2719
:1056D000BB2781339105A8F5FC01E95EFD4FEE0F74
:1056E000FF1F0590F491E02D09942091D70827FF22
:1056F00028C0B09124034B2F55274F5F5F4F9A016D
:1057000041505040C901807F9170281B390B609136
:1057100091022617B1F0FA01EE0FFF1FEE0FFF1FE7
:10572000EE0FFF1FE40FF51FEE56FD4F45E65BE25F
:1057300040835183A1E3A2831382148215822093B4
:10574000240380E090E015C220E090911E07309184
:105750001D07E92FFF27EE0FFF1FE85AF54F0190B5
:10576000F081E02D819B20E850913C0355FD2160A4
:10577000809B2064EF3FF10528F4983018F4323014
:1057800008F020627091360371112061F0913B03A3
:10579000F7FDEDC130913C0333FD24604091BA0820
:1057A0005091BB084B30510508F02260822F992799
:1057B000E0C18091840A9927DCC18091810A9927F0
:1057C000D8C180917F0A9927D4C18091800A9927F6
:1057D000D0C180917D0A9927CCC180917E0A9927FA
:1057E000C8C180912F03992788539F4FC8E477271A
:1057F00066278C9FA0019C9F500D611D1124DB0129
:10580000CA0157E0B695A795979587955A95D1F710
:10581000E82FFF27EE0FFF1FE652F84FA591B49136
:1058200077276627AC9FA001BC9F500D611D1124F6
:10583000DB01CA0147E0B695A795979587954A95EC
:10584000D1F78954992795C1C0E08091660A90915B
:10585000670A2FEF8F3F920709F0C82F87E00E9459
:105860009DB98C2F992785C120E08091660A90917F
:10587000670A7FEF8F3F970709F498CF892F992701
:10588000282F822F992775C1C0E080915A0A9091E4
:105890005B0A6FEF8F3F960709F0C82F81E0DFCFDB
:1058A00020E080915A0A90915B0A5FEF8F3F950745
:1058B00029F7822F99275DC120E08091580A9091A5
:1058C000590A3FEF8F3F9307C9F6822F992751C19D
:1058D000C0E08091620A9091630A2FEF8F3F920798
:1058E00009F0C82F85E0BBCFC0E08091580A9091A5
:1058F000590A4FEF8F3F940709F0C82F80E0AFCFD0
:1059000020E08091620A9091630AB3CFA0916A036C
:10591000B0916B0399E277276627A99FA001B99FF1
:10592000500D611D1124DB01CA01CAE0B695A7958F
:1059300097958795CA95D1F799271BC180914D03FB
:1059400090914E03992715C180914D0390914E037C
:10595000892F992799270DC1809129038B3908F048
:10596000E0C08C59992705C180912803992701C16E
:1059700020E08091600A9091610A97CF8091CE07D4
:105980009927F7C08091520386959927F2C080919C
:105990005B0390915C03929582958F7089279F702D
:1059A00089279927E6C080912E039927E2C0E091CC
:1059B0002B03F0912C03B1E177276627EB9FA00121
:1059C000FB9F500D611D1124BB27A72F962F852FFC
:1059D0009C01892F9927892B09F0A3C0822F992731
:1059E000C8C080912A039927C4C0809130039927A9
:1059F000C0C020E08091640A9091650A62CFC0E047
:105A000080915E0A90915F0A2FEF8F3F920709F015
:105A1000C82F83E024CF20E080915E0A90915F0A36
:105A200028CFC0E08091600A9091610A6FEF8F3FAC
:105A3000960709F0C82F84E012CF20E08091660A13
:105A40009091670A32CFC0E08091660A9091670A10
:105A50006FEF8F3F960709F401CFC82FFFCEC0E04C
:105A60008091640A9091650A4FEF8F3F940709F087
:105A7000C82F86E0F4CE8091450399277AC03091F3
:105A8000620631FF51C08091BE09992772C0809192
:105A90003E0399276EC09091270384E6989FB0013A
:105AA0001124872F992787FD9A958E5C992761C0CD
:105AB00080911407882309F448C080914C039927EA
:105AC0000024880F991F001C880F991F001C892F24
:105AD000902D99274EC080914F029091500296953B
:105AE00087959695879596958795992742C0809139
:105AF0003B0399273EC08091150299273AC08091B7
:105B00004203992736C020911407222329F180915E
:105B10004C03880F880F99272CC080914103992747
:105B200028C08FEF90E025C04091930645FF1AC032
:105B300080914D0290914E02969587959695879506
:105B4000969587959927992714C080913F03909146
:105B50004003892F9927FECE80913F039091400307
:105B6000992707C08091410290914202E5CF2860B9
:105B700011CECF910895CF93482F50919102252FA8
:105B80003327F901EE0FFF1FEE0FFF1FEE0FFF1F70
:105B9000E20FF31FEE56FD4F25818481C82FCF7091
:105BA000782F72957F704530B0F4842F992782301A
:105BB000910509F489C08330910534F4009709F008
:105BC0007DC0822F9927F1C08330910509F4DBC095
:105BD000049709F4A6C0403F08F053C063E0F1E029
:105BE000332727FD30952B36310509F472C02C364A
:105BF00031050CF055C02836310509F498C0293616
:105C000031050CF07CC02236310509F487C0A6EFBF
:105C1000B5E0ECE0E69F802D11248B5F481709F476
:105C20008AC0242F3327992701972817390709F4A9
:105C3000A7C0242F2450E79FC00111244F2F5527C0
:105C4000849FF001859FF00D949FF00D1124EA0FC1
:105C5000FB1F03C0261BE40FF51F2617D8F73327B9
:105C60002230310509F43FC023303105ACF5211550
:105C7000310521F02130310509F44BC080E290E07C
:105C800094C0652F7727FB01EE0FFF1FEE0FFF1F5C
:105C9000EE0FFF1FE60FF71FEE56FD4F138291CF59
:105CA0002E36310509F440C02F36310504F52C3667
:105CB000310509F0ACCFA6E6B5E0ABCF019709F00E
:105CC0008ACF8BE590E071C0872F0E946D63992782
:105CD0006CC0A2E0B6E09DCF23303105C9F024307E
:105CE000310561F6319780810E946D63F0CF2437D2
:105CF000310509F08CCFAAE1B6E0E8E08BCF2A3677
:105D0000310509F084CF65E0F2E0A7EBB3E081CF85
:105D1000319780810E946463992747C0AEE0B6E066
:105D200078CF8DE390E041C0A1E2B7E072CFAEE959
:105D3000B3E0E8E06FCF7C1749F17F5FA52FBB2769
:105D4000FD01EE0FFF1FEE0FFF1FEE0FFF1FEA0F0B
:105D5000FB1FEE56FD4F522F4427872F9927829520
:105D60009295907F9827807F9827480F591F4C0F56
:105D7000511D448355838FEE83838AE090E015C0E4
:105D80008DE090E012C08DE590E00FC0252F332705
:105D9000F901EE0FFF1FEE0FFF1FEE0FFF1FE20FC7
:105DA000F31FEE56FD4F8EEFE7CFCF910895CF93BF
:105DB000782FC09191028C2F9927FC01EE0FFF1FC5
:105DC000EE0FFF1FEE0FFF1FE80FF91FEE56FD4FFE
:105DD000A481B5819D012A0F3B1F2B5F354F60E0E9
:105DE00003C0225030406F5FF90145915491411535
:105DF0005105B9F3783F38F5470F511DFA018491E9
:105E0000882309F03CC0662361F42E5F3F4FF901FF
:105E100085919491892B09F058C0AE3FB10508F0E7
:105E200054C04C2F5527FA01EE0FFF1FEE0FFF1F36
:105E3000EE0FFF1FE40FF51FEE56FD4F27EF2383F4
:105E40008BE590E063C0872F99278B3F910591F0F8
:105E50008C3F9105B4F4893F910509F452C08A3F03
:105E600091050CF041C0883F910509F446C08AE7CE
:105E700090E04CC0AE5DB94F8C910E94646399274D
:105E800045C08D3F910509F43FC08D3F91057CF1E0
:105E90008E3F910561F78C2F9927FC01EE0FFF1FB4
:105EA000EE0FFF1FEE0FFF1FE80FF91FEE56FD4F1D
:105EB000A481B5811196A483B583AF3FB10510F4D9
:105EC0005FEF53838AE090E021C06C2F7727FB01BE
:105ED000EE0FFF1FEE0FFF1FEE0FFF1FE60FF71F66
:105EE000EE56FD4F3AEF33838DE390E00FC0AE5D89
:105EF000B94F8C910E946D63C2CF862F0E946D6353
:105F0000BECF8DE590E002C08DE090E0CF91089586
:105F10008F3F39F0E82FFF27EE5DF94F80819927F9
:105F2000089580E090E0089508959927009799F0EA
:105F3000019711F5809124039927FC01EE0FFF1FB3
:105F4000EE0FFF1FEE0FFF1FE80FF91FEE56FD4F7C
:105F5000848199270895809124039927FC01EE0FED
:105F6000FF1FEE0FFF1FEE0FFF1FE80FF91FEE568A
:105F7000FD4F8581992708958AE790E00895089557
:105F800090919102292F3327F901EE0FFF1FEE0F99
:105F9000FF1FEE0FFF1FE20FF31FEE56FD4F0480B1
:105FA000F581E02DE80FF11D8081992708959091EA
:105FB0009102292F3327F901EE0FFF1FEE0FFF1F6C
:105FC000EE0FFF1FE20FF31FEE56FD4F0480F58129
:105FD000E02DE80FF11D8491992708959091910289
:105FE000492F5527FA01EE0FFF1FEE0FFF1FEE0F8F
:105FF000FF1FE40FF51FEE56FD4F24813581280F5A
:10600000311DC901AA27BB27A160ABBFFC01879145
:1060100099270895CF93382FC09191028C2F9927FB
:10602000DC01AA0FBB1FAA0FBB1FAA0FBB1FA80F23
:10603000B91FAE56BD4FFD012481822F9927FC0167
:10604000E652F64F4491341770F5243009F43EC0FF
:10605000880F991F8E51964FFC01A591B491632F23
:106060007727A60FB71F5C91273009F444C0223070
:10607000D9F124502430A0F0842F99270197681774
:10608000790774F06C2F7727FB01EE0FFF1FEE0FDF
:10609000FF1FEE0FFF1FE60FF71FEE56FD4F128298
:1060A000852F992759C0832F841B8C3038F4E82F13
:1060B000FF27EA50FA4F808199274EC08C508C30D0
:1060C00068F08B3068F3FD011282EACFE32FFF27DF
:1060D000EE0FFF1FEA54FC4F8181EECFE82FFF2720
:1060E000EE5FF94F5081EDCF383018F2FB01EA5FD7
:1060F000F94F5081BECFA52FBB27A853BF4F28E42F
:1061000077276627A29FA001B29F500D611D112421
:10611000DB01CA0137E0B695A795979587953A9523
:10612000D1F7E82FFF27EE0FFF1FE652F84F8591BA
:10613000949177276627829FA001929F500D611D41
:106140001124DB01CA01C7E0B695A79597958795FD
:10615000CA95D1F78954B0CFCF910895E82FFF2782
:10616000EE5FF94F60830895E82FFF27EA50FA4F5A
:1061700060830895CF93DF93382F9091CE08492FF5
:106180005527FA01E652F64F84913817A0F494305F
:1061900021F1923009F468C09730A1F1A32FBB27F9
:1061A000440F551F4E51564FFA0145915491A40F7B
:1061B000B51F6C9361C09450943008F05DC0381BDB
:1061C000832F3C30C8F08C508C3008F055C0E82F3D
:1061D000FF27EE5FF94F60834FC0A62FBB279A2F92
:1061E00088278068A32FBB27ED01CA0FDB1FCA5485
:1061F000DC4F88839983D4CFE32FFF27EA50FA4FEF
:1062000060833AC0862F9927875B9F4F28E4FF273A
:10621000EE27829FE001929FD00DE11D1124CE0157
:10622000DF0177E0B695A795979587957A95D1F791
:10623000E82FFF27EE0FFF1FE652F84F659174918C
:10624000FF27EE27629FE001729FD00DE11D112410
:10625000CE01DF0167E0B695A795979587956A957A
:10626000D1F7682F685C9ACF383008F497CFE32FC6
:10627000FF27EA5FF94F6083DF91CF910895CF93B5
:10628000DF93EC01722F20912403A22FBB271196DC
:106290009D011197F901E07FF1702E1B3F0B80915A
:1062A00091022817B9F0FD01EE0FFF1FEE0FFF1F3F
:1062B000EE0FFF1FEA0FFB1FEE56FD4FC083D18389
:1062C000628313824483558376832093240380E082
:1062D00090E002C08FEF90E0DF91CF910895CF93CF
:1062E000DF93EC0120912403A22FBB2711969D017F
:1062F0001197F901E07FF1702E1B3F0B8091910205
:106300002817B9F0FD01EE0FFF1FEE0FFF1FEE0F74
:10631000FF1FEA0FFB1FEE56FD4FC083D183628340
:1063200013824483558316822093240380E090E0F7
:1063300002C08FEF90E09927DF91CF910895682FE9
:1063400080912303282F332721303105E9F02230B3
:10635000310501F1862F9927AA27BB27BC0161547B
:1063600070406733710578F4FB01E85BFD4FEE0F79
:10637000FF1F0590F491E02D099471E070932303C1
:106380002CE420933C01089560933B0122E020938C
:106390002303089540913C01242F33272E343105E7
:1063A00099F12F34310574F42A34310509F42AC2E5
:1063B0002B34310514F528343105E1F481E0809364
:1063C000CE080CC02435310509F420C2253531052D
:1063D00054F42F34310571F41092CE0880913B01B2
:1063E0000E94BA3007C02037310509F413C227379D
:1063F0003105A1F31092230308952C343105D1F710
:1064000087E08093CE08EACF86E08093CE08E6CF7F
:1064100070912403472F55274F5F5F4F9A014150DA
:106420005040B901607F7170261B370B922F30915D
:106430009102931709F4A7CFFA01EE0FFF1FEE0F99
:10644000FF1FEE0FFF1FE40FF51FEE56FD4FA5E6F1
:10645000BBE2A083B18381E382831382148215821D
:1064600020932403089580E00E94D444089520914D
:106470002403422F55274F5F5F4F9A0141505040F0
:10648000C901807F9170281B390BB09191022B17A5
:1064900009F479CFFA01EE0FFF1FEE0FFF1FEE0F89
:1064A000FF1FE40FF51FEE56FD4F44E35BE2408310
:1064B000518381E0D1CFB1E0B093230388E480938E
:1064C0003C01089531E0309323038AE4F8CFE1E002
:1064D000E09323038EE4F3CF31E0309323038FE482
:1064E000EECF90912403492F55274F5F5F4F9A01BC
:1064F00041505040B901607F7170261B370BE0910D
:1065000091022E1709F43FCFFA01EE0FFF1FEE0F95
:10651000FF1FEE0FFF1FE40FF51FEE56FD4FA5EE18
:10652000BAE2A083B18387E197CFF09124034F2F84
:1065300055274F5F5F4F9A0141505040C901807FFE
:106540009170281B390B70919102271709F41BCF0A
:10655000FA01EE0FFF1FEE0FFF1FEE0FFF1FE40FFC
:10656000F51FEE56FD4F4EEC5AE24083518388E111
:1065700073CF21E02093230384E5A1CF51E0509312
:10658000CE0820912403422F55274F5F5F4F9A0179
:1065900041505040B901607F7170261B370B8091CC
:1065A0009102281709F4EFCEFA01EE0FFF1FEE0F4C
:1065B000FF1FEE0FFF1FE40FF51FEE56FD4F4AE0E1
:1065C00050E3408351837FEF7283138281E090E038
:1065D00084839583168244CF52E05093230380E74F
:1065E0006ECF54E05093CE08F09124034F2F5527DF
:1065F0004F5F5F4F9A0141505040F901E07FF170C9
:106600002E1B3F0B70919102271709F4BCCEFA01A3
:10661000EE0FFF1FEE0FFF1FEE0FFF1FE40FF51F22
:10662000EE56FD4FAAE0B0E3A083B1834FEF428363
:10663000138284E090E084839583CCCF57E050931D
:10664000CE0830912403432F55274F5F5F4F9A01A7
:1066500041505040C901807F9170281B390BF09147
:1066600091022F1709F48FCEFA01EE0FFF1FEE0FE4
:10667000FF1FEE0FFF1FE40FF51FEE56FD4F6AE000
:1066800070E3608371839FEF9283138287E090E0D1
:10669000848395839FCF76E07093CE082091240366
:1066A000422F55274F5F5F4F9A0141505040B9012B
:1066B000607F7170261B370B80919102281709F4B7
:1066C00062CEFA01EE0FFF1FEE0FFF1FEE0FFF1F4E
:1066D000E40FF51FEE56FD4F4AE050E3408351832F
:1066E000BFEFB283138286E090E08483958372CFFC
:1066F0001092CE08F09124034F2F55274F5F5F4F24
:106700009A0141505040F901E07FF1702E1B3F0B80
:1067100070919102271709F436CEFA01EE0FFF1F90
:10672000EE0FFF1FEE0FFF1FE40FF51FEE56FD4F9C
:10673000AAE0B0E3A083B1834FEF428313821482B7
:10674000158216828DCE5091CE08652F7727209125
:106750002403422F55274F5F5F4F9A01415050400D
:10676000D901A07FB1702A1B3B0BE09191022E173B
:1067700009F409CEFA01EE0FFF1FEE0FFF1FEE0F17
:10678000FF1FE40FF51FEE56FD4F8AE090E3808374
:1067900091839FEF9283138264837583168260CE08
:1067A00082E08093CE0830912403432F55274F5F1A
:1067B0005F4F9A0141505040D901A07FB1702A1B10
:1067C0003B0BE09191022E1709F4DDCDFA01EE0F9B
:1067D000FF1FEE0FFF1FEE0FFF1FE40FF51FEE561A
:1067E000FD4F6AE070E3608371839FEF92831382B1
:1067F00082E090E084839583EDCE61E06093230393
:1068000087E75DCE84E08093CE08E8CD82E0809378
:10681000CE08E4CD683008F060E06093CE08EACDA1
:10682000109222031092230338E93AB926E020930C
:1068300095001092900087E689B91092910210920B
:10684000240308951F920F920FB60F9211242F93D5
:106850003F934F935F936F937F938F939F93AF93E8
:10686000BF93EF93FF938BB1992788719070892B19
:1068700011F08CB105C06CB18CE499E00E943CAA87
:10688000FF91EF91BF91AF919F918F917F916F9108
:106890005F914F913F912F910F900FBE0F901F90DE
:1068A00018951F920F920FB60F9211242F933F93BA
:1068B0004F935F936F937F938F939F93AF93BF9308
:1068C000EF93FF9389E299E00E94ECAA9C01892F43
:1068D0009927892B39F0559820912203222319F00A
:1068E000569A01C02CB9FF91EF91BF91AF919F9142
:1068F0008F917F916F915F914F913F912F910F9069
:106900000FBE0F901F9018951F920F920FB60F9207
:1069100011242F938F939F9355990FC02091220399
:10692000222361F09091240380919102981731F411
:106930001092900029B91092220356989F918F913E
:106940002F910F900FBE0F901F901895AC01EAE6A3
:10695000F3E020914906293C10F589E1289F900138
:10696000112488E08150F89422833383408351833B
:10697000789436968823B1F7909141069F70E92F5D
:10698000FF27E256FC4F208107C09150E92FFF27D7
:10699000E256FC4F3081232B9923B9F708C0285CBD
:1069A0006DE7269F9001112428573C4EDACF2093A3
:1069B0006303089530E83093270324E620932803E7
:1069C0001092290320932A0366EF75E070932C033D
:1069D00060932B0340E054E650932E0340932D0325
:1069E00088E380932F031092300320933103109299
:1069F0003203109233031092340310923503109235
:106A000036031092370310923803EAE6F3E09091D0
:106A10004906993C10F589E1989FC001112428E0AE
:106A20002150F89482839383108211827894369651
:106A30002223B1F7909141069F70E92FFF27E2567C
:106A4000FC4F208107C09150E92FFF27E256FC4FF1
:106A50005081252B9923B9F708C0985C8DE7989F42
:106A6000C001112488579C4EDACF209363032091F4
:106A700055083091560840915708509158085F6F5B
:106A80002093550830935608409357085093580860
:106A9000089529E333E0409141036AE08AE296E0F9
:106AA0000E9447280895F89480913B0381FF08C015
:106AB0008D7F8C6080933B038091290680936008D2
:106AC00078942091D20623FF089581E00E94016C02
:106AD000089508950F93CF93C0E080913B0382FF08
:106AE0000CC000916008002309F044C0F8940091A4
:106AF0003B030B7F00933B037894909141032091DB
:106B00003306921750F0F89440913B03477F40932F
:106B10003B037894C093290362C0F89470913B03BF
:106B2000786070933B03789450913A03A52FBB276C
:106B3000AE5DB94F8091390399278E5D994F0091D1
:106B40004103FD012289FC014289FD016085FC01B0
:106B500080850E940927853668F580E0282F2C0F54
:106B6000312D311DA901832F9927892BF9F44093E9
:106B7000290335C0209127064C2F609129068C2FC0
:106B80000E940927382F80912806389FB0011124D0
:106B9000872F992787FD9A9500914103282F432F2E
:106BA0006DEC8C2F0E940927C82FA7CF4FEF409381
:106BB000290315C0B82FB45680913E06B89FC00176
:106BC0001124892F990F990B00914B03282F4B2FDC
:106BD000609101068091F6050E940927BFCFCF91F1
:106BE0000F91089520913F03309140038091D50685
:106BF00099278F709070029709F44CC083E02C3F66
:106C00003807B8F12FEF30E0809119072817D0F13D
:106C1000332799270296821793070CF042C04091C0
:106C200032034B7F4093320390914B0330915D06CA
:106C3000391708F042C060914B0350915C0665170C
:106C400018F0416040933203A091450370916F06A4
:106C50007A17A8F58091D6089927969587959C0173
:106C60002170307080FD13C04D7F40933203C90105
:106C700008953695279536952795332780911907DE
:106C8000281730F62091320324602093320381E0EC
:106C900090E0089536952795369527953695279552
:106CA000ECCF40913203842F992784709070882311
:106CB00009F4BACF81E090E008954E7FC3CFB09140
:106CC0006008BB2331F04D7F4093320380E090E0B9
:106CD0000895242F3327B9016170707020FD0BC017
:106CE0002D7F232B31F0E0E8E09327034D7F409385
:106CF0003203CB010895426040933203C8CF089518
:106D0000EF92FF920F931F93CF93DF93CDB7DEB730
:106D100022970FB6F894DEBF0FBECDBF509125036A
:106D20005F5FF89460914D0660FF31C020913F0392
:106D3000309140038091D50699278F70907002970B
:106D400009F478C083E02C3F380708F464C08FEF63
:106D500090E0082F4091460378940417F8F450937C
:106D6000250360FF3DC020913F0330914003809197
:106D7000D50699278F709070029709F464C0F3E0EC
:106D80002C3F3F0708F44FC08FEF90E0CFC0009139
:106D90004503409146037894041708F3F02EF41A43
:106DA00080914E06F816F8F0E0903B03E4FC54C0E6
:106DB000F0915206F093300310922503B0915706DC
:106DC000B0932603F89470913B03706170933B037A
:106DD00050913B035F7D50933B03789460FDC3CF9C
:106DE00080914503A3C050932503E0903B03E5FC4D
:106DF00005C0A09126035A1708F4B3CFF894E09188
:106E00003B03EF7CE0933B03789414E6109331034B
:106E100010923003A6CF3695279536952795822F69
:106E20009927082F97CF3695279536952795822F46
:106E300099277CC0369527953695279536952795C1
:106E4000822F9927EECF369527953695279536953B
:106E50002795822F99276AC05093250300914103FB
:106E600024E6409158066DEC80E00E940927182F17
:106E70009E012F5F3F4F4F2D64E08EE496E00E940D
:106E800047280A81602F77276E5D794F898199277E
:106E90008E5D994F0F2DFB0120A9FC0140A9FB013C
:106EA00064A5FC0184A50E9409279927BC01812FB4
:106EB0000E946A287C01A92FBB27AB2B99F5009172
:106EC000410320E0409159066DEC822F0E94092772
:106ED0009701280F311D832F9927892B11F02EEF51
:106EE00030E08091300399278217930710F42093A4
:106EF0003003F0903B03F5FC06C0909125032091F0
:106F00002603921760F0F89440913B034F7C409326
:106F10003B03789434E63093310310923003609150
:106F20004D061FCFB8ECEB2EF12CC9CF8093460352
:106F300022960FB6F894DEBF0FBECDBFDF91CF9182
:106F40001F910F91FF90EF9008950F93809142064B
:106F500020914306682F620F712D711DAB016F3FA9
:106F6000710511F008F04FEF281710F020E002C073
:106F7000821B282F00913E0364EA8DE30E940927BB
:106F800099270F910895FC01662319F480E090E0A1
:106F9000089580913E03209147068E3358F13327A0
:106FA0009927CD97289FA001299F500D389F500DFC
:106FB0001124CA01892F990F990B8095282F332707
:106FC000629FD00111248B2F992787FD9A95482F16
:106FD0008AE2489FB001112475956795759567956C
:106FE0007595679575956795E617F70730F0842FC7
:106FF000992708952FEF30E0E3CF242F332788E13E
:1070000090E0E89FB001E99F700DF89F700D11248A
:10701000CB01B9010E940EC6E62FFF27E858F74EB4
:107020008491489FF00111248F2F992787FD9A950D
:107030009927089508950F93CF93DF9320914B03E1
:1070400040911D07442321F08091640388235CF163
:10705000819B2CC080915E06992733278217930766
:1070600010F140FF04C0029782179307B8F1809196
:107070006403877F8093640320913F033091400332
:107080004091D506642F77276F707070623071055C
:1070900049F153E02C3F350760F02FEF30E030919D
:1070A0001A07321778F480E090E0A3C18091F506CA
:1070B000D3CF3695279536952795332730911A07E4
:1070C000321788F38091D208882399F09927829506
:1070D0009295907F9827807F98278BC18091640339
:1070E0008860C8CF3695279536952795369527958C
:1070F000E4CF20913C0324FF23C090914B03509197
:1071000026065917E8F0409145034B3960F6409147
:107110002406493C08F05DC179E1479FA001112494
:1071200020912506293C08F04CC1B9E12B9F900124
:107130001124009141036DEC80E00E94BE2759C1EB
:10714000819B40C020913F0330914003E42FFF27F3
:10715000EF70F070329709F40CC163E02C3F3607F2
:1071600008F4F9C02FEF30E080911907281730F4A8
:107170008091320384608093320395CF332799271F
:107180000296821793070CF0FCC0209132032B7FEC
:107190002093320300914B0360915D06601708F461
:1071A00007C12E7F209332039091450340916F06D3
:1071B000491708F0F0C07091D60871FD74CF2D7F8B
:1071C000209332038091290399278C599F4FE09196
:1071D0003103DD27CC278E9FD0019E9FB00DC11DAE
:1071E00011249D01AE0190912A0380912803989F5C
:1071F000A00111246627539FF001429FE001529F96
:10720000D00DE11DF61F439FD00DE11DF61F112487
:107210009F014427552780912703992780589F4F26
:107220006627399FF001289FE001389FD00DE11DAE
:10723000F61F299FD00DE11DF61F11248D2F9E2FC3
:10724000AF2FBB279C0180913403882311F48091D8
:107250003303992780509F4F4427399FF001289F7F
:10726000E001389FD00DE11DF41F299FD00DE11DD5
:10727000F41F1124AE01BF01BB27A72F962F852F26
:107280009C0190932C0380932B03A0912D03B0912C
:107290002E034427B39FF001A29FE001B29FD00DBF
:1072A000E11DF41FA39FD00DE11DF41F1124D29501
:1072B000E295F295C0EFFE27FC23FE27ED27EC2395
:1072C000ED27BF0180912F03992788539F4F4427B3
:1072D000799FF001689FE001789FD00DE11DF41FB8
:1072E000699FD00DE11DF41F11249E01AF01BB2742
:1072F000A52F942F832FBC01C0916206C2FD1DC033
:1073000000914B03F09114070F1708F42AC08091E5
:107310003F03909140030E94D828FC0190913F06C2
:1073200055274427E99F9001F99F300D411D1124F5
:10733000BB27A52F942F832F5CC03CEAFF27EE27A5
:10734000839FE001939FD00DE11D11248D2F9E2F6F
:10735000AF2FBB27E2CF3695279536952795332754
:1073600003CF80914C039927880F991F880F991F8D
:10737000D2CF36952795369527953695279533277D
:10738000F3CE20913203822F992784709070882346
:1073900009F089CEFFCEA0916008AA2309F00FCF93
:1073A000822F992780FF1DC02260209332037BCE5D
:1073B00050914B0330915C06531708F4F5CE2160D1
:1073C000F1CE285CCDE72C9F9001112428573C4E2C
:1073D000B0CE485CADE74A9FA001112448575C4EEF
:1073E0009FCE8D7F892B09F4EDCEB0E8B0932703B3
:1073F000E6CEDF91CF910F910895EF92FF920F9318
:10740000CF93DF930E941B38EC01892BB9F1409197
:107410004606442309F088C020E030E0E22EFF2435
:10742000EE0CFF1CEE0CFF1CEC0EFD1E80914206C4
:1074300020914306682F620F712D711DAB016F3FC4
:10744000710511F008F04FEF281708F4A1C020E0F3
:1074500000913E0364EA8DE30E940927C82FDD27CF
:10746000CC0FDD1FCC0FDD1F9091300389E1989F79
:10747000A0011124C40FD51FCE0DDF1DEAE6F3E0F5
:1074800090914906993C08F047C089E1989FC00156
:10749000112428E02150F89482839383C083D18300
:1074A000789436962223B1F7909141069F70C92FA8
:1074B000DD27C256DC4F288107C09150E92FFF27F6
:1074C000E256FC4FF0802F299923B9F720936303EC
:1074D0003091480620914A06432F552760913E037C
:1074E000643A98F484EA90E0861B91093327829FDE
:1074F000D001839FB00D929FB00D11247D01EE0C41
:10750000EF2CEE1CFF084E0D5F1DC52FDD27CD2B88
:10751000E1F18FEF90E060C0985C8DE7989FC0012B
:10752000112488579C4EB5CF80913E032091470689
:107530008E3388F133279927CD97289FB001299F53
:10754000700D389F700D1124872F992787FD9A950C
:107550008095282F3327429FD00111248B2F992704
:1075600087FD9A95482F8AE2489F70011124F5946F
:10757000E794F594E794F594E794F594E794CE15A1
:10758000DF0560F0242F332749CF842F992724C0AB
:10759000821B282F5DCF2FEF30E0DDCF242F332744
:1075A00088E190E0C89FB001C99F700DD89F700D11
:1075B0001124CB01B9010E940EC6E62FFF27E8581F
:1075C000F74E8491489FF00111248F2F992787FD52
:1075D0009A95282F332722CF81BFDF91CF910F912A
:1075E000FF90EF9008950F9320914D0330914E033B
:1075F00036952795369527959091200789E1989F94
:10760000C00111248217930788F4281B390BC90184
:107610008070892B71F4022F20E140E060918F0689
:10762000842F0E9409278093370305C010923703E7
:1076300002C00FEFF1CF0F9108950F9320914D03EA
:1076400030914E03369527953695279590917C0677
:1076500089E1989FC0011124809903C08217930784
:1076600060F01092380310923403F89430913C0388
:107670003F7B30933C0378941EC0281B390BC90113
:107680008070892BB1F4022F20E140E060918F06D9
:10769000842F0E94092780933803F89420913C039B
:1076A000206420933C03789400915A06009334039D
:1076B00002C00FEFE9CF0F9108950F93CF93209160
:1076C0004D0330914E033695279536952795909129
:1076D000200789E1989FC00111248217930708F0C1
:1076E0004CC0281B390BC9018070892B09F07CC064
:1076F000022F20E140E060918F06842F0E9409272D
:1077000080933703C091370300911D07002309F0D0
:107710003DC020914D0330914E0336952795369507
:10772000279590917C0689E1989FC0011124809B48
:107730003BC01092380310923403F89450913C03EC
:107740005F7B50933C03789480913803C81708F40A
:10775000C82F80913503C81708F4C82F0E949F5B7B
:1077600080913603C81708F4C82FC13108F0C0E172
:10777000F894C093620378943BC010923703C09191
:10778000370300911D07002309F4C3CF80916403E0
:1077900099278C709070892B09F4BBCFF89420E165
:1077A00020936203789424C08217930708F0C1CF16
:1077B000281B390BD901A070AB2BC1F00FEF20E1D2
:1077C00040E060918F06842F0E9409278093380340
:1077D000F89440913C03406440933C03789430918A
:1077E0005A0630933403B0CF0FEF83CF022FE7CF89
:1077F000CF910F910895EF92FF920F931F93CF9324
:10780000DF93C091600AD091610A2091440622233F
:1078100009F432C08091490290914A021127002751
:10782000829F7001929FF00C011D1124A801970105
:107830008091D5069927929582958F7089279F70A0
:107840008927843009F49AC0813009F49AC088E00D
:1078500090E004C056954795379527958A95D2F7BD
:10786000E09045062E0D311D2138310508F483C006
:10787000C9018058904002C080E991E09093400394
:1078800080933F03E0914502F0914602F695E7951B
:10789000F695E795F695E795E050FD4F1491109316
:1078A000410320914702309148023695279536953D
:1078B000279536952795890100501E4FF801F490C1
:1078C000F092420320503F4FF901249140915F060E
:1078D000241708F443C02093280380914302909119
:1078E0004402969587959695879596958795082F46
:1078F0002FEF40E060916806809167060E94432761
:107900008093450380913F02909140029695879520
:107910009695879596958795982F80916306989F61
:10792000A0011124852F9927992780933E03FFEF0B
:10793000CF3FDF07D9F03091080711270027C39FF9
:107940007001D39FF00C011D1124BB27A12F902F94
:107950008F2D909344038093430316C000914B03F3
:107960006EE088E00E940927282FB5CF10924403CB
:107970001092430309C080E090E080CF87E090E060
:1079800068CF89E090E065CF84E00E949DB9DF91E7
:10799000CF911F910F91FF90EF900895CF93DF93B8
:1079A0008091620683FF55C020914406222309F08E
:1079B00052C080E991E0AC015695479556954795A0
:1079C00060916606262F332764E670E0DB01A21B78
:1079D000B30B4A175B0708F46EC0260F371F241736
:1079E000350708F468C0CA019070880F991F880F86
:1079F000991F880F991F9093500280934F0244362D
:107A0000510508F06DC0641B750BAAE9B0E06A9FD0
:107A1000A0016B9F500D7A9F500D1124FA019F0118
:107A200044275527205030484F4F5F4FCA01B901B6
:107A300024E630E040E050E00E94E3C5DC01CB01E9
:107A40007FE0B695A795979587957A95D1F7982F6A
:107A500061C094E65FC04091490250914A02DD271F
:107A6000CC27429FD001529FB00DC11D11249D0112
:107A7000AE018091D5069927929582958F708927BE
:107A80009F708927843031F1813009F440C088E04B
:107A900090E004C056954795379527958A95D2F77B
:107AA00050914506250F311D21383105B0F0C9012F
:107AB0008058904080CFC0E2D3E0D0935002C09372
:107AC0004F0294E6F89420913C03226020933C03FB
:107AD000789420C087E090E0DCCF80E090E06BCF2E
:107AE0002AE930E0429FB001439F700D529F700D14
:107AF0001124CB0188529C43AA27BB2720E030E801
:107B000040E050E0281B390B4A0B5B0B8FCF89E01C
:107B100090E0BFCF90932A03DF91CF9108950F9308
:107B2000F89480913B0330914B03009145034091C1
:107B300043035091440390B3927020913C03207210
:107B400060915103789481FD56C0992309F053C088
:107B50007091F106731708F04EC03091D8063017B7
:107B600008F449C08091F206882309F041C0809151
:107B7000F306882351F09927880F991F880F991FC2
:107B8000880F991F84179507B0F1222329F5F894DF
:107B900020913C03206220933C0360910907262F2B
:107BA000207F40E824276F70462F5527BA014230C6
:107BB000510509F4DAC0433051050CF0A4C0411559
:107BC000510509F4D5C04130510509F4EBC0789452
:107BD000F0919E06F093330320E04091650660919A
:107BE0008106809156060E9409278093350316C1AD
:107BF000861708F0BCCF222309F410C1F894209115
:107C00003C032F7D20933C0300910907602F607F88
:107C10000F70402F55279A014230510599F143309A
:107C200051058CF04630510509F45CC047305105D0
:107C300009F458C0FEEFF093510378941092330387
:107C400010923503EBC04115510591F141305105BA
:107C500089F767FD75C0862F992780779070959575
:107C6000879595958795959587959595879502C064
:107C7000220F331F8A95E2F7B22FB09588B38B237A
:107C800088BBD8CFE5E6F0E005B30F70062B05BB47
:107C900021E030E002C0220F331F4A95E2F7322F75
:107CA00030957081732370838081822B8083C2CF53
:107CB000862F9927807790709595879595958795CC
:107CC000959587959595879567FD0FC0E82FFF27B8
:107CD000E256FC4F6081ABB3A62BABBB8AB3862BBD
:107CE0008ABBA8CFE2E3F0E0CFCFE82FFF27E25630
:107CF000FC4F4081942F90955BB359235BBB8AB3B3
:107D0000842B8ABB97CF4630510521F0473051056F
:107D100009F05DCFE2E3F0E055B35F70522B55BB45
:107D200021E030E002C0220F331F4A95E2F7422FD4
:107D300040956081642360833081322B308347CF4C
:107D4000862F99278077907095958795959587953B
:107D5000959587959595879502C0220F331F8A9533
:107D6000E2F788B3822B88BB65CFE5E6F0E0D4CF9D
:107D7000822F99278077907095958795959587950F
:107D8000959587959595879527FD25C0E82FFF2721
:107D9000E256FC4FB0818BB38B2B8BBB8AB38B2B02
:107DA0008ABB15CF27FD25C0822F99278077907039
:107DB00095958795959587959595879595958795AB
:107DC00002C0660F771F8A95E2F7762F709588B309
:107DD000872388BBFCCEE82FFF27E256FC4F50815B
:107DE000952F9095ABB3A923ABBB8AB3852B8ABBE8
:107DF000EECE822F992780779070959587959595EF
:107E00008795959587959595879502C0660F771FFD
:107E10008A95E2F788B3862B88BBD9CE0F91089557
:107E2000CF93DF93F894209147033091480340911A
:107E3000490350914A0378948091B4089091B50811
:107E4000A091B608B091B708281739074A075B0711
:107E500040F42093B4083093B5084093B60850938B
:107E6000B708C091B008D091B108E091B208F09184
:107E7000B308C217D307E407F50740F42093B0080E
:107E80003093B1084093B2085093B308CA01AA27AF
:107E9000BB27892B61F0F89424E630E030934E0341
:107EA00020934D03789481E080934B0368C0B9011F
:107EB0008091DF069927880F991F880F991F28172F
:107EC000390778F4232B09F44FC03FEF30934B036D
:107ED000F8944CE953E650934E0340934D03789445
:107EE0004EC080914B069927382F222780914C064F
:107EF0009927282B392BA4ECB9E044273B9FF001AC
:107F00002A9FE0013A9FD00DE11DF41F2B9FD00D59
:107F1000E11DF41F11249B0144275527BE01CF0109
:107F20000E9422C6DA01C901F89430934E032093CF
:107F30004D03789459E2FF27EE27859FE001959F36
:107F4000D00DE11D1124D295E295F295C0EFFE27E8
:107F5000FC23FE27ED27EC23ED279F01A32FBB2752
:107F6000AB2B59F08FEFA0CF10924B03F8941092E7
:107F70004E0310924D03789402C020934B03DF917F
:107F8000CF910895F89480913B038260837F809322
:107F90003B03789408950F93CF93DF93409122068B
:107FA000442309F4C9C0809145038B3908F0C4C04B
:107FB000493C08F4ADC0485C2DE7429FA001112464
:107FC00048575C4E60912306FF27EE27469FE0014D
:107FD000569FD00DE11D11248D2F9E2FAF2FBB2753
:107FE000009141039C016DEC80E00E94BE27DC0102
:107FF0003091480620914A06432F552760913E0351
:10800000643A98F484EA90E0861B91093327829FB2
:10801000F001839FF00D929FF00D1124EF01CC0F22
:10802000CD2FCC1FDD0B4C0F5D1FC52FDD27CD2BBA
:1080300009F473C08FEF90E081BF109709F47CC002
:10804000EAE6F3E090914906993C08F069C089E1BD
:10805000989FC001112428E02150F89482839383D3
:10806000A083B183789436962223B1F7909141068C
:108070009F70E92FFF27E256FC4F208107C09150E7
:10808000C92FDD27C256DC4F4881242B9923B9F72D
:1080900020936303A0914F08B09150086CB57DB553
:1080A0007093500860934F086A177B0748F48091DB
:1080B000510890915208019690935208809351086C
:1080C00040916A0350916B0341155105F1F0E09125
:1080D0006C03F0916D03B09163032B2F20950BB3CC
:1080E00002230BBB9AB39B2B9ABBCB01840F951F2A
:1080F00090936F0380936E03E417F507C8F4CB01E8
:108100008E0F9F1F6BE10E9401700E947D7714C04B
:1081100009E1409FA001112455CF842F99278CCFCE
:10812000985C8DE7989FC001112488579C4E93CF8F
:108130006BE20E940170E9CFDF91CF910F9108951A
:108140008091ED06282F207F90E829278F70482FF7
:108150005527BA014230510559F1433051054CF0D1
:108160004630510509F454C04730510509F450C058
:1081700008954115510591F141305105C9F727FD89
:108180004AC0822F9927807790709595879595950D
:108190008795959587959595879502C0660F771F6A
:1081A0008A95E2F7762F709588B3872388BB089568
:1081B000E5E6F0E095B39F70922B95BB21E030E0AF
:1081C00002C0220F331F4A95E2F7822F8095B081BB
:1081D000B823B083A081A22BA0830895822F992772
:1081E00080779070959587959595879595958795C6
:1081F0009595879527FD24C0E82FFF27E256FC4F71
:1082000050816BB3652B6BBB8AB3852B8ABB0895FA
:10821000E2E3F0E0CFCF822F992780779070959599
:10822000879595958795959587959595879502C09E
:10823000660F771F8A95E2F788B3862B88BB08956F
:10824000E82FFF27E256FC4F2081422F40953BB399
:1082500034233BBB8AB3822B8ABB08958091ED0601
:10826000682F607F8F70482F55279A014230510543
:1082700059F1433051054CF04630510509F454C0D2
:108280004730510509F450C008954115510591F149
:1082900041305105C9F767FD4AC0862F992780777D
:1082A00090709595879595958795959587959595D2
:1082B000879502C0220F331F8A95E2F7622F6095DF
:1082C00088B3862388BB0895E5E6F0E085B38F7018
:1082D000862B85BB21E030E002C0220F331F4A9578
:1082E000E2F7B22FB095A081AB23A0837081722BEF
:1082F00070830895862F992780779070959587953C
:1083000095958795959587959595879567FD24C053
:10831000E82FFF27E256FC4F40815BB3542B5BBB39
:108320008AB3842B8ABB0895E2E3F0E0CFCF862F97
:1083300099278077907095958795959587959595D0
:1083400087959595879502C0220F331F8A95E2F78E
:1083500088B3822B88BB0895E82FFF27E256FC4F95
:108360002081922F90953BB339233BBB8AB3822B5C
:108370008ABB089510923B0360913C036461609353
:108380003C0310923D035FEF509364081092710814
:108390004FEF5FEF60E070E0409347035093480376
:1083A0006093490370934A0310924B0310924E035B
:1083B00010924D033091E806309352030E9436BA72
:1083C0002BE020938401F8948091ED06682F607F64
:1083D0008F70482F55279A014230510561F1433083
:1083E00051054CF04630510519F047305105C1F5A3
:1083F000E2E3F0E022C04115510509F49DC041308F
:10840000510571F567FDB2C0862F9927807790706E
:108410009595879595958795959587959595879544
:1084200002C0220F331F8A95E2F7322F309588B3AE
:10843000832388BB15C0E5E6F0E025B32F70262B1B
:1084400025BB21E030E002C0220F331F4A95E2F73E
:10845000522F50954081452340838081822B808319
:1084600078940000F89470918D06672F607F7F707C
:10847000472F55279A014230510571F1433051057C
:108480000CF54115510509F43DC04130510509F085
:10849000B2C067FD80C0862F992780779070959530
:1084A000879595958795959587959595879502C01C
:1084B000220F331F8A95E2F7322F309588B383233A
:1084C00088BB99C04630510521F04730510509F06D
:1084D00092C0E2E3F0E002C0E5E6F0E025B32F70E1
:1084E000262B25BB21E030E002C0220F331F4A9526
:1084F000E2F7522F50954081452340838081822BA3
:10850000808379C0862F992780779070959587957D
:1085100095958795959587959595879567FD5EC007
:10852000E82FFF27E256FC4FB081FBB3FB2BFBBBD0
:108530008AB38B2B8ABB5FC0862F99278077907078
:108540009595879595958795959587959595879513
:1085500067FD36C0E82FFF27E256FC4FB081FBB322
:10856000FB2BFBBB8AB38B2B8ABB7ACF862F992739
:108570008077907095958795959587959595879532
:108580009595879502C0220F331F8A95E2F788B32D
:10859000822B88BB65CF862F992780779070959521
:1085A000879595958795959587959595879502C01B
:1085B000220F331F8A95E2F788B3822B88BB1BC03A
:1085C000E82FFF27E256FC4F7081972F9095ABB3B1
:1085D000A923ABBB8AB3872B8ABB42CFE82FFF27E7
:1085E000E256FC4F6081962F9095ABB3A923ABBBAD
:1085F0008AB3862B8ABB78940000F89470910A02A3
:108600007F7370930A02789480E090E00E94A63411
:1086100008958091ED06282F207F90E829278F70FC
:10862000482F5527BA014230510569F143305105B1
:1086300054F04630510521F04730510509F075C01E
:10864000E2E3F0E022C04115510599F141305105B6
:1086500009F06BC027FD47C0822F99278077907063
:1086600095958795959587959595879595958795F2
:1086700002C0660F771F8A95E2F7762F709588B350
:10868000872388BB52C0E5E6F0E095B39F70922B3C
:1086900095BB21E030E002C0220F331F4A95E2F77C
:1086A000822F8095B081B823B083A081A22BA083B4
:1086B0003CC0822F992780779070959587959595E6
:1086C0008795959587959595879527FD21C0E82FE6
:1086D000FF27E256FC4F50816BB3652B6BBB8AB30F
:1086E000852B8ABB22C0822F992780779070959521
:1086F000879595958795959587959595879502C0CA
:10870000660F771F8A95E2F788B3862B88BB0DC06A
:10871000E82FFF27E256FC4F2081422F40953BB3C4
:1087200034233BBB8AB3822B8ABBF0913B03F160BD
:10873000F0933B03089583B7896783BF08951F9221
:108740000F920FB60F9211240F900FBE0F901F9033
:1087500018951F93CF93DF931092180240919A03BC
:1087600050919B0360919C0370919D03CB01AA27BC
:10877000BB270097A105B10561F0A091BC08B0919D
:10878000BD081196B093BD08A093BC0810924F038A
:108790003FC0E0916803F0916903A0919A03B09102
:1087A0009B03CC27FB9FB001EA9FA001FA9F500DCD
:1087B000611D7C1FEB9F500D611D7C1F1124252F17
:1087C000362F472F55271091E506612F772785E231
:1087D00093E01127939FF001829FE001929FD00DBB
:1087E000E11DF11F839FD00DE11DF11F11249E019A
:1087F000AF01CA01AA27BB27681B790BC72FDD274A
:10880000CD2B21F03FEF30934F0302C060934F0315
:10881000DF91CF911F9108951F93182F4FEF50E0D4
:1088200060E070E082E296E00E94F0C448E150E02F
:1088300067EE73E08EE993E00E94F0C41130A9F076
:1088400048E552E06FEF70E086EB93E00E94F0C4E1
:1088500040E950E067E573E081E297E00E94F0C4F0
:1088600044E150E06FEF73E014C048E552E063E18B
:1088700074E086EB93E00E94F0C440E950E06BE6C0
:1088800076E081E297E00E94F0C444E150E06BEFB3
:1088900076E08EE096E00E94F0C41F9108950F9359
:1088A0001F93CF93DF93982F8091390282FD74C07C
:1088B000892F99278A36910511F18B36910564F439
:1088C00083369105D1F1843691050CF046C082368D
:1088D000910509F061C04CC08E369105F9F08F36D4
:1088E000910584F58B36910509F44CC08C369105C1
:1088F00009F052C0C6E6D5E08FEA92E013C0062F19
:108900001127000F111FC80181509F4F0E9401C500
:108910000A541C4FF801808391833EC0C1E2D7E026
:1089200087E593E0062F1127800F911F0E94E8C46E
:108930000C0F1D1FE80188832FC0C2E2D6E080E043
:1089400090E0F0CF82379105C1F08437910521F591
:10895000CAE1D6E08BE094E0E5CF84369105B9F02A
:1089600088369105C9F4CEE9D3E087EE93E0DACFFB
:10897000CEE0D6E08FEF93E0D5CFC6EFD5E08FE322
:1089800093E0D0CFC2E0D6E08BE493E0CBCFC6ED4E
:10899000D4E08FE192E0C6CFDF91CF911F910F918C
:1089A0000895109239020895982F80919C0681387D
:1089B00018F020E820939C0630919B06313818F07F
:1089C00040E840939B065091390252FF03C080E07B
:1089D00090E00895923008F090E0709139027F7035
:1089E00070933902892F992782959295907F9827C5
:1089F000807F982760913902682B66606093390206
:108A000081E090E0089508952091190230911A02B2
:108A100080911B0290911C02820F931F0E94E8C458
:108A2000482FE0913B02F0913C0220911B023091D3
:108A30001C02E20FF31F6081861741F1461791F087
:108A40008091190290911A02820F931F0E940EC505
:108A500030913902316030933902E39A20911B0240
:108A600030911C02A0910B02B0910C0211972A17B1
:108A70003B0718F081E090E008952F5F3F4F30935F
:108A80001C0220931B0280E090E0089580910B026D
:108A900090910C0201972817390780F62F5F3F4FFE
:108AA00030931C0220931B028091190290911A02AC
:108AB000820F931F0E94E8C4482FE0913B02F0917F
:108AC0003C0220911B0230911C02E20FF31F6081D7
:108AD0008617E1F2B3CFCF93C0E080910E02282F2A
:108AE00033272230310509F499C02330310574F061
:108AF0002430310509F466C1243031050CF411C16C
:108B00002530310509F411C2C1E0AEC2211531058D
:108B100009F46AC021303105B9F72091190230916A
:108B20001A0280911B0290911C02820F931F0E94D7
:108B3000E8C4482FE0913B02F0913C0220911B02D7
:108B400030911C02E20FF31F6081861709F460C2A6
:108B5000461791F08091190290911A02820F931F8B
:108B60000E940EC530913902316030933902E39A88
:108B700020911B0230911C02A0910B02B0910C02BB
:108B800011972A173B0708F4C5C050913902507F4E
:108B900009F467C27091390272957F70272F3327CD
:108BA0006CEF72E0269FA001279F500D369F500D5D
:108BB0001124CA018D5E9B4F90931A028093190273
:108BC000E6EBF3E0F0933C02E0933B0288E592E0B1
:108BD00090930C0280930B0210921C0210921B02C5
:108BE00082E080930E0240C2A0E0B0E0B0931A028F
:108BF000A093190262E276E070933C0260933B021C
:108C00004FEF50E050930C0240930B0230931C0244
:108C100020931B0281E080930E0226C2A0911902CC
:108C2000B0911A0280911B0290911C028A0F9B1F27
:108C30000E94E8C4482FE0913B02F0913C02209151
:108C40001B0230911C02E20FF31F60818617E1F1D5
:108C5000461791F08091190290911A02820F931F8A
:108C60000E940EC590913902916090933902E39A67
:108C700020911B0230911C02A0910B02B0910C02BA
:108C800011972A173B0708F445C0B0913902B07F0D
:108C900009F0ABC187E593E090931A028093190223
:108CA000E1E2F7E0F0933C02E0933B0280E990E0E0
:108CB00090930C0280930B0210921C0210921B02E4
:108CC00083E080930E02D0C180910B0290910C0240
:108CD00001972817390708F0BBCF2F5F3F4F30931C
:108CE0001C0220931B028091190290911A02820F9C
:108CF000931F0E94E8C4482FE0913B02F0913C0290
:108D000020911B0230911C02E20FF31F6081861735
:108D1000D9F29ECF2F5F3F4F30931C0220931B024E
:108D2000A3C1A0911902B0911A0280911B029091E7
:108D30001C028A0F9B1F0E94E8C4482FE0913B024F
:108D4000F0913C0220911B0230911C02E20FF31FB4
:108D50006081861709F49DC0461791F08091190231
:108D600090911A02820F931F0E940EC53091390212
:108D7000316030933902E39A20911B0230911C023A
:108D8000A0910B02B0910C0211972A173B0710F229
:108D900027EE33E030931A02209319026EE973E054
:108DA00070933C0260933B0248E150E050930C0208
:108DB00040930B0210921C0210921B0284E08093DD
:108DC0000E0252C1A0911902B0911A0280911B02A9
:108DD00090911C028A0F9B1F0E94E8C4482FE091CB
:108DE0003B02F0913C0220911B0230911C02E20FE9
:108DF000F31F6081861709F472C0461791F08091C5
:108E0000190290911A02820F931F0E940EC5509171
:108E10003902516050933902E39A20911B0230913C
:108E20001C02A0910B02B0910C0211972A173B076C
:108E300008F470CF70913902707F09F40FC19091DE
:108E4000390292959F70292F33276CEF72E0269F8D
:108E5000A001279F500D369F500D1124CA01855047
:108E6000994F90931A0280931902EEE0F6E0F09386
:108E70003C02E0933B0284E190E090930C028093EB
:108E80000B0210921C0210921B0285E080930E02CE
:108E9000EBC080910B0290910C02019728173907C3
:108EA00008F05ACF2F5F3F4F30931C0220931B02D4
:108EB0008091190290911A02820F931F0E94E8C4B8
:108EC000482FE0913B02F0913C0220911B0230912F
:108ED0001C02E20FF31F60818617D9F23DCF80910B
:108EE0000B0290910C0201972817390708F085CFE3
:108EF0002F5F3F4F30931C0220931B028091190279
:108F000090911A02820F931F0E94E8C4482FE091AB
:108F10003B02F0913C0220911B0230911C02E20FB7
:108F2000F31F60818617D9F268CFA0911902B09122
:108F30001A0280911B0290911C028A0F9B1F0E94B3
:108F4000E8C4482FE0913B02F0913C0220911B02C3
:108F500030911C02E20FF31F6081861709F146175A
:108F600091F08091190290911A02820F931F0E9432
:108F70000EC5B0913902B160B0933902E39A2091E5
:108F80001B0230911C02A0910B02B0910C021197B0
:108F90002A173B0708F4BECE86E080930E0264C019
:108FA00080910B0290910C02019728173907B8F6AF
:108FB0002F5F3F4F30931C0220931B0280911902B8
:108FC00090911A02820F931F0E94E8C4482FE091EB
:108FD0003B02F0913C0220911B0230911C02E20FF7
:108FE000F31F60818617E1F2BACFF0913902F29552
:108FF000FF702F2F33276CEF72E0269FA001279F71
:10900000500D369F500D1124CA018559994F44CEF9
:1090100080910B0290910C0201972817390708F0F4
:1090200097CD2F5F3F4F30931C0220931B028091FE
:10903000190290911A02820F931F0E94E8C4482FD0
:10904000E0913B02F0913C0220911B0230911C0206
:10905000E20FF31F60818617D9F27ACD8FEF93E08C
:1090600000CF8FEF90E0A8CD8C2F9927CF91089556
:109070008091390282FF19C02091390221FF08C076
:10908000309139023D7F3093390210920E020895DB
:109090004091390240FD09C00E946B45882329F0A8
:1090A000509139025B7F50933902089508951F92C1
:1090B0000F920FB60F9211248F93809139028E7FF9
:1090C00080933902E3988F910F900FBE0F901F90FD
:1090D000189580914103909169069817E8F4F894E7
:1090E00030916B06232F207F90E829273F70432F74
:1090F0005527BA014230510509F46EC0433051057D
:109100000CF449C04630510509F4B8C04730510548
:1091100009F4B4C07894089520914103422F552753
:10912000692F7727F0916A066F1B7109641775071D
:109130008CF1F89470916B06672F607F7F70472FDA
:1091400055279A014230510509F45DC0433051055D
:109150000CF08AC04115510509F493C04130510506
:10916000C1F467FDDAC0862F9927807790709595B6
:10917000879595958795959587959595879502C03F
:10918000220F331F8A95E2F7322F309588B383235D
:1091900088BB789408954115510509F44BC04130BE
:1091A000510509F0B7CF27FDA3C0822F99278077FB
:1091B00090709595879595958795959587959595B3
:1091C000879502C0660F771F8A95E2F7A62FA095B4
:1091D00088B38A2388BB9ECFE5E6F0E095B39F7005
:1091E000922B95BB21E030E002C0220F331F4A953D
:1091F000E2F7322F3095808183238083B081B22BB8
:10920000B08378940895E5E6F0E025B32F70262B1F
:1092100025BB21E030E002C0220F331F4A95E2F760
:10922000422F40956081642360839081922B9083CC
:109230007894B0CF822F99278077907095958795F5
:1092400095958795959587959595879527FD34C034
:10925000E82FFF27E256FC4F60817BB3762B7BBB68
:109260008AB3862B8ABB56CF4630510521F0473052
:10927000510509F08ECFE2E3F0E0C7CFE2E3F0E082
:10928000ADCF862F99278077907095958795959586
:109290008795959587959595879567FD1BC0E82FD0
:1092A000FF27E256FC4FB0818BB38B2B8BBB8AB36D
:1092B0008B2B8ABB78946ECFE82FFF27E256FC4FAA
:1092C0002081522F50954BB345234BBB8AB3822B41
:1092D0008ABB20CFE82FFF27E256FC4F5081A52FF5
:1092E000A095EBB3EA23EBBB8AB3852B8ABBE2CF15
:1092F000822F99278077907095958795959587957A
:10930000959587959595879502C0660F771F8A95E5
:10931000E2F788B3862B88BBFDCE862F992780770E
:109320009070959587959595879595958795959541
:10933000879502C0220F331F8A95E2F788B3822BEC
:1093400088BB27CF80914103909112079817E8F4CA
:10935000F89430911607232F207F90E829273F703B
:10936000432F5527BA014230510509F46EC04330EE
:1093700051050CF449C04630510509F4B8C04730D6
:10938000510509F4B4C07894089520914103422F07
:109390005527692F7727F09115076F1B71096417FF
:1093A00075078CF1F89470911607672F607F7F70B6
:1093B000472F55279A014230510509F45DC04330CB
:1093C00051050CF08AC04115510509F493C0413094
:1093D0005105C1F467FDDAC0862F99278077907018
:1093E0009595879595958795959587959595879565
:1093F00002C0220F331F8A95E2F7322F309588B3CF
:10940000832388BB789408954115510509F44BC016
:109410004130510509F0B7CF27FDA3C0822F99270E
:109420008077907095958795959587959595879573
:109430009595879502C0660F771F8A95E2F7A62F4C
:10944000A09588B38A2388BB9ECFE5E6F0E095B36C
:109450009F70922B95BB21E030E002C0220F331F9A
:109460004A95E2F7322F3095808183238083B08143
:10947000B22BB08378940895E5E6F0E025B32F7021
:10948000262B25BB21E030E002C0220F331F4A9576
:10949000E2F7422F40956081642360839081922B94
:1094A00090837894B0CF822F99278077907095958C
:1094B000879595958795959587959595879527FD9A
:1094C00034C0E82FFF27E256FC4F60817BB3762B38
:1094D0007BBB8AB3862B8ABB56CF4630510521F021
:1094E0004730510509F08ECFE2E3F0E0C7CFE2E369
:1094F000F0E0ADCF862F992780779070959587956E
:1095000095958795959587959595879567FD1BC04A
:10951000E82FFF27E256FC4FB0818BB38B2B8BBB20
:109520008AB38B2B8ABB78946ECFE82FFF27E25645
:10953000FC4F2081522F50954BB345234BBB8AB330
:10954000822B8ABB20CFE82FFF27E256FC4F5081A9
:10955000A52FA095EBB3EA23EBBB8AB3852B8ABB7F
:10956000E2CF822F99278077907095958795959572
:109570008795959587959595879502C0660F771F76
:109580008A95E2F788B3862B88BBFDCE862F992774
:109590008077907095958795959587959595879502
:1095A0009595879502C0220F331F8A95E2F788B3FD
:1095B000822B88BB27CF20914B038091060782170F
:1095C00088F590E8F89480910707282F207F2927B5
:1095D0008F70482F5527BA0142305105B9F14330F9
:1095E00051050CF04AC04115510509F04FC0822FBA
:1095F00099278077907095958795959587959595FE
:1096000087959595879527FD5EC0E82FFF27E25641
:10961000FC4F40815BB3542B5BBB8AB3842B8ABB6A
:109620007894089533279927029782179307CCF3EC
:1096300090E0F89480910707282F207F29278F70CA
:10964000482F5527BA014230510549F6E5E6F0E0CA
:1096500085B38F70822B85BB21E030E002C0220FE2
:10966000331F4A95E2F7B22FB095A081AB23A083B8
:109670006081622B60837894D4CF4630510519F015
:109680004730510569F6E2E3F0E0E2CF41305105A1
:1096900039F627FD26C0822F9927807790709595FF
:1096A000879595958795959587959595879502C00A
:1096B000660F771F8A95E2F7762F709588B3872318
:1096C00088BB7894AECFE82FFF27E256FC4F20816D
:1096D000922F90953BB339233BBB8AB3822B8ABB35
:1096E0009FCF822F99278077907095958795959534
:1096F0008795959587959595879502C0660F771FF5
:109700008A95E2F788B3862B88BBDBCF40914B0369
:109710005091450320913F03309140038091D5063D
:1097200099278F709070029709F487C083E02C3FCF
:109730003807E0F18FEF90E0982F8091F6064817F8
:1097400008F040C090E0F8947091FC06272F207F2D
:1097500029277F70472F5527BA014230510509F458
:1097600056C0433051050CF048C04115510509F46D
:109770006BC04130510509F0A3C027FD7FC0822F87
:10978000992780779070959587959595879595956C
:1097900087959595879502C0660F771F8A95E2F7A2
:1097A000362F309588B3832388BB8AC0369527959A
:1097B00036952795822F9927982F8091F60648177E
:1097C00008F4C0CF2091F706421708F0BBCF3091C4
:1097D000F806531708F4B6CF4091F906541708F06D
:1097E000B1CF5091FA06951708F4ACCF6091FB0603
:1097F000961708F0A7CF90E8A6CF4630510521F084
:109800004730510509F05CC0E2E3F0E002C0E5E654
:10981000F0E065B36F70622B65BB21E030E002C001
:10982000220F331F4A95E2F7522F5095408145236E
:1098300040838081822B808343C03695279536955F
:10984000279536952795B6CF822F992780779070E8
:1098500095958795959587959595879595958795F0
:1098600027FD21C0E82FFF27E256FC4F2081FBB3E4
:10987000F22BFBBB8AB3822B8ABB22C0822F992793
:10988000807790709595879595958795959587950F
:109890009595879502C0660F771F8A95E2F788B382
:1098A000862B88BB0DC0E82FFF27E256FC4FA08116
:1098B0009A2F9095BBB3B923BBBB8AB38A2B8ABBC3
:1098C0007894089540914B035091450320913F03B4
:1098D000309140038091D50699278F709070029740
:1098E00009F487C083E02C3F3807E0F18FEF90E068
:1098F000982F8091FD06481708F040C090E0F8943A
:1099000070910307272F207F29277F70472F552726
:10991000BA014230510509F456C0433051050CF0EC
:1099200048C04115510509F46BC04130510509F09B
:10993000A3C027FD7FC0822F9927807790709595CF
:10994000879595958795959587959595879502C067
:10995000660F771F8A95E2F7362F309588B38323F9
:1099600088BB8AC03695279536952795822F9927EB
:10997000982F8091FD06481708F4C0CF2091FE066D
:10998000421708F0BBCF3091FF06531708F4B6CF4B
:1099900040910007541708F0B1CF50910107951777
:1099A00008F4ACCF60910207961708F0A7CF90E8B3
:1099B000A6CF4630510521F04730510509F05CC073
:1099C000E2E3F0E002C0E5E6F0E065B36F70622B21
:1099D00065BB21E030E002C0220F331F4A95E2F759
:1099E000522F50954081452340838081822B808374
:1099F00043C0369527953695279536952795B6CF4A
:109A0000822F992780779070959587959595879562
:109A1000959587959595879527FD21C0E82FFF2778
:109A2000E256FC4F2081FBB3F22BFBBB8AB3822BA7
:109A30008ABB22C0822F9927807790709595879551
:109A400095958795959587959595879502C0660F0D
:109A5000771F8A95E2F788B3862B88BB0DC0E82F65
:109A6000FF27E256FC4FA0819A2F9095BBB3B923F4
:109A7000BBBB8AB38A2B8ABB78940895CF93C091DD
:109A80001B07CF3F09F47EC1F89480914703909162
:109A90004803A0914903B0914A039C0178948091B6
:109AA0001C07823008F472C099270297F90102C09E
:109AB000EE0FFF1F8A95E2F7F89480914F0890917E
:109AC00050086CB57DB57093500860934F086817C7
:109AD000790748F4A0915108B09152081196B093BB
:109AE0005208A09351089B0178944091B10750917E
:109AF000B207241B350B2E173F0708F443C1CF01D3
:109B0000880F991F8217930708F444C04E0F5F1FF8
:109B10005093B2074093B10720913D0120952093C7
:109B20003D01222309F442C0F8942C2F207F30E815
:109B30002327CF704C2F5527BA014230510509F425
:109B400077C0433051050CF060C04115510509F450
:109B5000B8C041305105C1F427FDFFC0822F9927BD
:109B6000807790709595879595958795959587952C
:109B70009595879502C0660F771F8A95E2F7B62FF5
:109B8000B09588B38B2388BB7894FCC0F901F69517
:109B9000E79592CF7093B2076093B10720913D0192
:109BA000209520933D01222309F0BECFF8946C2F1D
:109BB000607FCF704C2F55279A014230510509F430
:109BC0004EC0433051055CF54115510509F45EC0A6
:109BD00041305105C1F467FDABC0862F99278077CE
:109BE0009070959587959595879595958795959579
:109BF000879502C0220F331F8A95E2F7622F609586
:109C000088B3862388BB7894BDC04630510521F0C7
:109C10004730510509F0B8CFE2E3F0E00BC0463021
:109C2000510519F04730510571F7E2E3F0E019C032
:109C3000E5E6F0E035B33F70322B35BB21E030E094
:109C400002C0220F331F4A95E2F7822F8095A08130
:109C5000A823A083C081C22BC083789493C0E5E67B
:109C6000F0E0A5B3AF70A62BA5BB21E030E002C0A9
:109C7000220F331F4A95E2F7C22FC095B081BC2353
:109C8000B0837081722B708378947CC0862F992763
:109C900080779070959587959595879595958795FB
:109CA0009595879567FD28C0E82FFF27E256FC4F62
:109CB00050819BB3952B9BBB8AB3852B8ABB789431
:109CC00061C0822F9927807790709595879595959B
:109CD0008795959587959595879527FD1BC0E82FC6
:109CE000FF27E256FC4F60817BB3762B7BBB8AB3A8
:109CF000862B8ABB789446C0E82FFF27E256FC4F9C
:109D00002081422F4095FBB3F423FBBB8AB3822B07
:109D10008ABBD5CFE82FFF27E256FC4F4081942F16
:109D200090955BB359235BBB8AB3842B8ABBE2CF8C
:109D3000862F99278077907095958795959587952B
:109D4000959587959595879502C0220F331F8A9523
:109D5000E2F788B3822B88BB56CF822F9927807772
:109D600090709595879595958795959587959595F7
:109D7000879502C0660F771F8A95E2F788B3862B16
:109D800088BB02CFCF910895209160063327207FB2
:109D900030703595279535952795359527952E5F04
:109DA00077276627829FA001929F500D611D112485
:109DB000DB01CA0126EB77276627829FA001929FCD
:109DC000500D611D1124BB27A72F962F852F0895B5
:109DD0000F9300914B03509113076091140720914A
:109DE0003F03309140038091D50699278F70907082
:109DF000029769F083E02C3F380718F02FEF30E02E
:109E00000DC03695279536952795332707C036958B
:109E100027953695279536952795F7CF4091450399
:109E2000852F0E940927992780934C0323EB37E065
:109E3000482F6CE082E096E00E94472825EB37E04F
:109E400040914B036CE086EF95E00E9447280F910C
:109E500008952F923F924F925F926F927F928F92CE
:109E60009F92AF92BF92CF92DF92EF92FF920F93A9
:109E70001F93CF93DF93CDB7DEB760970FB6F894FB
:109E8000DEBF0FBECDBFC090B407EC2DFF27EE5F45
:109E9000F94F50808090B307E82DFF27EE5FF94F10
:109EA00060805618E52DFF27EE0FFF1FE652F84F92
:109EB000A590B4900091B607E02FFF27EA50FA4F23
:109EC0009081E090B507EE2DFF27EA50FA4F3080E1
:109ED000492E4318E42DFF27EE0FFF1FE652F84FDF
:109EE0004591549189E1989F9001112480914D03EF
:109EF00090914E039695879596958795821793072F
:109F000008F02EC2281B390B13EA77246624419FE0
:109F10002001519F500C611C1124B301A2015295E4
:109F20006295729540EF7627742376276527642320
:109F300065273B01EE27739EB001629EA001729ED1
:109F4000500D611D7E1F639E500D611D7E1F1124EB
:109F5000BA013B0160947094EE2DFF27E25FF94F48
:109F60009080E02FFF27E25FF94F4081292D3327B2
:109F7000872D9927289FF001299FF00D389FF00D1C
:109F80001124CF015527472E5524449D1001459D8E
:109F9000300C549D300C11249101929582958F7054
:109FA00089279F708927329522952F7023273F702C
:109FB0002327820F931F929582958F7089279F7018
:109FC000892780936703EC2DFF27EE5FF94FE0812F
:109FD00080914C038E1708F055C2E81BBB27AA27B7
:109FE000AE9EC001BE9E900DA11D11245C012501F5
:109FF000409450944427B79ED001A69EC001B69EBF
:10A00000900DA11DB41FA79E900DA11DB41F11247A
:10A01000CD01AA27BB2789839A834427B79CD00107
:10A02000A69CC001B69C900DA11DB41FA79C900DCD
:10A03000A11DB41F1124CD01AA27BB278B839C83AC
:10A040004427579ED001469EC001569E900DA11DEB
:10A05000B41F479E900DA11DB41F1124CD01AA2746
:10A06000BB271C01EE27579CB001469CA001569CC3
:10A07000500D611D7E1F479C500D611D7E1F1124D8
:10A08000CB01AA27BB272C015CE0859EC0011124CF
:10A09000DE2CD80EF02EF80EC59EC0011124E80E5D
:10A0A000080F8D2C9924F401E80DF91DEA54FC4F9A
:10A0B000A081B181CF2CDD24F601EC0DFD1DEA5409
:10A0C000FC4F808191818D839E83FF24F701EE0DEB
:10A0D000FF1DEA54FC4F608071801127F801E00FEA
:10A0E000F11FEA54FC4FA080B180E981FA818F2FE3
:10A0F00099272B813C81432F55274F835887E32D88
:10A10000FF27ED87FE87652D77276F87788B55278B
:10A110004427A89F9001B89F300D411D1124DA01FA
:10A12000C901ED81FE812F8177276627E29FA0017B
:10A13000F29F500D611D1124840F951FA61FB71F9C
:10A140006D8555274427669E9001769E300D411DF2
:10A150001124820F931FA41FB51F7F855527442705
:10A16000A79E9001B79E300D411D1124820F931FB1
:10A17000A41FB51F892F9A2FAB2FBB2790932E03B7
:10A1800080932D03F401EA59FA4FB081F601EA59A0
:10A19000FA4F7081F701EA59FA4FA080F801EA59A5
:10A1A000FA4F7080E981FA8155274427EB9F90018F
:10A1B000FB9F300D411D1124DA01C901EB81FC81A7
:10A1C00055274427E79F9001F79F300D411D11242B
:10A1D000820F931FA41FB51F552744272A9C900167
:10A1E0003A9C300D411D1124820F931FA41FB51FEF
:10A1F00055274427479C9001579C300D411D112441
:10A20000820F931FA41FB51FCD01AA27BB278093E0
:10A210002F0381E2482F87E0582F840E951ED4012A
:10A22000BC90C40ED51EF6013081E40EF51ED70198
:10A230006C91040F151FF801708149815A81112713
:10A2400000274B9D70015B9DF00C011D11245701EF
:10A250006801EB81FC8111270027E39F7001F39FC8
:10A26000F00C011D1124AE0CBF1CC01ED11E992480
:10A270008824269E3001369E700C811C1124A60C69
:10A28000B71CC81CD91C11270027479E7001579E78
:10A29000F00C011D1124AE0CBF1CC01ED11EC60146
:10A2A000AA27BB27882E99244091D6060FEF10E0ED
:10A2B000041B1109801691060CF0E2C0182F140F30
:10A2C000F0913C03F6FF4FC020915B06211708F484
:10A2D00060C080E00E94D75B782F8091DE088823E1
:10A2E00009F461C0782F6091D606472F5527109149
:10A2F000E506212F3327220F331F260F311D42176A
:10A30000530708F475C0E0E0F0E04091E90646FF2D
:10A3100097C09090E606492D552742955295507F5B
:10A320005427407F542720913E032637B8F4A6E7F0
:10A33000B0E0A21BB1092091E7063327A29F40019C
:10A34000A39F900CB29F900C11246401D594C794E4
:10A35000D594C794D594C7944C0D5D1DCA01AFC068
:10A3600060E070E0F6CD90913C0395FD95C0809142
:10A370005A039927FC01EE0FFF1FEE0FFF1FEE0F90
:10A38000FF1FE80FF91FE358F54F2481211708F04C
:10A39000A0CF812F821B0E94D75B782F8091DE088F
:10A3A000882309F09FCF50904B0330902606351438
:10A3B00008F499CF4091E806E42EFF246091D60678
:10A3C0000FEF10E0061B1109E016F1060CF075C046
:10A3D000742F760F472F55271091E506212F33272D
:10A3E000220F331F260F311D4217530708F08BCF62
:10A3F000241B350B809160069927807F907095957E
:10A40000879595958795959587958E5F7724662492
:10A41000289F2001389F500C611C112436EB112716
:10A420000027439E7001539EF00C011D1124BB2791
:10A43000A12F902F8F2DFC014091E90646FD69CF99
:10A440008AE991E0B0905203772466248B9D200125
:10A450009B9D500C611C1124BB27A72D962D852D8B
:10A4600001E08836900798F029E130E0B0914B0385
:10A47000BB3058F443FF09C0C90180509E4F1FC034
:10A480001FEF1ECFAA24BB24B2CDC90118C020E8FB
:10A4900031E0281B390BEACF0091450320E04091C1
:10A4A000F4066091D8068091D7060E94092781178B
:10A4B00008F00FCF181B812F0DCF7FEF16CFF89428
:10A4C00070935203F0935E03E0935D0390935C03FB
:10A4D00080935B0370905A0370927A0A7894609626
:10A4E0000FB6F894DEBF0FBECDBFDF91CF911F91A5
:10A4F0000F91FF90EF90DF90CF90BF90AF909F9023
:10A500008F907F906F905F904F903F902F90089525
:10A51000CF92DF92EF92FF920F931F93CF93DF932F
:10A52000982FF42E722F203809F4A4C08091CE0603
:10A53000841708F09FC0062F1127C92FDD272CE0B4
:10A5400030E0029FF001039FF00D129FF00D1124E7
:10A55000EC0FFD1FEE0FFF1FEA54FC4F0190F0813E
:10A56000E02D77FD81C080E8871B55274427E89FB1
:10A570009001F89F300D411D1124DA01C901292FE6
:10A580003A2F4B2F55278091CF06F89EA00111241A
:10A590006627359F7001249F6001349FD00CE11C19
:10A5A000F61E259FD00CE11CF61E1124C701AA2718
:10A5B000BB27AC0177FD4EC0E81BF90BAF016CE087
:10A5C00070E0069FF001079FF00D169FF00D11241B
:10A5D000EC0FFD1FEA52FB4F20818091D006289F8F
:10A5E000700111248F2D992787FD9A95332799277C
:10A5F000F901E80FF91FEF3FF105E9F0E0F0EFEFA7
:10A60000FFEF281B390B322F2227E417F507E8F458
:10A61000AF01ACE0B0E00A9FF0010B9FF00D1A9F74
:10A62000F00D1124EC0FFD1FEE0FFF1FEA54FC4F3D
:10A63000408351831FC0FE2FEE27EF6F281B390B7D
:10A64000322F2227E417F50718F34217530708F7AC
:10A65000A901DFCFCC24DD24CE1ADF0A8C159D059D
:10A6600030F04FEF5FEFABCF872F80587ECF4E0F8C
:10A670005F1FA5CFDF91CF911F910F91FF90EF90BA
:10A68000DF90CF9008952F923F924F925F926F92FA
:10A690007F928F929F92AF92BF92CF92DF92EF9272
:10A6A000FF920F931F93CF93DF93CDB7DEB7299718
:10A6B0000FB6F894DEBF0FBECDBF6C015091B4074A
:10A6C000E52FFF27EE5FF94FF0804091B307E42FAD
:10A6D000FF27EE5FF94F1081F11AEF2DFF27EE0FE4
:10A6E000FF1FE652F84FE590F490B090B607EB2DBF
:10A6F000FF27EA50FA4F6080A090B507EA2DFF27A8
:10A70000EA50FA4F70806718E62DFF27EE0FFF1F03
:10A71000E652F84F059114919E012F5F3F4FFC01C7
:10A7200040816CE086EF95E00E9447289E012D5FF6
:10A730003F4FF60141816CE082E096E00E9447289D
:10A740003E010894611C711CF3013181A32EBB24CE
:10A75000F501EA50FA4F9080F601508095184C8030
:10A76000642D7727FB01EE5FF94F8080F601318081
:10A77000831855244424099D1001199D300C411C57
:10A780001124BB27A52D942D832D182F5524442447
:10A79000E89C1001F89C300C411C1124BB27A52D0E
:10A7A000942D832D982E812E8094582E5094909124
:10A7B000B9078091BA07989F90011124992796951F
:10A7C000982F882797958795281B390B232F332798
:10A7D000022F00588091D10682FFD4C1199DD0016B
:10A7E00011248B2F9927848349803B803D82682FD9
:10A7F000003809F48EC07091CE06781708F089C031
:10A80000A32CBB24E42CFF248CE090E0A89EF00154
:10A81000A99EF00DB89EF00D1124EE0DFF1DEE0F58
:10A82000FF1FEA54FC4F0190F081E02D002314F04B
:10A8300020E8201BBB27AA27E29FC001F29F900DB2
:10A84000A11D1124892F9A2FAB2FBB278E839F83A5
:10A85000A887B9878091CF06689FD00111242E80E8
:10A860003F8022273B9EB0012A9EA0013A9E500DB8
:10A87000611D721F2B9E500D611D721F1124DB0183
:10A88000CA01CD01AA27BB279C0107FDF2C3DF0146
:10A89000A21BB30B4CE050E0A49EF001A59EF00D6E
:10A8A000B49EF00D1124EE0DFF1DEA52FB4F2081E6
:10A8B0008091D006289F10011124832D992787FDB0
:10A8C0009A95422F55279927BA01680F791F6F3F34
:10A8D000710511F008F018C3762F66276F6F481BBB
:10A8E000590B942F88276A177B0708F007C3DB01F1
:10A8F0008CE090E0A89EF001A99EF00DB89EF00DAE
:10A900001124EE0DFF1DEE0FFF1FEA54FC4FA08334
:10A91000B183159D700111248F2D9927F601858330
:10A920002C81182F003829F0B091CE06B81708F402
:10A93000C5C1899C500111248B2D9927F60186836E
:10A94000F3012181182F003809F48BC0F091CE0655
:10A95000F81708F086C09D81A92EBB24E22EFF24A3
:10A960006CE070E0A69EF001A79EF00DB69EF00D83
:10A970001124EE0DFF1DEE0FFF1FEA54FC4F608106
:10A98000718107FD9AC380E8801B55274427689F83
:10A990009001789F300D411D1124DA01C901892FE2
:10A9A0009A2FAB2FBB278E839F83A887B98780916F
:10A9B000CF06189FD00111242E803F80FF273B9E99
:10A9C000A0012A9E90013A9E300D411D5F1F2B9ED3
:10A9D000300D411D5F1F1124CA01AA27BB2707FDA7
:10A9E0005EC3681B790B4CE050E0A49EF001A59E6D
:10A9F000F00DB49EF00D1124EE0DFF1DEA52FB4F39
:10AA000020818091D006289F10011124832D992741
:10AA100087FD9A9533279927A901480F591F4F3F62
:10AA2000510511F008F079C2542F44274F6F281BAD
:10AA3000390B322F22274617570708F068C2BA0190
:10AA4000ACE0B0E0AA9EF001AB9EF00DBA9EF00D16
:10AA50001124EE0DFF1DEE0FFF1FEA54FC4F608323
:10AA60007183859C700111248F2D9927F6018783AE
:10AA7000F30121813C81182F003809F40AC4C090E9
:10AA8000CE06C81608F005C4A32EBB24C22EDD24B2
:10AA90006CE070E0A69EF001A79EF00DB69EF00D52
:10AAA0001124EC0DFD1DEE0FFF1FEA54FC4F6081D9
:10AAB000718107FDFFC280E8801B55244424689FF4
:10AAC0001001789F300C411C11245527452D342D41
:10AAD000232D8091CF06189F100111248824339DC7
:10AAE0003001229D2001329D500C611C781C239D59
:10AAF000500C611C781C1124C301AA27BB2707FD39
:10AB0000C3C2681B790B0CE010E0A09EF001A19E6F
:10AB1000F00DB09EF00D1124EC0DFD1DEA52FB4F1F
:10AB200020818091D006289F20011124852D99270E
:10AB300087FD9A9533279927A901480F591F4F3F41
:10AB4000510511F008F0D7C1542F44274F6F281B2F
:10AB5000390B322F22274617570708F0C6C1BA0112
:10AB60002CE030E0A29EF001A39EF00DB29EF00D0D
:10AB70001124EC0DFD1DEE0FFF1FEA54FC4F608306
:10AB8000718387C387FC20C1F6011682178257FCA8
:10AB9000D0C1F6011582199D700111248F2D9927BE
:10ABA00084834981EB81682F003809F472C3B09027
:10ABB000CE06B81608F06DC3CE2EDD24E42EFF2499
:10ABC000ACE0B0E0CA9EF001CB9EF00DDA9EF00D35
:10ABD0001124EE0DFF1DEE0FFF1FEA54FC4F0190F4
:10ABE000F081E02D07FD02C020E8201B55244424FD
:10ABF000E29F1001F29F300C411C11245527452D76
:10AC0000342D232D8091CF06689F50011124662496
:10AC10003B9D20012A9D10013A9D300C411C561C81
:10AC20002B9D300C411C561C1124C201AA27BB27A6
:10AC30009C0107FD45C2DF01A21BB30B8CE090E035
:10AC4000C89EF001C99EF00DD89EF00D1124EE0DA6
:10AC5000FF1DEA52FB4F70818091D006789FA001C2
:10AC60001124852F992787FD9A95472F55279927D6
:10AC7000BA01680F791F6F3F710511F008F0E8C144
:10AC8000762F66276F6F481B590B942F88276A17FA
:10AC90007B0708F0D7C1DB010CE010E0C09EF0019B
:10ACA000C19EF00DD09EF00D1124EE0DFF1DEE0F94
:10ACB000FF1FEA54FC4FA083B183EBC2E22EFF24B6
:10ACC000A42CBB24ACE0B0E0EA9EF001EB9EF00DBA
:10ACD000FA9EF00D1124EA0DFB1DEE0FFF1FEA5442
:10ACE000FC4F6081718107FDC1C180E8801B552741
:10ACF0004427689F9001789F300D411D1124DA018F
:10AD0000C901892F9A2FAB2FBB278E839F83A887DA
:10AD1000B9878091CF06189FD00111242E803F80E3
:10AD2000FF273B9EA0012A9E90013A9E300D411DB7
:10AD30005F1F2B9E300D411D5F1F1124CA01AA27E2
:10AD4000BB2707FD88C1681B790B4CE050E0E49EEF
:10AD5000F001E59EF00DF49EF00D1124EA0DFB1DAF
:10AD6000EA52FB4F20818091D006289F10011124C8
:10AD7000832D992787FD9A9533279927A901480F95
:10AD8000591F4F3F510511F008F0D0C0542F4427F0
:10AD90004F6F281B390B322F22274617570708F011
:10ADA000BFC0BA01ACE0B0E0EA9EF001EB9EF00D4E
:10ADB000FA9EF00D1124EA0DFB1DEE0FFF1FEA5461
:10ADC000FC4F60837183B5CDF6011482158257FC68
:10ADD00082C1F6011782899C20011124852D9927B3
:10ADE0008683EB81682F003809F453C23090CE0679
:10ADF000381608F04EC2EE2EFF244CE050E0E49EE0
:10AE0000F001E59EF00DF49EF00D1124EA0DFB1DFE
:10AE1000EE0FFF1FEA54FC4F0190F081E02D07FD7B
:10AE200002C020E8201B55244424E29F1001F29F19
:10AE3000300C411C11245527452D342D232D809194
:10AE4000CF06689F400111246624399D2001289D6A
:10AE50001001389D300C411C561C299D300C411CA2
:10AE6000561C1124C201AA27BB279C0107FDDEC185
:10AE7000DF01A21BB30B0CE010E0E09EF001E19EAD
:10AE8000F00DF09EF00D1124EA0DFB1DEA52FB4F70
:10AE900050808091D006589E600111248D2D9927F5
:10AEA00087FD9A95452D55279927BA01680F791F77
:10AEB0006F3F710511F008F0A3C1762F66276F6F01
:10AEC000481B590B942F88276A177B0708F09BC1F2
:10AED000DB012CE030E0E29EF001E39EF00DF29EFB
:10AEE000F00D1124EA0DFB1DE2CE6217730708F086
:10AEF00037CEB90135CE4FEF5FEF29CEA817B9078E
:10AF000008F0F6CCDC01F4CC6FEF7FEFE8CC6217F1
:10AF1000730708F095CDB90193CD4FEF5FEF87CD63
:10AF20006217730708F03ECFB9013CCF4FEF5FEFD8
:10AF300030CF1482159D500111248B2D99278583C4
:10AF40004981182F003809F4A4C13091CE06381772
:10AF500008F09FC1E42EFF24ACE0B0E06A9FF0014E
:10AF60006B9FF00D7A9FF00D1124EE0DFF1DEE0F7B
:10AF7000FF1FEA54FC4F0190F081E02D07FD02C055
:10AF800020E8201B77246624E29F2001F29F500CCA
:10AF9000611C11245527472D362D252D8091CF0674
:10AFA000189FA00111246624359F2001249F1001C1
:10AFB000349F300C411C561C259F300C411C561CE4
:10AFC0001124C201AA27BB279C0107FD39C1DF015B
:10AFD000A21BB30B0CE010E0609FF001619FF00D2D
:10AFE000709FF00D1124EE0DFF1DEA52FB4F708093
:10AFF0008091D006789E40011124892D992787FDE4
:10B000009A95472D55279927FA01E80FF91FEF3F29
:10B01000F10511F008F003C1FE2FEE27EF6F481B7A
:10B02000590B942F8827EA17FB0708F0F2C0DF01BD
:10B030002CE030E0629FF001639FF00D729FF00DF5
:10B04000112433CEA817B90708F026CEDC0124CE90
:10B050006FEF7FEF18CE22273327261B370B82177F
:10B06000930708F4CAC06FEF7FEF6FCE802F805830
:10B070003ECE662777276E1B7F0B8617970708F44F
:10B08000B5C0AFEFBFEF06CC88249924861A970A83
:10B090008815990508F4A7C06FEF7FEF34CD2227FC
:10B0A0003327261B370B8217930708F4A3C06FEFD3
:10B0B0007FEF99CC802F805800CD802F805865CCB1
:10B0C000662777276E1B7F0B8617970708F4AAC0A1
:10B0D000AFEFBFEFB3CD1682859CA0011124852F61
:10B0E00099278783182F003809F4D3C0D090CE0653
:10B0F000D81608F0CEC0ACE0B0E06A9FF0016B9FBC
:10B10000F00D7A9FF00D1124EA0DFB1DEE0FFF1FCD
:10B11000EA54FC4F0190F081E02D07FD02C020E8C9
:10B12000201BBB27AA27E29FC001F29F900DA11D03
:10B130001124292F3A2F4B2F55278091CF06189F86
:10B140007001112466243F9D20012E9D10013E9D1B
:10B15000300C411C561C2F9D300C411C561C1124D8
:10B16000C201AA27BB279C0107FD85C0DF01A21BE6
:10B17000B30B0CE010E0609FF001619FF00D709F39
:10B18000F00D1124EA0DFB1DEA52FB4F90808091D7
:10B19000D006989E30011124872D992787FD9A9516
:10B1A000492D55279927FA01E80FF91FEF3FF105BF
:10B1B00011F008F04FC0FE2FEE27EF6F481B590B20
:10B1C000942F8827EA17FB0708F047C0DF012CE01F
:10B1D00030E0629FF001639FF00D729FF00D11242B
:10B1E000EA0DFB1D64CD680F791F8DCCDF01A20F26
:10B1F000B31F50CB680F791FF6CB680F791FA5CD11
:10B200006FEF7FEF5DCEA817B90708F062CEDC01C3
:10B2100060CEA817B90708F00BCFDC0109CFEFEF1C
:10B22000FFEFFDCEDF01A20FB31F08CD6627772702
:10B230006E1B7F0B86179707B0F0AFEFBFEF1BCEEB
:10B24000882799278E1B9F0B2817390780F0AFEFAF
:10B25000BFEFC0CEEFEFFFEFB1CFA817B90708F0EF
:10B26000B6CFDC01B4CFDF01A20FB31F04CEDF01E4
:10B27000A20FB31FAFCE222433242E1A3F0A821509
:10B28000930518F0AFEFBFEF74CFDF01A20FB31F2C
:10B2900070CF29960FB6F894DEBF0FBECDBFDF91F9
:10B2A000CF911F910F91FF90EF90DF90CF90BF90C3
:10B2B000AF909F908F907F906F905F904F903F9056
:10B2C0002F900895869F90011124832F992787FD41
:10B2D0009A95982F8091CA06981718F481E090E00B
:10B2E000089580E090E008950895CF92DF92EF9264
:10B2F000FF920F931F93CF93DF93DC018B0140E00C
:10B3000050E0FC012FE08191480F511D215027FF93
:10B31000FACFEA01D295C295CF70CD27DF70CD2745
:10B32000F801C08320E030E060E0FD01A9018191D7
:10B3300099278C1B9D0B2227999F7001889F600184
:10B34000989FD00CE11CF21E899FD00CE11CF21ECC
:10B3500011249A012C0D3D1D2417350720F06F5F35
:10B36000603120F302C04FEF5FEF529542954F706E
:10B3700045275F704527E80149835A83DF91CF91C4
:10B380001F910F91FF90EF90DF90CF900895689FED
:10B39000C00111248F3F910518F080E090E00895DE
:10B3A0008095992708950895EF92FF920F931F9328
:10B3B000CF9340913E01E42FFF27E05CFE4F809148
:10B3C0004B038083709620913F033091400380911E
:10B3D000D50699278F709070029709F463C103E036
:10B3E0002C3F3007B8F08FEF90E08083E42FFF27E9
:10B3F000E05CFE4FE0902703E0A2E42FEF5FE03136
:10B40000D8F4E0933E01F0903C03F3FC1BC0109293
:10B410003F016CC13695279536952795822F992740
:10B420008083E42FFF27E05CFE4FE0902703E0A23B
:10B43000E42FEF5FE03128F310923E01F0903C03DF
:10B44000F3FEE5CF909141030091C9069017F8F201
:10B45000C0913F01CF5FCA3108F42BC120E030E03A
:10B46000E0E4F1E09FE01191210F311D915097FF31
:10B47000FACFB901729562956F7067277F70672761
:10B480006093C20780E090E030E0E0E4F1E0AC01DE
:10B4900081919927861B970B2227999F8001889F6E
:10B4A0007001989FF00C011D121F899FF00C011D67
:10B4B000121F1124D801C701840F951F8417950707
:10B4C00008F400C13F5F303110F3529542954F7040
:10B4D00045275F704527E2ECF7E04183528320E087
:10B4E00030E0E0E5F1E09FE04191240F311D915003
:10B4F00097FFFACFB901729562956F7067277F70D9
:10B5000067276093C50780E090E030E0E0E5F1E078
:10B51000AC0181919927861B970B2227999F800167
:10B52000889F7001989FF00C011D121F899FF00CDD
:10B53000011D121F1124D801C701840F951F841704
:10B54000950708F4BCC03F5F303110F35295429527
:10B550004F7045275F704527E5ECF7E04183528344
:10B5600020E030E0E0E6F1E09FE05191250F311D51
:10B57000915097FFFACFB901729562956F70672766
:10B580007F7067276093C80780E090E030E0E0E6D6
:10B59000F1E0AC0181919927861B970B2227999F97
:10B5A0008001889F7001989FF00C011D121F899FD8
:10B5B000F00C011D121F1124D801C701840F951F23
:10B5C0008417950708F478C03F5F303110F3529527
:10B5D00042954F7045275F704527E8ECF7E04183BF
:10B5E00052833091C2072091C507329FD0011124A8
:10B5F0008B2F992787FD9A957091CA06871708F0B7
:10B600004DC03093B7072093B8072091C807209307
:10B61000B9079091C3078091CB06899FC00111247F
:10B620008F3F910508F458C080E090E0582F90912A
:10B63000C6078091CC06899FC00111248F3F9105D8
:10B6400008F447C080E090E0482F9091C9078091AE
:10B65000CD06899FC00111248F3F910508F435C0A4
:10B6600020E030E05093BF074093C0072093C1070C
:10B67000549F7001112477276627E29EA001F29E55
:10B68000500D611D1124CB01AA27BB278093BA0757
:10B69000882321F03091D10631FF21C0BAE0B09368
:10B6A0003F0124C0369527953695279536952795E1
:10B6B000B5CEC0933F011AC04FEF5FEF88CF4FEF79
:10B6C0005FEF44CF4FEF5FEF00CF8095282F3327F8
:10B6D000C9CF80959927B8CF80959927A7CFC093D8
:10B6E0003F0187EB97E00E944353D8CFCF911F9142
:10B6F0000F91FF90EF90089520E0E6EDF4E0DF0178
:10B70000A052B1408D919D9180589F4F892F9927CC
:10B7100081932F5F2039B0F3089520E0E6EDF4E047
:10B72000DF01A052B14081919927982F88278F6718
:10B730008D939D932F5F2039B0F3089508950F9353
:10B740006091450320914D0330914E033695279526
:10B75000369527950091730699E1099FA001112460
:10B7600080916D0687FD03C0109236031EC0709154
:10B770003C0375FDF9CFA0916F06A617A8F34217F9
:10B78000530790F7241B350BF901E070EF2B59F0AC
:10B790000FEF20E140E060917206842F0E9409279C
:10B7A0008093360302C0022FF4CF0F910895CF93F8
:10B7B000DF93382F80916D0684FF04C020913B03F6
:10B7C00027FD04C0832F432F552758C040914D03B8
:10B7D00050914E039091CB078AE0989FC0011124AD
:10B7E0004817590720F5841B950BA0918E067727E3
:10B7F00066278A9FA0019A9F500D611D1124FB01AD
:10B80000EA018D2F9E2FAF2FBB27BC0180919006A0
:10B8100099278617970778F1432F55279A01260F06
:10B82000371FE32FFF27EF2B41F18FEF27C0481B76
:10B83000590B60918E06FF27EE27469FE001569F29
:10B84000D00DE11D11248D2F9E2FAF2FBB27BC01E2
:10B850008091910699278617970758F0432F55270F
:10B860009A01261B370B832F9927892B31F080E013
:10B8700005C0BC01F3CFBC01CFCF822F282F3327C7
:10B88000C901841B950B9093DF078093DE07C901E4
:10B89000DF91CF910895282F80916D06992783FF1E
:10B8A00012C082FF10C08091CC0782FD12C090911F
:10B8B000CE07291778F4921B9093CD078D7F816076
:10B8C0008093CC0708952093E2072093CE0710922F
:10B8D000CD070895291B2093CD078360F1CF0895EC
:10B8E000CF92DF92EF92FF920F931F93CF93DF934C
:10B8F00080913B0380FF04C0C0903B03C1FE71C038
:10B90000F89400913B030F7700933B0378941092D7
:10B91000D2071092D10780917E0699279695982F8D
:10B920008827979587959093D0078093CF0710929B
:10B93000D4071092D3071092D6071092D507109211
:10B94000D8071092D7071092DA071092D9071092F1
:10B95000DC071092DB07909182068AE0989FC00175
:10B9600011248093DD071092DF071092DE07E0902C
:10B970007706E09272019091760690937301D090D1
:10B980007206D90ED092CB07D09274010091410378
:10B9900020917506409174066DEC80E00E940927A5
:10B9A00090916E06981708F050C19093E00720918F
:10B9B000E00780916D06992783FF40C182FF3EC159
:10B9C0008091CC0782FD36C29091CE07291708F0EE
:10B9D000EEC1921B9093CD078D7F81608093CC0741
:10B9E00029C210914503F0906F06F11608F430C19A
:10B9F00020913B0327FD07C0F89430913B0330684A
:10BA000030933B037894C0904D03D0904E03009147
:10BA100041032091730640917206609171068091F6
:10BA200070060E940927282F90917201992309F42A
:10BA30004AC191509093720180917301820F80935B
:10BA4000CB075AE0859F900111242C193D094091A4
:10BA50006D0646FF05C01216130614F4220F331F9D
:10BA60003093D2072093D1074091D1075091D2074C
:10BA70009A0157FDAAC18091800699272817390796
:10BA80000CF42AC160917001709171016C197D09EB
:10BA90007093D4076093D3079A0157FDA7C1809193
:10BAA0007F069927281739070CF02EC17091790667
:10BAB0004050504811270027479F7001579FF00CB6
:10BAC000011D1124BB27A12F902F8F2DFC01472F83
:10BAD00055275695542F442757954795E41BF50B4A
:10BAE000F093D807E093D707C091CF07D091D00744
:10BAF00010917A06C050D04877276627C19FA001D1
:10BB0000D19F500D611D1124BB27A72F962F852F84
:10BB1000BC01E12EFF24F694FE2CEE24F794E7946A
:10BB20006E197F097093DA076093D907A091D30744
:10BB3000B091D407F0907B06A050B048332722275D
:10BB4000AF9D8001BF9D100D211D1124BB27A32F88
:10BB5000922F812F8C018F2D99279695982F8827CA
:10BB600097958795081B190B1093DC070093DB074B
:10BB70007F01E60EF71EE00EF11EF594E794F594B2
:10BB8000E794F594E794F594E794F092D607E09261
:10BB9000D507F0913A036F2F77276E5D794F9B01A0
:10BBA0002F593F4F90913903E92FFF27EE5DF94F51
:10BBB000AF014F595F4F00914103E9012881EA012C
:10BBC0004881EB01688580850E9409279701280F2D
:10BBD000311DE091CE07EE2341F48091DD078823EB
:10BBE00009F4F8C081508093DD0780916E06992793
:10BBF00040E050E0BC01C9010E945A298093E0074F
:10BC0000982FB0916D062B2F332723FFD7C022FF2B
:10BC1000D5C08091CC0782FD0CC02091CE07921731
:10BC200008F0FCC0291B2093CD078D7F8160809395
:10BC3000CC07D0927101C0927001FCC02093E20742
:10BC40002093CE071092CD07F5C08093E007AFCECA
:10BC5000C0903B03C7FEEEC0F89430913B033F77A2
:10BC600030933B0378941092D2071092D107109230
:10BC7000D0071092CF071092D4071092D3071092DA
:10BC8000D6071092D5071092D8071092D7071092B6
:10BC9000DA071092D9071092DC071092DB07909117
:10BCA00082068AE0989FC00111248093DD0780916D
:10BCB0006D06992783FFBEC082FDBCC01092E207CB
:10BCC0001092CE07BFCF80917301882309F4B6CEBE
:10BCD000815080937301B2CE2091DE073091DF074F
:10BCE00037FD89C0809192069927281739070CF4EF
:10BCF000A0CF8091CE079927141615060CF08AC0A4
:10BD00009C012F5F3F4F71CF9091E007992319F469
:10BD100055230CF4CBCE70916E06791709F475C0DB
:10BD2000A091CF07B091D007ED01EE27D7FDE095A8
:10BD3000FE2FCA01AA2797FDA095BA2FC80FD91FB9
:10BD4000EA1FFB1F8D2F9E2FAF2FBB27A7FDBA9594
:10BD5000803891050CF453C08FEF9FE79093D00784
:10BD60008093CF07B0917E06CB2FDD27D695DC2FB1
:10BD7000CC27D795C79580917D0699279695982FC2
:10BD8000882797958795909581959F4FAC01BE0127
:10BD90008091CF079091D0070E945A299093D007A5
:10BDA0008093CF074091D1075091D2077FCE291BB6
:10BDB0002093CD0783608093CC073CC09093E2072B
:10BDC0009093CE071092CD0734CF22273327241B20
:10BDD000350B51CE909182068AE0989FC0011124C4
:10BDE0008093DD0751E05093CE07FFCE2227332703
:10BDF000241B350B54CE309521953F4F73CF80587F
:10BE00009F4F9CF480E090E8A9CF141615060CF41F
:10BE10004DCE86CF9C0121503040E7CE921B9093AF
:10BE2000CD0783608093CC0704CFD093D007C09315
:10BE3000CF0798CFDF91CF911F910F91FF90EF9097
:10BE4000DF90CF900895F89485B3806F85BB969866
:10BE5000969A789480916D06992783FF3BC082FD66
:10BE600039C0E1EEF7E040E04093E1074093E2079C
:10BE7000F89460914F08709150082CB53DB53093FF
:10BE8000500820934F082617370748F4A09151080F
:10BE9000B09152081196B0935208A093510878942B
:10BEA000BB27AA27249FC001349F900DA11D1124F8
:10BEB000892F9A2FAB2FBB278383948325833683C7
:10BEC0002091CC072A7F2093CC071092CE071092A6
:10BED000CD07089545E04093CC0730916E06365F5C
:10BEE0003093CE073093CD07089508959927813078
:10BEF000910551F082309105D4F08230910551F0D6
:10BF0000039771F0E0E018C0E0916C06E695E695C5
:10BF1000E37012C0E0916C06E295EF70E3700CC024
:10BF2000E0916C06E295E695E695E37005C0892BF5
:10BF300049F7E0916C06E370FF27E854F74E8491CF
:10BF4000992708959091CD07992309F475C08091A0
:10BF50006D0681FF05C020913E03253408F4A4C07E
:10BF6000692F61506093CD074091CC07477F41FD19
:10BF70009CC030917501532F51508091CE07815054
:10BF80008093CE07F894852F83709927813091058F
:10BF900009F49CC0823091050CF4B0C08230910548
:10BFA00009F4A0C0039709F4BEC0E0E0FF27E854FD
:10BFB000F74E8491A5B3AF70992782959295907FA3
:10BFC0009827807F98278068A82BA5BB9698969A7B
:10BFD00078940000F8943370832F9927813091056D
:10BFE00009F47AC0823091050CF48FC0823091053B
:10BFF00009F47EC0039709F48FC0E0E0FF27E854FE
:10C00000F74E949175B37F709295907F792B75BBA5
:10C010009698969A78940000F89435B3306F35BBB3
:10C020009698969A789450937501662309F03AC0D1
:10C030004A7F4093CC0708955091CC075A7F509384
:10C04000CC0740916D0640FF2FC0F89485B38F70E8
:10C05000806785BB9698969A78940000F894F5B31B
:10C06000FF70F063F5BB9698969A78940000F89468
:10C07000E5B3EF70E064E5BB9698969A789400007B
:10C08000F894B5B3BF70B065B5BB9698969A78949E
:10C090000000F89465B36F70606665BB9698969AD9
:10C0A000789408954093CC07089530917501532FEB
:10C0B0005F5F8091CE078F5F8093CE07F894852FC6
:10C0C000837099278130910509F064CFE0916C0667
:10C0D000E695E695E3706ACFE0916C06E695E69505
:10C0E000E3708CCFE0916C06E295EF70E3705ECF69
:10C0F000E0916C06E295EF70E37080CF892B09F038
:10C1000054CFE0916C06E37051CF892B09F075CFC5
:10C11000E0916C06E37072CFE0916C06E295E695D3
:10C12000E695E3706BCFE0916C06E295E695E695B7
:10C13000E3703CCFAF92BF92CF92DF92EF92FF922B
:10C140001F93CF93DF9310916D0613FFB2C0B1EE32
:10C15000EB2EB7E0FB2EF89480914F089091500899
:10C160004CB55DB55093500840934F084817590798
:10C1700008F4D5C07894E091E607F091E707709154
:10C18000E2076091E107C1EED7E02091E40730912A
:10C19000E5074E175F0730F4862F9927D82ECC2459
:10C1A0002C193D097617A9F0671708F0D9C0972F09
:10C1B000961BDD24CC24499F5001599FB00CC11C13
:10C1C0001124BB27AD2D9C2D8B2D280F391F70936B
:10C1D000E1072B833C834D835E83B090E307BB2054
:10C1E00041F0EA01CE1BDF0B2C0F3D1FF70123832B
:10C1F0003483BB27AA27479FC001579F900DA11DDD
:10C200001124492F5A2F6B2F7727241B350B832F8F
:10C210009927853508F0DBC020E030E0E7012A836C
:10C22000A22FF89430918D06232F207F2A273F706C
:10C23000432F5527BA014230510509F04FC0E5E6BA
:10C24000F0E085B38F70822B85BB21E030E002C027
:10C25000220F331F4A95E2F7922F9095C080C92292
:10C26000C0821081122B108310916D0615FF1FC024
:10C2700078940000F89430918D06305F40E84A27AA
:10C28000232F207F24273F70432F5527BA014230A8
:10C29000510509F4ADC0433051050CF071C0411592
:10C2A000510509F4BBC04130510509F4D1C078945F
:10C2B0002EC1E090410390916406E916D0F1A0E010
:10C2C000F89430918D06232F207F2A273F70432F2B
:10C2D0005527BA014230510509F4B1CF4330510519
:10C2E000ACF54115510509F055C0822F992780778B
:10C2F0009070959587959595879595958795959542
:10C30000879527FDBEC0C82FDD27C256DC4F788138
:10C31000BBB3B72BBBBB8AB3872B8ABBA7CFA0917C
:10C320005108B09152081196B0935208A093510849
:10C3300021CFF09041032F2D3327892F9927039781
:10C34000281739070CF0E3C0A0E8BACF46305105F2
:10C3500021F04730510509F089CFE2E3F0E071CFD9
:10C36000671BDD24CC24469F5001569FB00CC11C96
:10C370001124BB27AD2D9C2D8B2D281B390B27CFCE
:10C380004630510521F04730510509F090CFE2E3E6
:10C39000F0E030C04130510509F068CF27FD8DC075
:10C3A000822F992780779070959587959595879599
:10C3B000959587959595879502C0660F771F8A9505
:10C3C000E2F7F62FF09588B38F2388BB4FCF8C3AD6
:10C3D00060F4A091B808B091B9081196B093B9086B
:10C3E000A093B808F7014383548320E830E016CFC8
:10C3F000E5E6F0E075B37F70722B75BB21E030E0AD
:10C4000002C0220F331F4A95E2F7622F60955081D8
:10C4100056235083F080F22AF08249CF822F992749
:10C420008077907095958795959587959595879543
:10C430009595879527FD33C0C82FDD27C256DC4F61
:10C44000D880EBB2ED28EBBA8AB38D298ABB2FCF07
:10C4500027FD48C0822F9927807790709595879502
:10C4600095958795959587959595879502C0660FC3
:10C47000771F8A95E2F7262F209588B3822388BB01
:10C4800016CFE82FFF27E256FC4F4081642F6095BE
:10C490005BB356235BBB8AB3842B8ABBE7CEE82F02
:10C4A000FF27E256FC4FA080AA2DA095BBB2BA226E
:10C4B000BBBA8AB38A298ABBFACE822F99278077A2
:10C4C0009070959587959595879595958795959570
:10C4D000879502C0660F771F8A95E2F788B3862B8F
:10C4E00088BBC4CE822F99278077907095958795C9
:10C4F00095958795959587959595879502C0660F33
:10C50000771F8A95E2F788B3862B88BBD0CEDF9160
:10C51000CF911F91FF90EF90DF90CF90BF90AF90A1
:10C5200008958B9A9398E3B34E2F55274F70507010
:10C530008B98B0916400B160B0936400A0916500E5
:10C54000AE7FA093650042955295507F5427407F5F
:10C55000542783B399278F709070482B592B909153
:10C5600064009E7F90936400709164007260709389
:10C570006400309165003D7F30936500429552958F
:10C58000507F5427407F542763B3262F33272F70C3
:10C590003070809164008D7F80936400CA01822B8B
:10C5A000932B08958B9A9398E3B32E2F33272F70F4
:10C5B00030708B98B0916400B160B0936400A0912A
:10C5C0006500AE7FA093650022953295307F3227BB
:10C5D000207F322783B399278F709070282B392BB7
:10C5E000909164009E7F90936400709164007260EB
:10C5F00070936400509165005D7F509365002295B3
:10C600003295307F3227207F322783B399278F706E
:10C610009070282B392B409164004D7F409364002B
:10C620004091760150917701609178017091790184
:10C630004623572340955095422B532B70937701F7
:10C64000609376013093790120937801CA019F703D
:10C650008F5F9F4091F020E061E070E0CA01862783
:10C660009727FC01E170F07080FD0AC05695479550
:10C670002F5F2C3098F3CF01089580E090E008956B
:10C68000E22FFF27E85FFE4F8081992708950895E4
:10C6900054B3507F54BB45B34F6045BB8B9830912A
:10C6A00064003E7F30936400209164002D7F2093CE
:10C6B00064008FEF9FEF90937901809378019093BE
:10C6C000770180937601089582958F70E82FFF2778
:10C6D000EC53F74E849199270895E82FFF27EF70C8
:10C6E000F070EC53F74E849199270895E0E002C072
:10C6F000EC5E86518631E0F7882359F0823060F095
:10C70000FF27E851F84FE80FF11D319780819927F5
:10C7100008958DE090E008958AE090E008950895EE
:10C72000282F869586958695A82FBB27A75CB74F9F
:10C73000E22FFF27E770F070E454F74E94918C914C
:10C740008923992787FD909508958091D306982F86
:10C7500092959F709A95F1F7A99A8F708A95F1F743
:10C76000A9980895582FF89465B36F70606865BBF9
:10C7700060E470E0EFEB72B37E2372BB32B3362B12
:10C7800032BB78940000F89425B32F70807F822B01
:10C7900085BBB091D3064B2F42954F70F42FFA957D
:10C7A000F1F7A99A7B2F7F70972F9A95F1F7A998A7
:10C7B00078940000F894A5B3AF70852F99278295DF
:10C7C0009295907F9827807F9827A82BA5BB4A95A4
:10C7D000F1F7A99A7A95F1F7A99878940000F8945E
:10C7E00035B33F7035BB22B32E2322BB82B3862BD9
:10C7F00082BB78940E9465210895F8946FE064BB31
:10C80000A998A89A3091D306932F92959F70592F8B
:10C810005A95F1F7A99A3F70432F4A95F1F723B340
:10C82000A9989A95F1F7A99A3A95F1F7A998A89835
:10C830008FEF84BB78942078822F99270895982FC2
:10C84000862F8F5F8035E8F010924508262F33271A
:10C85000D901A851B84FFD018181891789F09183D1
:10C86000669566956695A62FBB27A75CB74F277080
:10C8700030702454374EF90194912C91292B2C932C
:10C88000089580934508E2CF0F931F93CF93DF93D2
:10C890008C0150E0962F6035C8F5E80128812223ED
:10C8A000A9F1A0E0B0E027C010924508292F332756
:10C8B000D901A851B84FED0169816E1789F0E9835C
:10C8C000969596959695C92FDD27C75CD74F27700B
:10C8D00030702454374EF90194913881392B3883C4
:10C8E000942F403598F4A52FBB27FD01E00FF11FD1
:10C8F0004081442359F0A00FB11F5F5FEC91492F95
:10C900004F5F403588F640934508D0CFDF91CF91F7
:10C910001F910F910895AC0197FD26C0862F8F5F60
:10C920008035F8F480934508262F3327C9018851B4
:10C93000984FFC01B181BB3291F09BE291836695E7
:10C9400066956695A62FBB27A75CB74F27703070FA
:10C950002454374EF90164913C91362B3C93CA0123
:10C96000089510924508E0CF862F8F5F803508F537
:10C9700080934508262F3327F901E851F84F81812C
:10C980008D3291F07DE27183669566956695A62F4E
:10C99000BB27A75CB74F277030702454374EF9017E
:10C9A00094912C91292B2C9388279927841B950BE4
:10C9B000089510924508DECFEF92FF920F931F93D8
:10C9C000CF93DF93EC01162FB2E0FB2EE0E4FCE9FD
:10C9D00024E040E350E00EE06EE070E0CE17DF07A9
:10C9E00020F0CE1BDF0B420F511DF695E7952695E3
:10C9F000CB0183709070892B49F5E12E1F5F2E2D9E
:10CA00003327D901A851B84FFD015181541789F03E
:10CA10004183E694E694E694AE2DBB27A75CB74F1E
:10CA2000277030702454374EF9012491EC90E22A9B
:10CA3000EC92EF2DFF27EE0FFF1FEC5EFE4FFA94F6
:10CA40000190F081E02D28E040E350E0015061507A
:10CA5000704007FFC3CF9C2F905D812F8F5F803583
:10CA6000E0F010924508212F3327F901E851F84FE3
:10CA7000F180F916A9F09183169516951695C12F98
:10CA8000DD27C75CD74F277030702454374EF9012B
:10CA900014910881012B088303C080934508E3CFDC
:10CAA000DF91CF911F910F91FF90EF9008951F9309
:10CAB000CF93DF93EC01742F77FD55C0E72FFF274D
:10CAC000EE0FFF1FEC5EFE4F71500190F081E02DE4
:10CAD00040E350E0CE17DF0720F0CE1BDF0B48E32A
:10CAE00050E0CF0196958795C817D90720F0C81B4D
:10CAF000D90B4C5F5F4FCF0196958795969587959B
:10CB0000C817D90720F0C81BD90B4E5F5F4FF695A9
:10CB1000E795F695E795F695E795CE17DF0720F0B0
:10CB2000CE1BDF0B4F5F5F4F162F6F5F212F332719
:10CB3000D901A851B84FFD018181841709F4BCCFF8
:10CB40004183169516951695A12FBB27A75CB74F65
:10CB5000277030702454374EF90124911C91122B08
:10CB60001C9377FFABCFCA30D10508F1862F8F5FBA
:10CB7000803578F110924508262F3327F901E851C6
:10CB8000F84F41814D3A59F15DEA518366956695BA
:10CB90006695C62FDD27C75CD74F277030702454A9
:10CBA000374EF90164913881362B388318C09C2F99
:10CBB000905D862F8F5F803578F010924508262F84
:10CBC0003327F901E851F84F7181791741F09183CA
:10CBD000DDCF80934508D0CF80934508F0CFDF911B
:10CBE000CF911F910895482FA998F89435B33F70BD
:10CBF000407F342B35BB9091D306292F22952F707F
:10CC00002A95F1F7A99A892F8F708A95F1F7A9983B
:10CC100078940895582FF894A5B3AF70782F707F4B
:10CC20007A2B75BB6091D306462F42954F70942F97
:10CC30009A95F1F7A99A362F3F70832F8A95F1F7CD
:10CC4000A99878940000F89425B32F70852F992720
:10CC500082959295907F9827807F9827282B25BBD7
:10CC60004A95F1F7A99A3A95F1F7A99878940E9414
:10CC700065210895F89465B36F7065BB5091D30634
:10CC8000452F42954F70942F9A95F1F7A99A352F19
:10CC90003F70832F8A95F1F7A99878940000F89453
:10CCA00025B32F7081E090E082959295907F982730
:10CCB000807F9827282B25BB4A95F1F7A99A3A95AA
:10CCC000F1F7A99878940E9465210895109244087C
:10CCD000F89465B36F7065BB5091D306452F4295AC
:10CCE0004F70942F9A95F1F7A99A352F3F70832FA3
:10CCF0008A95F1F7A99878940000F89425B32F70DD
:10CD000082E090E082959295907F9827807F982787
:10CD1000282B25BB4A95F1F7A99A3A95F1F7A998DE
:10CD200078940E94652110924508089558E081305A
:10CD300029F0613031F0413041F406C05CE06130EF
:10CD4000D1F75260413009F45160F894A5B3AF7047
:10CD5000752F707F7A2B75BB6091D306462F429555
:10CD60004F70942F9A95F1F7A99A362F3F70832F21
:10CD70008A95F1F7A99878940000F89425B32F705C
:10CD8000852F992782959295907F9827807F982765
:10CD9000282B25BB4A95F1F7A99A3A95F1F7A9985E
:10CDA00078940E9465210895582F5068F894A5B38F
:10CDB000AF70752F707F7A2B75BB6091D306462FAD
:10CDC00042954F70942F9A95F1F7A99A362F3F709C
:10CDD000832F8A95F1F7A99878940000F89425B3E9
:10CDE0002F70852F992782959295907F9827807F25
:10CDF0009827282B25BB4A95F1F7A99A3A95F1F780
:10CE0000A99878940E9465210895CF93C82F8C33F8
:10CE100018F0582F585E0BC0883218F0582F545114
:10CE200006C0843118F0582F545D01C0582F506847
:10CE3000F894A5B3AF70752F707F7A2B75BB609196
:10CE4000D306462F42954F70942F9A95F1F7A99AE1
:10CE5000362F3F70832F8A95F1F7A99878940000B8
:10CE6000F89425B32F70852F992782959295907FFE
:10CE70009827807F9827282B25BB4A95F1F7A99AF8
:10CE80003A95F1F7A99878940E946521C0934308D8
:10CE9000CF9108951F93CF93DF935091D20650FF07
:10CEA00020C0F8946FE064BBA998A89A1091D306AB
:10CEB000912F92959F70492F4A95F1F7A99A1F706B
:10CEC000312F3A95F1F723B3A9989A95F1F7A99ADA
:10CED0001A95F1F7A998A8988FEF84BB789427FD4D
:10CEE000BDC010914408C12FC695C695C695AC2FFC
:10CEF000BB27A75CB74FC12FDD27FE01E770F0709D
:10CF0000E454F74E94914C91742F7923272F3327B3
:10CF100027FD3095222309F43FC0209143082117B3
:10CF200009F470C01C3308F06AC0183208F487C0D6
:10CF3000512F54515068F89445B34F70352F307FBE
:10CF4000342B35BB8091D306F82FF295FF709F2FBD
:10CF50009A95F1F7A99AA82FAF70BA2FBA95F1F761
:10CF6000A99878940000F89425B32F70852F9927FD
:10CF700082959295907F9827807F9827282B25BBB4
:10CF8000FA95F1F7A99AAA95F1F7A99878940E94D1
:10CF900065211093430862C0912F9F5E96959695E8
:10CFA00096958AE0981748F5E92FFF27E75CF74F39
:10CFB000E081EE2371F4815009F44BC09F5F9A30F9
:10CFC00098F390E0E92FFF27E75CF74FE081EE232D
:10CFD00091F3990F990F990F5E2F507F19F49C5F71
:10CFE000E295E07F1E2F107C19F49E5FEE0FEE0F8E
:10CFF000E7FF9F5F9093440831C0922FD5CF512F08
:10D00000585E98CF909549234C93C851D84FE981E9
:10D01000812F8F5F8035C0F01092440851FF08C007
:10D02000822F8F5F843121F0883211F08C3309F424
:10D030008FEF809343088E2F0E94B2630FC014318C
:10D0400030F0512F545D76CF80934408E7CF512FB5
:10D0500071CF990F990F990F90934408DF91CF9159
:10D060001F91089580934508089580914508992758
:10D070000895CF93DF93982FE09145088E2F8F5F0F
:10D080008035E8F0109245082E2F3327D901A8519A
:10D09000B84FED0189818917A9F09983E695E69546
:10D0A000E695CE2FDD27C75CD74F2770307024540C
:10D0B000374EF90194912881292B288303C080934E
:10D0C0004508E2CFDF91CF910895CF93DF93AC0174
:10D0D000EC019881992319F52BC0109245082E2F49
:10D0E0003327D901A851B84FED018981891789F0FB
:10D0F0009983E695E695E695CE2FDD27C75CD74F59
:10D10000277030702454374EF90194912881292BCF
:10D1100028834F5F5F4FFA019081992349F0E09196
:10D1200045088E2F8F5F8035C0F680934508D7CF96
:10D13000DF91CF910895CF93DF93FC01AC014F5F56
:10D140005F4F9491992371F16091450822C060E08E
:10D150002E2F3327D901A851B84FED0189818917A6
:10D1600089F09983E695E695E695CE2FDD27C75C95
:10D17000D74F277030702454374EF901949128818D
:10D18000292B2883FA014F5F5F4F3491932F33236C
:10D1900039F0E62F862F8F5F8035C8F6682FD8CFFD
:10D1A00060934508DF91CF910895CF93DF93FC0101
:10D1B000AC014F5F5F4F94919923A1F161506F3F94
:10D1C00089F17091450825C070E02E2F3327D901D1
:10D1D000A851B84FED018981891789F09983E695A7
:10D1E000E695E695CE2FDD27C75CD74F27703070C8
:10D1F0002454374EF90194912881292B2883FA0170
:10D200004F5F5F4F3491932F332351F061506F3F45
:10D2100039F0E72F872F8F5F8035B0F6782FD5CF85
:10D2200070934508DF91CF910895CF93DF93E091FC
:10D2300045088E2F81508F3450F550E220C040E0D9
:10D240002E2F3327D901A851B84FED0169816032E3
:10D2500089F05983E695E695E695CE2FDD27C75CE4
:10D26000D74F277030702454374EF901949128819C
:10D27000292B2883E42F342F31503F3430F48E2F64
:10D280008F5F8035E0F6482FDBCF40934508DF9174
:10D29000CF910895CF93DF93582FE0914508EE2367
:10D2A00081F18E1770F1E03560F560E222C040E058
:10D2B0002E2F3327D901A851B84FED018981803233
:10D2C00089F06983E695E695E695CE2FDD27C75C64
:10D2D000D74F277030702454374EF901949128812C
:10D2E000292B2883E42F442351F0541740F0403574
:10D2F00030F48E2F8F5F8035D0F6482FD9CF4093F2
:10D300004508DF91CF910895CF93DF93E0914508D1
:10D31000EC3370F150E54E2FE51718F136C010923E
:10D3200045082E2F3327D901A851B84FED01898127
:10D33000803291F060E26983E695E695E695CE2F1E
:10D34000DD27C75CD74F277030702454374EF90162
:10D3500094912881292B28834F5F4517B0F4E091E1
:10D3600045088E2F8F5F8035D0F680934508D9CF42
:10D37000E83228F05CE34E2FE51798F306C0E4315D
:10D3800010F058E2C8CF54E1C6CFDF91CF91089595
:10D39000CF93DF93682F50E84091450823C0E42FD6
:10D3A000842F8F5F803590F1492F2E2F3327D9019D
:10D3B000A851B84FED018981803391F080E38983D2
:10D3C000E695E695E695CE2FDD27C75CD74F27700B
:10D3D00030702454374EF90194912881292B2883E9
:10D3E0005695C1F0962F9523D1F2E42F842F8F5FAD
:10D3F000803570F040E02E2F3327C9018851984FB7
:10D40000EC017981713361F381E3D9CF482FCDCF1E
:10D41000482FF1CF40934508DF91CF910895CF93E6
:10D42000DF93682F282F22952F70E22FFF27EC53D0
:10D43000F74E8491482F5527942FE09145088E2F61
:10D440008F5F803508F449C0109245082E2F33278E
:10D45000D901A851B84FED015981591789F0498375
:10D46000E695E695E695CE2FDD27C75CD74F27706A
:10D4700030702454374EF90194913881392B388318
:10D48000E62FFF27EF70F070EC53F74E4491E42F36
:10D49000FF274E2F90914508892F8F5F803500F12F
:10D4A00010924508292F3327D901A851B84FED0113
:10D4B00069816417C1F0E983969596959695C92F71
:10D4C000DD27C75CD74F277030702454374EF901E1
:10D4D000B49178817B2B788306C080934508B6CFC2
:10D4E00080934508DFCFDF91CF9108951F93CF93AD
:10D4F000DF93482F843608F055C01AE0612F0E9450
:10D5000002C6582F982F905DE09145088E2F8F5FAF
:10D51000803508F07BC0809345082E2F3327D90132
:10D52000A851B84FED018981891789F09983E69553
:10D53000E695E695CE2FDD27C75CD74F2770307074
:10D540002454374EF90194912881292B2883519F27
:10D55000C0011124642F681B605DE09145088E2F87
:10D560008F5F803508F455C0109245082E2F332761
:10D57000A9014851584FEA011981161709F44EC004
:10D580006983E695E695E695AE2FBB27A75CB74F76
:10D59000277030702454374EF90154913C91352B4B
:10D5A0003C933CC0E5EDF8E1AF014F5F5F4F9491D4
:10D5B0009923A1F16091450822C060E02E2F332706
:10D5C000D901A851B84FED017981791789F0998374
:10D5D000E695E695E695CE2FDD27C75CD74F2770F9
:10D5E00030702454374EF9018491B881B82BB88338
:10D5F000FA014F5F5F4F2491922F222369F0E62FAB
:10D60000862F8F5F8035C8F6682FD8CF10924508D7
:10D6100084CF80934508AACF60934508DF91CF91CE
:10D620001F9108950F931F93CF93DF93EC0183E035
:10D63000C83ED80708F093C004E610E0CE01B80158
:10D640000E940EC6962F905D40914508842F8F5FF3
:10D65000803508F0B8C080934508242F3327D901BE
:10D66000A851B84FFD018181891789F091834695B2
:10D6700046954695A42FBB27A75CB74F27703070FF
:10D680002454374EF90194912C91292B2C93609FAF
:10D69000A001619F500D709F500D11248E01041B3D
:10D6A000150BC8016AE070E00E940EC6962F905DCF
:10D6B000E09145088E2F8F5F803508F48AC0109264
:10D6C00045082E2F3327D901A851B84FED015981B4
:10D6D000591789F09983E695E695E695CE2FDD27D3
:10D6E000C75CD74F277030702454374EF901B4917E
:10D6F00038813B2B3883FB01EE0FFF1FEE0FFF1F1E
:10D70000EE0FFF1FE60FF71FE60FF71F0E1B1F0B95
:10D71000602F605DE09145088E2F8F5F803508F4A3
:10D7200055C0109245082E2F3327C9018851984FB4
:10D73000EC010981061709F451C06983E695E69565
:10D74000E695AE2FBB27A75CB74F277030702454E7
:10D75000374EF90164911C91162B1C933FC0E8EDE4
:10D76000F8E1AF014F5F5F4F94919923B9F1609158
:10D77000450822C060E02E2F332789010851184F39
:10D78000E8017981791789F09983E695E695E69520
:10D79000CE2FDD27C75CD74F277030702454374E0B
:10D7A000F9012491F881F22BF883FA014F5F5F4F62
:10D7B0003491932F332381F0E62F862F8F5F8035AE
:10D7C000C8F6682FD8CF1092450847CF80934508F8
:10D7D000AACF8093450875CF60934508DF91CF911C
:10D7E0001F910F910895A19AA09A08959FEFE9E3E0
:10D7F000F8E089E09193815087FFFCCF9093430834
:10D800000895CF93DF938093E80710924408109215
:10D8100045088091D20683FD31C0E8E4F8E04091EC
:10D82000D4064093480840934908F89460914F0803
:10D83000709150082CB53DB53093500820934F0897
:10D840002617370748F4A0915108B0915208119655
:10D85000B0935208A0935108C9017894DD27CC27D2
:10D86000249FD001349FB00DC11D11242B2F3C2FBC
:10D870004D2F5527238334838583968390E2E9EEE9
:10D88000F7E08FE49193815087FFFCCF9FEFE9E3AE
:10D89000F8E089E09193815087FFFCCF9093430893
:10D8A0009FB7F894A19AA09AA998A89834B3306F1A
:10D8B00034BB9FBFDF91CF910895CF93DF9329EDC4
:10D8C0002093E80710924408109245088091D206F0
:10D8D00083FD31C0E8E4F8E04091D4064093480865
:10D8E00040934908F89460914F08709150082CB506
:10D8F0003DB53093500820934F082617370748F45A
:10D90000A0915108B09152081196B0935208A0937B
:10D910005108C9017894DD27CC27249FD001349F7A
:10D92000B00DC11D11242B2F3C2F4D2F55272383C4
:10D9300034838583968390E2E9EEF7E08FE4919358
:10D94000815087FFFCCF9FEFE9E3F8E089E09193F6
:10D95000815087FFFCCF909343089FB7F894A19A1A
:10D96000A09AA998A89834B3306F34BB9FBFDF91B9
:10D97000CF9108952FEF209343088CEF8093E80711
:10D980000895282F90E0E9EEF7E0822F890F819328
:10D990009F5F9035D0F39FEFE9E3F8E089E0919342
:10D9A000815087FFFCCF909343080895CF93DF9376
:10D9B0003091E807232F2F5F832F9927873F910509
:10D9C00009F469C0883F91051CF1893F910509F46C
:10D9D000BCC0893F91050CF490C08A3F910509F4C1
:10D9E000D4C08C3F910509F43CC02093E8073D3F2B
:10D9F00008F444C1509145085F5F50934508552392
:10DA000009F498C07091E80771507093E80736C127
:10DA10002093E807843F910571F0853F910544F01C
:10DA2000853F910541F0863F910509F790E204C0DA
:10DA3000833F9105E1F690E3A998F89435B33F70E0
:10DA4000932B95BB9091D306292F22952F702A9561
:10DA5000F1F7A99A892F8F708A95F1F7A998789490
:10DA60000DC1809143088F5F80934308582F5695CE
:10DA70005F3708F487C02093E80780FFFDC0E52FDB
:10DA8000FF27E0FFEEC0EF70F070EC53F74E84918B
:10DA90000E94B263F3C02093E80758E2F89495B36C
:10DAA0009F70652F607F692B65BBF091D3064F2F68
:10DAB00042954F70342F3A95F1F7A99A3F2F3F7056
:10DAC000B32FBA95F1F7A99878940000F89425B38C
:10DAD0002F70852F992782959295907F9827807F28
:10DAE0009827282B25BB4A95F1F7A99A3A95F1F783
:10DAF000A99878940E946521C1C02093E807F89402
:10DB000045B34F7045BB6091D306462F42954F7089
:10DB1000742F7A95F1F7A99A362F3F70532F5A95A3
:10DB2000F1F7A99878940000F89425B32F708CE051
:10DB300090E0D1CF9FEFE9E3F8E089E09193815045
:10DB400087FFFCCF9093430899C02093E807F8948F
:10DB5000E5B3EF70E5BBB091D3064B2F42954F7004
:10DB6000C42FCA95F1F7A99A3B2F3F70A32FAA950E
:10DB7000F1F7A99878940000F89425B32F7086E007
:10DB800090E0A9CF3093E80778CF2093E807F89486
:10DB900045B34F7045BB6091D306562F52955F70C9
:10DBA000752F7A95F1F7A99A362F3F70932F9A9592
:10DBB000F1F7A99878940000F89425B32F7081E0CC
:10DBC00090E082959295907F9827807F9827282BC8
:10DBD00025BB5A95F1F7A99A3A95F1F7A998789447
:10DBE0000E9465218FEF8093430810924508F091C1
:10DBF000D206F3FD33C0E8E4F8E04091D406409348
:10DC0000480840934908F894A0914F08B0915008F3
:10DC10002CB53DB53093500820934F082A173B0789
:10DC200048F4C0915108D09152082196D0935208DF
:10DC3000C0935108C9017894DD27CC27249FD001D7
:10DC4000349FB00DC11D11249D01AE01232F342F2F
:10DC5000452F552723833483858396831092E807C5
:10DC60000DC0829586958770E82FFF27EC53F74EFD
:10DC700084910E94B26302C0506810CFDF91CF91AF
:10DC800008950F931F93CF93DF938C01462F97FD39
:10DC90002AC0E09145088E2F8F5F803508F580936C
:10DCA00045082E2F3327C9018851984FEC0169810F
:10DCB0006B3291F0BBE2B983E695E695E695AE2F1F
:10DCC000BB27A75CB74F277030702454374EF9013B
:10DCD00074913C91372B3C9360914508C80130C04A
:10DCE00010924508DECF90914508892F8F5F8035CF
:10DCF00020F580934508292F3327D901A851B84F23
:10DD0000ED0189818D3291F05DE25983969596956A
:10DD10009695C92FDD27C75CD74F277030702454E4
:10DD2000374EF90194912881292B28836091450869
:10DD300088279927801B910B03C010924508DBCFE1
:10DD40000E945765DF91CF911F910F910895FC01BB
:10DD5000E058FF4F11921192108208950F931F9374
:10DD6000CF93DF939C018A01DC01A058BF4FEC9157
:10DD7000EF3138F0FC01EF57FF4F80818F5F8083D8
:10DD800049C04E2F4F5F4C93423090F0542F569520
:10DD9000A52FBB27AA0FBB1FAA0FBB1FFD01E80FB2
:10DDA000F91F80819181EB01C81BD90BD7FD0CC0F5
:10DDB000E42FFF27EE0FFF1FEE0FFF1FE20FF31FF1
:10DDC00060837183028326C0E42FFF27EE0FFF1FBD
:10DDD000EE0FFF1FE20FF31FA20FB31F8D919C9157
:10DDE000119780839183ED011A811283452F523060
:10DDF000F8F25695A52FBB27AA0FBB1FAA0FBB1F72
:10DE0000ED01C20FD31F88819981FB01E81BF90B3B
:10DE1000DAF2CECFDF91CF911F910F910895CF927B
:10DE2000DF92EF92FF920F931F93CF93DF936C01DA
:10DE3000DC01A058BF4F8C91882339F4F601EE57CE
:10DE4000FF4F80818F5F808364C0E82EEA94EC925C
:10DE5000EE2009F45EC0E82FFF27EE0FFF1FEE0F44
:10DE6000FF1FEC0DFD1D00811181E6010C831D8358
:10DE7000F280FE8221E0F22E3DC0062F1127D8014C
:10DE8000AA0FBB1FAA0FBB1FAC0DBD1D472F5527E7
:10DE9000EA01CC0FDD1FCC0FDD1FCC0DDD1D8D91F8
:10DEA0009C9128813981821B930B97FD2FC0AF2D48
:10DEB000BB27AA0FBB1FAA0FBB1FAC0DBD1DFA01CC
:10DEC000EE0FFF1FEE0FFF1FEC0DFD1D4D915C913E
:10DED000119720813181CA01821B930BD2F02D93BF
:10DEE0003C93119740835183ED019A8112811A83EB
:10DEF0009283F72E7F2D770FE71658F0672F6F5F0D
:10DF0000E61608F0BACF472F5527D1CF762FA801B4
:10DF1000CECFDF91CF911F910F91FF90EF90DF90C7
:10DF2000CF900895CF92DF92EF92FF920F931F93BD
:10DF3000CF93DF936C01F60164837583468391E090
:10DF4000F92E00E810E0C00ED11EE601E880E0E8FE
:10DF5000FFEFCE0EDF1E3DC0062F1127D801AA0FFE
:10DF6000BB1FAA0FBB1FAC0DBD1D472F5527FA01C4
:10DF7000EE0FFF1FEE0FFF1FEC0DFD1DCD91DC918D
:10DF800020813181C21BD30BD7FD2FC0AF2DBB2702
:10DF9000AA0FBB1FAA0FBB1FAC0DBD1DFA01EE0FD0
:10DFA000FF1FEE0FFF1FEC0DFD1D4D915C911197B2
:10DFB00020813181CA01821B930BD2F02D933C93B7
:10DFC000119740835183ED019A81F280FA82928306
:10DFD000F72E7F2D770FE71658F0672F6F5FE61645
:10DFE00008F0BACF472F5527D1CF762FA801CECF33
:10DFF000DF91CF911F910F91FF90EF90DF90CF9025
:10E0000008959C01862F9927AC01B90187E891E01A
:10E010000E94AE6E089508959C0180917A01882334
:10E0200049F0A62FBB27AD01B90187E891E00E9416
:10E03000AE6E089541E040937A01E62FFF27AF01CD
:10E04000B90187E891E00E94926F08950895809148
:10E050007A01882319F010927A01089587E891E0F7
:10E060000E940F6F089508959C01862F9927AC0197
:10E07000B90187E891E00E94926F08950F931F9372
:10E08000CF93DF93E82F86E0E89FD0011124A659B3
:10E09000BC4F4D915C9111974115510571F1ED0106
:10E0A0000A811B81C0914F08D09150083E2F3295B4
:10E0B000307FFF27E256FC4F2081922F90957BB353
:10E0C00079237BBB6AB3622B6ABBBE01640F751FE9
:10E0D000FD01648375830417150748F0832F865F5D
:10E0E0009927AC0187E891E00E94926F0AC0BE01B7
:10E0F000600F711F832F875FF3CF87E891E00E9445
:10E100000F6FDF91CF911F910F9108950F931F9380
:10E11000CF93DF93E82F86E0E89FD0011124A65922
:10E12000BC4F4D915C9111974115510571F1ED0175
:10E130000A811B81C0914F08D09150083E2F329523
:10E14000307FFF27E256FC4F2081922F90957BB3C2
:10E1500079237BBB6AB3622B6ABBBE01640F751F58
:10E16000FD01648375830417150748F0832F865FCC
:10E170009927AC0187E891E00E94926F0AC0BE0126
:10E18000600F711F832F875FF3CF87E891E00E94B4
:10E190000F6FDF91CF911F910F910895282F332793
:10E1A000D901A256BC4F9C9190955BB359235BBBA0
:10E1B0004AB349234ABBF901EE0FFF1FEE0FFF1FC1
:10E1C000E20FF31FE20FF31FE659FC4F80914F0857
:10E1D0009091500864817581861B970B499778F060
:10E1E00022953295307F3227207F3227822F865F1B
:10E1F0009927AC0187E891E00E94926F08953C91C5
:10E200006BB3632B6BBB2AB3232B2ABB87E891E04C
:10E210000E940F6F08950895A82FBB27FD01EE0FF0
:10E22000FF1FEE0FFF1FEA0FFB1FEA0FFB1FE65950
:10E23000FC4F80914F089091500824813581821BBA
:10E24000930B499748F4A256BC4F3C914BB3432BD8
:10E250004BBB9AB3932B9ABB87E891E00E940F6F58
:10E26000089599278130910551F0823091058CF104
:10E270000297D9F087E891E00E940F6F08956091AE
:10E28000630360957BB376237BBB5AB356235ABB9B
:10E2900040914F085091500860916E0370916F0348
:10E2A000461B570B4931510568F4B0916303EBB33A
:10E2B000EB2BEBBBAAB3AB2BAABB87E891E00E9488
:10E2C0000F6F08954BE250E087E891E00E94926F53
:10E2D0000895892B79F640916A0350916B0341159B
:10E2E000510541F2A0916C03B0916D03E0914F088C
:10E2F000F091500820916303922F90953BB33923FE
:10E300003BBB8AB3822B8ABBBF01640F751F70931E
:10E310006F0360936E03A417B50758F4BF016A0F2B
:10E320007B1F8BE19927AC0187E891E00E94AE6EDC
:10E33000A1CF8BE2F7CF982F20916F0A3091700A0E
:10E340008FEF2F3F3807B9F0AB9A4091710A4F70A9
:10E3500040614093710A90936C0A80914F089091AC
:10E360005008820F931F4DE050E0BC0187E891E018
:10E370000E94926F089587E891E00E940F6F0895C0
:10E380000895AB988091710A805F8093710A87E845
:10E3900091E00E940F6F089580915A03E82FFF27A4
:10E3A000E256FC4F30894091E90640FF35C08F3F6F
:10E3B00009F44FC065B36F70832F992782959295AA
:10E3C000907F9827807F98278068682B65BB209175
:10E3D00065002B7F209365008091650084608093A9
:10E3E000650041FF36C0315045B34F70832F9927E8
:10E3F00082959295907F9827807F98278068482BF8
:10E4000045BBF0916500FB7FF0936500309165009E
:10E410003460309365001DC08F3FD9F0A5B3AF7055
:10E42000932F9295907FA92BA5BB709165007B7F60
:10E43000709365005091650054605093650041FFF2
:10E4400008C03150B5B3BF703295307FB32BB5BB28
:10E45000D8CF87E891E00E940F6F08952091620362
:10E460009091610392959F709F5F8091610389589D
:10E4700080936103222309F45CC0291708F459C072
:10E48000309161033F5F3093610320913D0320622F
:10E4900020933D0350917A0AE0915A035E1729F0C8
:10E4A00060917B0A6F5F60937B0A709153037330B6
:10E4B00009F4CDC090915303913009F4D0C0B091CC
:10E4C0005303BB2389F580915A03E82FFF27E256B7
:10E4D000FC4F30894091E90640FD8EC08F3F21F10D
:10E4E00075B37F70932F9295907F792B75BB609158
:10E4F00065006B7F60936500809165008460809308
:10E50000650041FF11C03150A5B3AF703295307F27
:10E51000A32BA5BBB0916500BB7FB0936500309184
:10E52000650034603093650087E891E00E940F6FCA
:10E53000089540913D034F7D40933D0380915A03E0
:10E54000E82FFF27E256FC4F30894091E90640FF53
:10E5500028C08F3F09F49ECF75B37F70932F92959B
:10E56000907F792B75BB609165006B7F6093650030
:10E570005091650054605093650041FF8BCF31503E
:10E58000A5B3AF703295307FA32BA5BB309165004A
:10E590003B7F3093650080916500846080936500C7
:10E5A00079CF8F3F09F476CF25B32F70832F99272A
:10E5B00082959295907F9827807F98278068282B56
:10E5C00025BBF0916500FB7FF0936500B09165007D
:10E5D000B460B093650041FF5DCF315045B34F70DB
:10E5E000832F992782959295907F9827807F9827EF
:10E5F0008068482B45BBCACF8F3F09F495CF55B3F0
:10E600005F70832F992782959295907F9827807FBE
:10E6100098278068582B55BB209165002B7F20934D
:10E620006500F0916500F460F093650041FF7CCFD8
:10E63000315045B34F70832F992782959295907FE3
:10E640009827807F98278068482B45BB63CF87E851
:10E6500091E00E940F6F84E0809353030895A0918E
:10E660005F03B091600341E050E0BD0187E891E0B5
:10E670000E94926F82E080935303089508950F9350
:10E680001F93CF93DF9380915A03E82FFF27E25621
:10E69000FC4F30894091E90640FF65C08F3FC9F0CB
:10E6A00025B32F70832F992782959295907F982775
:10E6B000807F98278068282B25BB009165000B7F01
:10E6C000009365008091650084608093650041FD42
:10E6D000FFC0C0917A0AB0915A03CB1729F0F0918C
:10E6E0007C0AFF5FF0937C0AC0915A03E0913D03DE
:10E6F000E4FF57C080913D038F7E80933D0380915E
:10E70000EA0680935A03A0914F08B0915008609197
:10E710005F0370916003A61BB70B40E1BD0184E766
:10E7200098E00E940C7B20913C0327FD48C000919B
:10E73000710A02FF3FC080914F08909150084091AC
:10E740006D0A50916E0A840F951FC295C07FC45FF9
:10E750006C2F7727AB01BC0187E891E00E94926F94
:10E76000109253033AC18F3F09F4B3CF75B37F7052
:10E77000932F9295907F792B75BB609165006B7F8D
:10E78000609365005091650054605093650041FFAF
:10E79000A0CF315045B34F703295307F432B45BBEE
:10E7A000A5C000915A03002309F4A9CF80915A0310
:10E7B0008150A7CF87E891E00E940F6FD1CF809161
:10E7C000470390914803A0914903B0914A03AD01DA
:10E7D00066277727411551056105710509F0A7CF17
:10E7E00040915B0350915C038091470390914803F3
:10E7F000A0914903B0914A039C010C2F1127D80125
:10E80000A256BC4F60915A03E62FFF27E256FC4FF9
:10E81000ED0198897089971709F4ABC04217530727
:10E8200008F47DC034E0309353032091620390914B
:10E83000610301C096953A95EAF79F5F5091610395
:10E84000595850936103222309F05BC020913D0386
:10E850002F7D20933D0380915A03C82FDD27C25698
:10E86000DC4F38894091E90640FF8CC08F3F21F191
:10E87000A5B3AF70632F6295607FA62BA5BB909167
:10E8800065009B7F90936500709165007460709344
:10E89000650041FF11C0315045B34F703295307F54
:10E8A000432B45BBB0916500BB7FB09365003091B1
:10E8B000650034603093650087E891E00E940F6F37
:10E8C000C091710AC2FD3BC013E01093530385C091
:10E8D000315015B31F70832F992782959295907FA1
:10E8E0009827807F98278068182B15BBA09165001A
:10E8F000AB7FA09365003091650034603093650074
:10E90000E8CE291708F4A2CFF0916103FF5FF093DE
:10E910006103B0913D03B062B0933D03CDCF241BA2
:10E92000350BE0914F08F0915008E20FF31F40E0E3
:10E9300050E0BF0187E891E00E94926FC1CF209123
:10E940004F0830915008A0916D0AB0916E0A2A0FBD
:10E950003B1F02951295107F1027007F1027802FF4
:10E96000845F9927AC01B90187E891E00E94AE6EFF
:10E97000ABCFCA018C599F4F8217930780F224E6D0
:10E9800030E0CFCF8F3F09F497CF55B35F70832F1F
:10E99000992782959295907F9827807F9827806805
:10E9A000582B55BBE0916500EB7FE09365008091AB
:10E9B000650084608093650041FF7ECF3150F5B3E0
:10E9C000FF70832F992782959295907F9827807F5B
:10E9D00098278068F82BF5BB65CFDF91CF911F9109
:10E9E0000F9108951F93CF93DF93A091D808B09112
:10E9F000D908A431B10508F47DC080910507682FBE
:10EA0000607F8F70482F55279A014230510579F168
:10EA1000433051050CF073C04115510509F079C020
:10EA2000862F9927807790709595879595958795EE
:10EA3000959587959595879567FD88C0C82FDD27A3
:10EA4000C256DC4F38814BB3432B4BBB8AB3832B6D
:10EA50008ABB6091DC087091DD089091DB089923F6
:10EA600039F1192F1150EB01CA0FDB1F35C0E5E654
:10EA7000F0E0B5B3BF70B62BB5BB21E030E002C00B
:10EA8000220F331F4A95E2F7A22FA09570817A23B7
:10EA900070836081622B6083A091D808B091D908FF
:10EAA0006091DC087091DD089091DB089923C9F62C
:10EAB0008091DA08F82FF295F695F770F160182F2B
:10EAC0001F7355274427AF9F9001BF9F300D411DF5
:10EAD0001124EB01C20FD31F45E050E0BE0187E8CF
:10EAE00091E00E94926FD093DD08C093DC081093F0
:10EAF000DB084FC087E891E00E940F6F4AC04630A4
:10EB0000510521F04730510509F0CACFE2E3F0E0AA
:10EB1000B0CF4130510509F0C3CF67FD25C0862F26
:10EB20009927807790709595879595958795959578
:10EB300087959595879502C0220F331F8A95E2F736
:10EB4000522F509588B3852388BBAACFE82FFF2783
:10EB5000E256FC4F2081922F90951BB319231BBBCB
:10EB60008AB3822B8ABB75CF862F992780779070C6
:10EB7000959587959595879595958795959587957D
:10EB800002C0220F331F8A95E2F788B3822B88BB1D
:10EB900087CFDF91CF911F910895EF92FF920F934E
:10EBA0001F938091D8089091D908809708F467C086
:10EBB00000910507202F207F90E829270F70402F14
:10EBC0005527BA014230510511F1433051050CF07F
:10EBD0005BC04115510509F060C0822F99278077ED
:10EBE0009070959587959595879595958795959529
:10EBF000879527FD6EC0E82FFF27E256FC4F108156
:10EC00003BB3312B3BBB8AB3812B8ABB15C0E5E6F6
:10EC1000F0E0A5B3AF70A22BA5BB21E030E002C0AD
:10EC2000220F331F4A95E2F7722F70956081672398
:10EC300060835081522B50830091DC081091DD08D5
:10EC400080914F0890915008801B910B049641E0F1
:10EC5000BC018FED98E00E940C7BE090D808F0900A
:10EC6000D908E00EF11E44E050E0B70187E891E0DA
:10EC70000E94926FF092DD08E092DC084DC087E8B8
:10EC800091E00E940F6F48C04630510519F047309F
:10EC9000510591F6E2E3F0E0BCCF4130510561F659
:10ECA00027FD25C0822F99278077907095958795AD
:10ECB00095958795959587959595879502C0660F4B
:10ECC000771F8A95E2F7462F409588B3842388BB47
:10ECD000B3CFE82FFF27E256FC4F2081F22EF094AD
:10ECE000EBB2EF20EBBA8AB3822B8ABBA5CF822F7F
:10ECF00099278077907095958795959587959595A7
:10ED000087959595879502C0660F771F8A95E2F7DC
:10ED100088B3862B88BB90CF1F910F91FF90EF9007
:10ED2000089520E226BF87B7806287BF87E891E019
:10ED30000E940F6F089520E220937C0080917D0057
:10ED4000806280937D0087E891E00E940F6F0895B4
:10ED5000809107028730B0F40E9477C5BC018EE332
:10ED60006138780740F09B01317060914F087091D5
:10ED70005008620F731F46E050E087E891E00E9460
:10ED8000926F089587E891E00E940F6F08950895AB
:10ED900080914F089091500820916503309166034F
:10EDA000821B930B499708F08BC030911107632F9A
:10EDB000607F3F70432F55279A0142305105A9F0DB
:10EDC0004330510544F44115510529F141305105B5
:10EDD00009F076C03AC04630510521F04730510560
:10EDE00009F06EC0E2E3F0E002C0E5E6F0E025B332
:10EDF0002F70262B25BB21E030E002C0220F331FED
:10EE00004A95E2F7322F3095808183238083B08149
:10EE1000B22BB08355C0862F992780779070959537
:10EE2000879595958795959587959595879567FD90
:10EE300025C0E82FFF27E256FC4F60817BB3762B7D
:10EE40007BBB8AB3862B8ABB3BC067FD25C0862F60
:10EE50009927807790709595879595958795959545
:10EE600087959595879502C0220F331F8A95E2F703
:10EE7000A22FA09588B38A2388BB22C0E82FFF2742
:10EE8000E256FC4F4081942F90955BB359235BBBB6
:10EE90008AB3842B8ABB14C0862F99278077907001
:10EEA000959587959595879595958795959587954A
:10EEB00002C0220F331F8A95E2F788B3822B88BBEA
:10EEC00087E891E00E940F6F089587E891E00E9423
:10EED0000F6F8091A8089091A908A091AA08B091FD
:10EEE000AB080196A11DB11D8093A8089093A908B5
:10EEF000A093AA08B093AB0808950F931F93CF93E4
:10EF0000DF930091070240914F08509150086CB573
:10EF10007DB56417750748F4A0915108B091520867
:10EF20001196B0935208A09351089B012F5F3F4F59
:10EF3000002349F0C0918B01D0918C01FE01E21BAE
:10EF4000F30B0AF471C0232F3327909153089217C3
:10EF5000D9F17093500860934F0820935308809123
:10EF60003A02882331F0815080933A02882309F4D1
:10EF700071C08091BB098131E8F0109170081111C6
:10EF80001150112319F48F3F09F467C080913E029C
:10EF90000E94372A882361F080913E028F5F88307B
:10EFA00008F43FC010923E0280913E020E94322A35
:10EFB0001093700880919808909199080196909309
:10EFC0009908809398089FCF892F8F5F002331F194
:10EFD000282F3327922F88278860AE01481B590BB2
:10EFE0001AF0D22FCC27C5602CB53DB5A901261744
:10EFF000370748F4E0915108F09152083196F093A8
:10F000005208E09351082C5F3F4FDE01A21BB30B67
:10F0100024503040BB230CF47ACF23C0282F332751
:10F02000E0CF80933E02C0CF7093500860934F08AA
:10F0300090918D01892F8F70880F282F33272452AC
:10F04000374EF90145915491892F82958F70FA01BD
:10F05000099557CF0E948D958CCF1BE00E9444AE3E
:10F06000A7CF3093500820934F08D0937900C093D6
:10F07000780001E000937C00DF91CF911F910F9108
:10F0800008951F920F920FB60F9211240F931F93A2
:10F090002F933F934F935F936F937F938F939F93A0
:10F0A000AF93BF93CF93DF93EF93FF93009107024A
:10F0B00040914F08509150086CB57DB564177507A5
:10F0C00048F4A0915108B09152081196B09352089B
:10F0D000A09351089B012F5F3F4F002349F0C0913F
:10F0E0008B01D0918C01FE01E21BF30B0AF471C07D
:10F0F000232F3327909153089217D9F1709350081A
:10F1000060934F082093530880913A02882331F08E
:10F11000815080933A02882309F471C08091BB0921
:10F120008131E8F01091700811111150112319F478
:10F130008F3F09F467C080913E020E94372A8823DE
:10F1400061F080913E028F5F883008F43FC01092DA
:10F150003E0280913E020E94322A109370088091F4
:10F16000980890919908019690939908809398082F
:10F170009FCF892F8F5F002331F1282F3327F22F64
:10F18000EE27E860AE014E1B5F0B1AF0D22FCC27A2
:10F19000C5602CB53DB5A9012617370748F4809105
:10F1A000510890915208019690935208809351080B
:10F1B0002C5F3F4FDE01A21BB30B24503040BB231A
:10F1C0000CF47ACF23C0282F3327E0CF80933E0260
:10F1D000C0CF7093500860934F0890918D01892F94
:10F1E0008F70880F282F33272452374EF90145910D
:10F1F0005491892F82958F70FA01099557CF0E94FB
:10F200008D958CCF1BE00E9444AEA7CF3093500861
:10F2100020934F08D0937900C093780001E00093C9
:10F220007C00FF91EF91DF91CF91BF91AF919F91C2
:10F230008F917F916F915F914F913F912F911F918E
:10F240000F910F900FBE0F901F9018959C01462FA5
:10F2500080914F08909150086CB57DB5709350081F
:10F2600060934F086817790748F4A0915108B0914E
:10F2700052081196B0935208A0935108620F731F61
:10F28000242F3327A90187E891E00E94AE6E0895EC
:10F290009C01462F80914F08909150086CB57DB528
:10F2A0007093500860934F086817790748F4A0914D
:10F2B0005108B09152081196B0935208A09351088A
:10F2C000620F731F242F3327A90187E891E00E9462
:10F2D000926F08959C01462F80914F08909150089D
:10F2E0006CB57DB57093500860934F086817790727
:10F2F00048F4A0915108B09152081196B093520869
:10F30000A0935108620F731F20917A01222341F0CC
:10F31000E42FFF27AF0187E891E00E94AE6E0895C9
:10F3200031E030937A01842F9927AC0187E891E08E
:10F330000E94926F0895089520B5216820BD109213
:10F3400089001092880014BC1DBC1CBC80B58F774E
:10F3500080BD08950F931F93CF93DF9303E00EBDFD
:10F3600080917D00816080937D0010927A0187E812
:10F3700091E00E94A76E0E94037B10928900109278
:10F3800088001DBC1CBC1092500810924F080091C0
:10F39000070260914F08709150082CB53DB530932D
:10F3A000500820934F082617370748F4A0915108BA
:10F3B000B09152081196B0935208A09351082F5F54
:10F3C0003F4F002349F0C0918B01D0918C01FE0189
:10F3D000E21BF30B0AF471C0232F332790915308DB
:10F3E0009217B9F12093530880913A02882331F0A3
:10F3F000815080933A02882309F471C08091BB093F
:10F400008131E8F01091700811111150112319F495
:10F410008F3F09F467C080913E020E94372A8823FB
:10F4200061F080913E028F5F883008F443C01092F3
:10F430003E0280913E020E94322A10937008809111
:10F44000980890919908019690939908809398084C
:10F45000A0CF892F8F5F002351F1282F3327722FE0
:10F4600066276860AE01461B570B1AF0D22FCC27D7
:10F47000C560E0914F08F09150082CB53DB5309330
:10F48000500820934F082E173F0748F480915108E9
:10F4900090915208019690935208809351082C5FE6
:10F4A0003F4FDE01A21BB30B0AF473CF1FC0282FFE
:10F4B0003327DCCF80933E02BCCF90918D01192F72
:10F4C0001F70110F212F33272452374EF901459118
:10F4D0005491892F82958F70FA01099558CF0E9417
:10F4E0008D958CCF1BE00E9444AEA7CFD0937900BE
:10F4F000C093780051E050937C00DF91CF911F9131
:10F500000F91089521B180917B01822790E082FFC5
:10F510000FC080917C01853018F08D3308F491E0A4
:10F5200010927C0180917D018E7F80937D0114C0BB
:10F5300022FD10C080917C018F3F71F08F5F80931E
:10F540007C01883C49F480917D0180FD05C092E0FA
:10F550008160EBCF90937C0120937B01892F9927C9
:10F56000089591B180917B01892720E082FF15C029
:10F5700080917C01853018F08D3308F421E01092E1
:10F580007C0180917D018E7F80937D0190937B0132
:10F590002130D9F0223021F1089592FD10C08091E0
:10F5A0007C018F3F99F38F5F80937C01883C71F7DA
:10F5B00080917D0180FDEACF22E08160E5CF20933C
:10F5C0007C0190937B01213029F7809173088F5F34
:10F5D000833018F01092730808958093730808958B
:10F5E00080E00E94D4440E947C5B0895089526ED3B
:10F5F00034E03093CD082093CC081092CF088FEFE1
:10F600008093D108089587E3EBECF8E010823197FE
:10F61000815087FFFBCF0895CF93DF93EC01242F18
:10F620008091AC089091AD08A091AE08B091AF0860
:10F630000196A11DB11D8093AC089093AD08A093D5
:10F64000AE08B093AF0833276217730738F0F9019B
:10F65000E20FF31FEC0FFD1F329705C0FB01E60F11
:10F66000F71FEC0FFD1FA081B1811196A083B1831C
:10F67000DF91CF910895882309F444C0813009F4C3
:10F680004CC08250982F969596959695E92FFF2716
:10F69000EE0FFF1FE152F74F0190F081E02D8770D0
:10F6A000282F332723303105D9F1243031057CF060
:10F6B0002530310511F125303105CCF026303105EA
:10F6C00041F12730310509F185E690E008952130B8
:10F6D000310549F1223031052CF0892F0E946D63EC
:10F6E00099270895232B81F780E290E008958F2FCA
:10F6F00099270E946463992708958F2F99270E9464
:10F700006D63EECF8DE090E008958E2F0E946D63C3
:10F71000E7CF8E2F0E946463EECF8AE090E00895D9
:10F720008DE390E0089585E490E00895089588239E
:10F7300009F444C0813009F44CC08250982F96954A
:10F7400096959695E92FFF27EE0FFF1FEC56F74F82
:10F750000190F081E02D8770282F33272330310569
:10F76000D9F1243031057CF02530310511F12530F7
:10F770003105CCF02630310541F12730310509F152
:10F7800085E690E008952130310549F122303105B8
:10F790002CF0892F0E946D6399270895232B81F700
:10F7A00080E290E008958F2F99270E946463992743
:10F7B00008958F2F99270E946D63EECF8DE090E022
:10F7C00008958E2F0E946D63E7CF8E2F0E94646391
:10F7D000EECF8AE090E008958DE390E0089582E412
:10F7E00090E008950895882309F444C0813009F415
:10F7F0004CC08250982F969596959695E92FFF27A5
:10F80000EE0FFF1FEC58F74F0190F081E02D87704D
:10F81000282F332723303105D9F1243031057CF0EE
:10F820002530310511F125303105CCF02630310578
:10F8300041F12730310509F185E690E00895213046
:10F84000310549F1223031052CF0892F0E946D637A
:10F8500099270895232B81F780E290E008958F2F58
:10F8600099270E946463992708958F2F99270E94F2
:10F870006D63EECF8DE090E008958E2F0E946D6352
:10F88000E7CF8E2F0E946463EECF8AE090E0089568
:10F890008DE390E0089589E490E008950895CF9372
:10F8A000DF93882309F450C0813009F450C0282F19
:10F8B0002250422F46954695469580919102992770
:10F8C000DC01AA0FBB1FAA0FBB1FAA0FBB1FA80FEB
:10F8D000B91FAE56BD4FED01EC81FD81E40FF11D66
:10F8E00080819927277033272330310599F12430FF
:10F8F00031057CF02530310519F125303105CCF08A
:10F9000026303105B9F02730310551F085E690E019
:10F9100023C02130310589F0223031052CF0842FAD
:10F920000E946D63992718C0232B81F780E290E035
:10F9300013C080E00E946463F5CFFD018681F2CFA1
:10F9400080E00E946D63EECF8DE090E005C08AE01C
:10F9500090E002C08DE390E0DF91CF910895909107
:10F96000CF089923A1F18091D0088F5F8917B0F05B
:10F970001092D0088091D10880FD2AC082FD40C03D
:10F9800085FD36C086FD2CC087FD44C081FF1FC0A9
:10F9900060E186E299E90E94A12A08958093D00847
:10F9A0009F3FA9F48091D10880FD3FC082FD55C0E2
:10F9B00085FD4BC086FD41C087FD59C081FF05C054
:10F9C00060E186E299E90E94A12A1092CF08089589
:10F9D00068E586E793E60E94A12A8091D108CECF00
:10F9E0006AE08BE39BE70E94A12A8091D108CCCFEB
:10F9F00062EE87E99BE70E94A12A8091D108C2CFDD
:10FA000047E851E06CE48FE49CE70E946F318091FD
:10FA1000D108B6CF29E444E758E062E88FE49CE7D8
:10FA20000E943F318091D108B1CF68E586E793E627
:10FA30000E94A12A8091D108B9CF6AE08BE39BE7AD
:10FA40000E94A12A8091D108B7CF62EE87E99BE797
:10FA50000E94A12A8091D108ADCF47E851E06CE423
:10FA60008FE49CE70E946F318091D108A1CF29E4F7
:10FA700044E758E062E88FE49CE70E943F318091C0
:10FA8000D1089CCF40E050E0009749F02FEF3FEFC6
:10FA9000420F531F21503040D9F70197F5CFCA01CB
:10FAA0000895CF93DF93882309F453C0813009F47C
:10FAB00053C0282F2250422F469546954695809157
:10FAC00091029927DC01AA0FBB1FAA0FBB1FAA0F27
:10FAD000BB1FA80FB91FAE56BD4FE42FFF27EE0F77
:10FAE000FF1FED018C819D81E80FF91F80819181BD
:10FAF000277033272330310591F1243031057CF014
:10FB00002530310509F125303105CCF0263031059D
:10FB1000C1F02730310551F085E690E025C0213055
:10FB2000310501F1223031052CF0842F0E946D63E4
:10FB300099271AC0232B81F780E290E015C0892F06
:10FB400099270E946463F4CF892F99270E946D63DF
:10FB5000EFCF8DE090E008C08AE090E005C08DE333
:10FB600090E002C084E590E0DF91CF910895CF93BB
:10FB7000C5E080E20E943968C150D9F786E09EE373
:10FB80000E949B68CF91089580E20E9439688FE0BF
:10FB90009EE30E949B688AE19EE30E949B68089511
:10FBA00081E29EE30E949B68089585E39EE30E94A4
:10FBB0009B680895CF93DF93C0914D03D0914E037E
:10FBC00087E2C031D80738F442E060914508CE01A1
:10FBD0000E94576511C08EE30E943968CD2FDD2742
:10FBE000C695C6958C2F40E06091450899270E94E4
:10FBF00057658BE60E943968DF91CF91089580E2C6
:10FC00000E94396808958AE39EE30E949B680895E4
:10FC10008AE39EE30E949B688AE39EE30E949B68BE
:10FC200008958DE39EE30E949B68089583E49EE31C
:10FC30000E949B6808951F93CF939EE8899FC001FF
:10FC40001124892F990F990BC82F883258F0182F3B
:10FC50001852143610F041E00BC080E20E9439685F
:10FC600040E006C08DE20E94396818E21C1BF8CF04
:10FC700060914508812F99270E945765CF911F9168
:10FC800008951F93CF93909142038EE8989FC001EF
:10FC90001124892F990F990BC82F883258F0182FEB
:10FCA0001852143610F041E00BC080E20E9439680F
:10FCB00040E006C08DE20E94396818E21C1BF8CFB4
:10FCC00060914508812F99270E945765CF911F9118
:10FCD0000895CF9390913E038EE1989F9001112457
:10FCE000832F9927582F843618F053E6C9E010C0A7
:10FCF000D901B0709D01220F331F220F331F220F35
:10FD0000331F2A0F3B1F2A0F3B1F832F9927C82F12
:10FD100040E060914508852F99270E9457658EE243
:10FD20000E943968609145088C2F805D0E941F6495
:10FD300086E50E943968CF91089585E49EE30E948C
:10FD40009B68089580913F039091400341E060914A
:10FD5000450896958795969587950E9457650895CD
:10FD600094E1899F802D11240E94326808956CE1EE
:10FD700080E20E941F64089587E49EE30E949B68CE
:10FD80000895CF932091D8093091D90921153105D3
:10FD900009F439C03695279593E377276627299F7D
:10FDA000A001399F500D611D1124BB27A72F962F4D
:10FDB000852F9C01832F9927582F843608F5B90188
:10FDC00070709B01220F331F220F331F220F331F2E
:10FDD000260F371F260F371F832F9927C82F40E084
:10FDE00060914508852F99270E9457658EE20E94F1
:10FDF0003968609145088C2F805D0E941F6407C0A0
:10FE000053E6C9E0ECCF8CE49EE30E949B68CF915F
:10FE100008958091620681FF05C081E59EE30E94FE
:10FE20009B68089585E59EE30E949B680895089568
:10FE3000CF93DF938091620681FF52C02091D30956
:10FE40003091D4094FEF2F3F340709F46EC096E488
:10FE500077276627299FA001399F500D611D112426
:10FE6000BB27A72F962F852F9C01C901AA27BB2747
:10FE70009295A295B29580EFBA27B823BA27A92701
:10FE8000A823A927BD01462F6A3008F04BC03F7058
:10FE900054E6FF27EE27259FE001359FD00DE11D99
:10FEA0001124CE01DF019295A295B29580EFBA2779
:10FEB000B823BA27A927A823A927FD01CE2F60912F
:10FEC0004508842F805D0E941F648EE20E9439687D
:10FED00040E0609145088C2F99270E9457656CC0BF
:10FEE0003091930635FD19C08091410290914202F4
:10FEF0009695879596958795969587959927880FD6
:10FF0000843608F083E640E06091450899270E9416
:10FF1000576586E50E9439684FC080914D029091E7
:10FF20004E02E6CF49E0C3E6CACF2091D80930910E
:10FF3000D9092115310509F43BC03695279543E3CE
:10FF4000FF27EE27249FE001349FD00DE11D1124EF
:10FF50009E01AF01BB27A52F942F832F9C01892FD2
:10FF60009927582F843698F053E6C9E040E0609115
:10FF70004508852F99270E9457658EE20E943968AF
:10FF8000609145088C2F805D0E941F6415C0E901B7
:10FF9000D070DE01AA0FBB1FAA0FBB1FAA0FBB1F89
:10FFA000AC0FBD1FAC0FBD1F8B2F9927C82FDECF05
:10FFB0008CE49EE30E949B68DF91CF910895CF93DC
:10FFC0008BE59EE30E949B68C0912703C13830F007
:10FFD0008BE20E9439688C2F805805C08DE20E9408
:10FFE000396880E88C1B40E06091450899270E94A1
:10FFF0005765CF910895CF9381E69EE30E949B6859
:020000021000EC
:10000000809171099091720996958795969587953B
:10001000C82F813830F08BE20E9439688C2F8058CD
:1000200005C08DE20E94396880E88C1B40E0609139
:10003000450899270E945765CF91089587E69EE36A
:100040000E949B6808951F93CF93909141038EE87F
:10005000989FC0011124892F990F990BC82F8832BE
:1000600058F0182F1852143610F041E00BC080E2FF
:100070000E94396840E006C08DE20E94396818E2AB
:100080001C1BF8CF60914508812F99270E94576566
:1000900083E40E943968CF911F9108958CE69EE316
:1000A0000E949B6808958091450341E06091450856
:1000B00099270E945765089582E79EE30E949B68F6
:1000C0000895809145038F3FC1F08091450399E1E8
:1000D000899FC001112440E0609145080024880FE9
:1000E000991F001C880F991F001C892F902D0E94BA
:1000F000576585E20E943968089586E79EE30E946D
:100100009B680895089580E20E9439688091640395
:100110000E940F6A089580E20E9439688091CB079F
:1001200041E06091450899270E94576508958AE744
:100130009EE30E949B6808958091CE0741E0609104
:10014000450899270E945765089580E89EE30E941C
:100150009B6808958091CC0781FF02C08BE201C0AB
:100160008DE20E9439688091CD0740E0609145089A
:1001700099270E945765089586E89EE30E949B6830
:10018000089580913B0387FD05C083E99EE30E94AB
:100190009B6808958BE89EE30E949B6808950895EC
:1001A00085E60E94396862E08091D1079091D2077C
:1001B0000E94416E089589E60E94396862E080914C
:1001C000CF079091D0070E94416E089584E60E9467
:1001D000396862E08091D3079091D4070E94416E04
:1001E000089580E70E94396862E08091D507909178
:1001F000D6070E94416E089580E50E94396862E04A
:100200008091D7079091D8070E94416E089589E4A4
:100210000E94396862E08091D9079091DA070E94C4
:10022000416E089584E40E94396862E08091DB07A2
:100230009091DC070E94416E089580E00E940F6A51
:1002400080E00E940F6A0895CF93DF93C091DE078C
:10025000D091DF07D7FD05C08BE20E9439688C2F53
:1002600005C08DE20E9439688C2F819541E0609134
:10027000450899270E945765DF91CF9108958BE932
:100280009EE30E949B6808958091D10680FF0AC07A
:1002900020913C0323FF06C0909141033091C90691
:1002A000931718F40E948469089585EA9EE30E94DA
:1002B0009B684091D10641FFF5CF8DEA9EE30E94F5
:1002C0009B680895089582E70E94396880914B03E6
:1002D0000E940F6A8DE20E9439688091B7070E94E0
:1002E0000F6A80E20E94396808958DE60E9439689D
:1002F00020913F03309140038091D50699278F705C
:100300009070029771F083E02C3F380718F08FEF60
:1003100090E00EC03695279536952795822F992720
:1003200007C0369527953695279536952795F6CFAC
:100330000E940F6A8DE20E9439688091B8070E947E
:100340000F6A80E20E943968089581E60E94396848
:10035000809127030E940F6A8DE20E943968809184
:10036000B9070E940F6A089583E60E943968809158
:10037000BA070E940F6A80E20E943968089580914E
:10038000BF070E940F6A8DE39EE30E949B68089559
:100390008091C0070E940F6A8DE39EE30E949B68D4
:1003A00008958091C1070E940F6A08958091BB074C
:1003B0000E940F6A80E20E9439688091BC070E9407
:1003C0000F6A80E20E9439688091BD070E940F6A1F
:1003D00080E20E9439688091BE070E940F6A0895EA
:1003E000A0916A03B0916B0326E677276627A29F48
:1003F000A001B29F500D611D1124DB01CA01892F9C
:100400009A2FAB2FBB2742E0609145080E945765A9
:10041000089582EB9EE30E949B680895EF92FF92FD
:100420000F931F9340916A0350916B0328E31127A8
:100430000027429F7001529FF00C011D1124609112
:100440004D0370914E039B0144275527C801B70106
:100450000E94E3C5DC01CB018B2F9927AA27BB277C
:1004600041E0609145080E94576585E20E94396825
:100470001F910F91FF90EF90089586EB9EE30E94ED
:100480009B680895CF93C09152038091D606C817F8
:1004900050F08BE20E9439688C2F99272091D60664
:1004A000821B910908C08DE20E9439688091D606AE
:1004B00099278C1B910940E0609145089595879597
:1004C000959587950E945765CF91089580914F0328
:1004D000883C28F08BEB9EE30E949B6808958091F6
:1004E0004F03869540E06091450899270E94576523
:1004F000089508958EEB9EE30E949B680895A09155
:100500005B03B0915C0326E677276627A29FA001D4
:10051000B29F500D611D1124BB27A72F962F852F49
:1005200041E0609145080E9457650895809150030D
:1005300041E06091450899270E9457650895CF933F
:1005400085EC9EE30E949B68809152038695909172
:100550004F03891740F4209152032695C0914F0311
:10056000C21B8BE207C0C0915203C69530914F0366
:10057000C31B8DE20E94396841E0609145088C2FD1
:1005800099270E945765CF910895CF938DEC9EE3F4
:100590000E949B6840915003242F332780915B0376
:1005A00090915C03929582958F7089279F7089271F
:1005B0008217930778F480915B0390915C03929586
:1005C00082958F7089279F708927C0915003C81B1F
:1005D0008BE20FC080915B0390915C0392958295B2
:1005E0008F7089279F70892730915003C82FC31BB4
:1005F0008DE20E94396841E0609145088C2F99276F
:100600000E945765CF9108950F931F9384E60E942F
:1006100039680091BE081091BF088091C008909180
:10062000C108081B190B812F99270E940F6A802F80
:100630000E940F6A1F910F91089585E60E94396804
:100640008091C3080E940F6A8091C2080E940F6ABD
:10065000089587E50E9439688091BA080E940F6A60
:10066000089583E50E943968809164080E940F6AAA
:10067000089589E40E9439689091BE0880919C0891
:10068000981B892F0E940F6A089580913B0381FD7A
:100690002AC020913C0325FD22C030913C0334FD4B
:1006A00028C040913B0342FD28C050913C0352FDBD
:1006B0001EC060913B0363FD24C070913B0374FD39
:1006C00024C090913B0395FD22C0A0913C03A3FD63
:1006D0001AC0B0913B03B0FF1CC080E201C081E4AE
:1006E0000E943968089583E40E94396808958FE470
:1006F000F7CF83E60E943968089587E70E9439683A
:10070000089587E5EDCF8FE6EBCF81E6E9CF84E66C
:10071000E7CF8FE5E5CF80913D0382FD10C02091AA
:100720003C0321FD08C03091640837FD0CC080E215
:100730000E943968089582E40E943968089585E42A
:100740000E94396808954091DA0641FDF0CF83E5B3
:10075000EFCF85ED9EE30E949B688091C0090E94C7
:100760000F6A8091BF090E940F6A089589ED9EE388
:100770000E949B688091C2090E940F6A8091C10902
:100780000E940F6A089581EE9EE30E949B6880910B
:10079000C9090E940F6A089587EE9EE30E949B6834
:1007A0008091C5090E940F6A08958091BD0980FF5C
:1007B00005C08DEE9EE30E949B68089581EF9EE345
:1007C0000E949B68089508958091C0090E940F6A55
:1007D0008091BF090E940F6A80E20E94396880916F
:1007E000C2090E940F6A8091C1090E940F6A80E2CB
:1007F0000E9439688091C9090E940F6A089580910A
:10080000C0090E940F6A8091BF090E940F6A80E2AE
:100810000E9439688091C9090E940F6A8CE20E9487
:100820003968089580E20E9439688091C2090E9467
:100830000F6A8091C1090E940F6A80E20E943968A4
:100840008091C5090E940F6A089580E20E9439686C
:100850008091BD0981FF12C087E50E94396820910F
:10086000BD0922FF12C080E50E9439683091BD09A0
:1008700034FF12C086E40E943968089580E20E9425
:1008800039682091BD0922FDEECF80E20E943968CF
:100890003091BD0934FDEECF80E20E9439680895A1
:1008A0008091CA080E940F6A80E20E943968809194
:1008B000CB080E940F6A80E20E94396880919508F7
:1008C0000E940F6A80E20E943968809194080E9419
:1008D0000F6A80E20E9439688091E7090E940F6ADE
:1008E0008091E6090E940F6A08951F939C01232FAF
:1008F000332726952695322F937024E6772766278F
:10090000829FA001929F500D611D1124DB01CA013D
:100910002AE0B695A795979587952A95D1F7182F30
:1009200040E060914508832F99270E9457658EE229
:100930000E94396840E060914508812F99270E9404
:1009400057651F9108951F93CF93DF9385EF9EE323
:100950000E949B684091D3095091D4098FEF4F3F7B
:10096000580761F1CA01892F992786958695282F06
:10097000537084E6FF27EE27489FE001589FD00D73
:10098000E11D1124CE01DF015AE0B695A795979598
:1009900087955A95D1F7182F40E060914508822F2E
:1009A00099270E9457658EE20E94396840E0609165
:1009B0004508812F99270E9457650BC08FE30E943D
:1009C00039688AE39EE30E949B688AE39EE30E9463
:1009D0009B68DF91CF911F9108951F93CF93DF9371
:1009E0008AEF9EE30E949B680E945DACAC018FEF92
:1009F0004F3F580761F1CA01892F9927869586953F
:100A0000282F537084E6FF27EE27489FE001589F68
:100A1000D00DE11D1124CE01DF017AE0B695A79536
:100A2000979587957A95D1F7182F40E06091450802
:100A3000822F99270E9457658EE20E94396840E014
:100A400060914508812F99270E9457650BC08FE35D
:100A50000E9439688AE39EE30E949B688AE39EE3D2
:100A60000E949B68DF91CF911F9108958FEF9EE3C5
:100A70000E949B6880916E0A0E940F6A80916D0AA5
:100A80000E940F6A82E09FE30E949B688091700A37
:100A90000E940F6A80916F0A0E940F6A089586E093
:100AA0009FE30E949B6880917E0A0E940F6A80915A
:100AB0007D0A0E940F6A80E20E94396880916B0A69
:100AC0000E940F6A80E20E9439688091710A0E9438
:100AD0000F6A089589E09FE30E949B688091800AD5
:100AE0000E940F6A80917F0A0E940F6A8CE09FE348
:100AF0000E949B688091810A0E940F6A80E20E9496
:100B000039688091840A0E940F6A80E20E943968E5
:100B100080917C0A0E940F6A0895CF93DF9381E150
:100B20009FE30E949B6820917D0A30917E0A80910C
:100B30007F0A9091800A8217930728F4E901C81B65
:100B4000D90B8BE204C0EC01C21BD30B8DE20E94D7
:100B5000396841E060914508CE010E945765DF91F8
:100B6000CF91089586E19FE30E949B688091770A68
:100B70000E940F6A8091760A0E940F6A08958AE1A6
:100B80009FE30E949B68089583E60E9439688091E4
:100B9000BF080E940F6A8091BE080E940F6A80E21F
:100BA0000E94396889E60E94396880919D080E94F8
:100BB0000F6A80919C080E940F6A0895CF938091DC
:100BC000930685FF22C080914D0290914E0296952A
:100BD000879596958795969587959927880F84365A
:100BE00008F083E640E06091450899270E94576528
:100BF00080E20E943968C0912703C13858F08BE227
:100C00000E9439688C2F80580AC0809141029091CF
:100C10004202DDCF8DE20E94396880E88C1B40E003
:100C20006091450899270E94576580E20E943968C3
:100C3000CF9108958FE59FE30E949B6808950F93DD
:100C40001F9320910B07022F112702951295107FF9
:100C50001027007F10274091450368E08AE196E065
:100C60000E94CC2990916703989FC001112492950E
:100C700082958F7089279F708927080F191F41E07F
:100C800060914508C801929582958F7089279F7061
:100C900089270E9457651F910F9108958AE69FE367
:100CA0000E949B6841E06091450880913F039091CC
:100CB00040030E94576508954091450368E08AE12A
:100CC00096E00E94CC290E940F6A89E60E9439684A
:100CD000809167030E940F6A08958FE69FE30E9448
:100CE0009B680895809143039091440327E28031EB
:100CF000920710F080E090E042E0609145080E9489
:100D000057650895BF92CF92DF92EF92FF920F93B3
:100D10001F93CF93DF938091E40899278130910549
:100D200041F0823091050CF4BEC0029709F0B8C4BE
:100D300044C0E091E308EF3F09F4E2C0CE2FC29532
:100D4000CF701E2F1F70E091E208EC0FE83208F020
:100D5000A8C0FF27EE0FFF1FE450F74E8591949136
:100D6000009731F4ECEFF8E185919491C0E01C2FED
:100D7000E12FFF27EE0FFF1FE80FF91F85919491D8
:100D8000009709F0B8C0FF24C33008F4B2C0CF2DDB
:100D900024E1C29F800111248091450899270817FA
:100DA000190711F00E948469802F0E943268C29551
:100DB000C07FCF0DC093E30873C41091E3081F5F99
:100DC0001093E308C090E608D090E708E601898117
:100DD00099278836910509F4A0C0893691050CF051
:100DE00091C08336910509F437C18436910509F421
:100DF00094C060E08AE191E00E944464E601898148
:100E00000E94396887E79FE30E949B688F810E9458
:100E10000F6A8DE79FE30E949B681F81EB81FC8135
:100E2000E10FF11D80810E940F6A0E94156984E123
:100E30000E9432681F814A81842F8F5F133008F02F
:100E400086C120E030E0B22EE601EB80FC80E20EAD
:100E5000F11C83E0489FC00111248E5F682F84E15C
:100E60000E948529C82FF60107810B1910E010C0D8
:100E7000CC2359F01F5F113009F453C1101709F446
:100E800055C180E20E943968C150C23008F408C4DC
:100E9000C23070F3F70181917F010E940F6AC25046
:100EA000E7CFE0E056CF892B09F0FAC380915108D3
:100EB00090915208099708F0C7C080E00E943268FC
:100EC000C5E080E20E943968C150D9F786E09EE310
:100ED0000E949B6884E10E94326880E20E94396827
:100EE0008FE09EE30E949B688AE19EE30E949B68DC
:100EF000D7C3CF5F4DCFFC010995F12EF39457CFA7
:100F0000E0E01CCF8C36910541F08D3691050CF058
:100F100033C18A36910509F06CCF3091E308343043
:100F200020F01092E3083091E308F6012681223088
:100F300008F005C180E090E0C82FF601278123303A
:100F400008F0F6C080E090E0182F832F99278130B9
:100F5000910509F44BC1823091050CF412C1823025
:100F6000910509F48FC1039709F09AC3F601B28481
:100F7000B0FED4C18BE30E944A698091B6070E94FB
:100F80006D630E94396882E50E943968E091B60776
:100F9000EE2309F054C28FEF0E940F6A80E20E9494
:100FA00039688091B4070E946D630E9439688BE4B0
:100FB0000E943968E091B407EE2309F4C6C220917B
:100FC0003F03309140038091D50699278F70907030
:100FD000029709F43AC3F3E02C3F3F0708F4B7C285
:100FE0004FEF50E0FF27EE5FF94FE090B307CE2DB3
:100FF000DD27CE5FD94F608188810E9421280E9421
:101000000F6A80E20E94396880913A030E946D6302
:101010000E94396884E50E94396890913A039923C7
:1010200009F47BC0B0913903EB2FFF27EE5DF94F38
:10103000F090410340854F1508F456C080E00E94AF
:101040000F6A0E9415692CC301E00093E4080E9416
:101050003A660E94F66B24C380E00E943268F60173
:101060008681992782959295907F9827807F9827EF
:10107000B780B82AEB2CFF24C7018E0D9F1D8E541C
:10108000954EC0E002C00297CF5FFC01059114911C
:1010900001151105C1F384E79FE30E949B688B2D26
:1010A0008C1B0E940F6A8FE20E9439688C2F0E946D
:1010B0006D630E9439688DE30E943968E601EB8117
:1010C000FC81EE0DFF1D80810E940F6A80E20E946C
:1010D0003968B090D608B7FC41C266E4C8010E94E6
:1010E000D5680E941569DCC2C92FDD27CE5DD94FB6
:1010F000909141032885921780F490914103941BAD
:10110000241B33278FEF989FC0011124B9010E943F
:101110000EC6CB010E940F6A94CF8FEF0E940F6A18
:1011200090CF002309F0AACE8CE3ACCE8EE3AACEFA
:10113000822F99270897C4F086E090E005CF622FB0
:1011400077276A307105A4F089E090E0F5CEA12FF1
:10115000BB2799270597A817B9070CF443C0465039
:10116000242F33274A5F6FCE2250822F9927ECCE4F
:101170002150822F9927E0CE8E36910509F039CE85
:10118000CCCE892B09F08CC260E08AE191E00E940C
:101190004464E60189810E943968E12EFF2426EF2C
:1011A00035E0E20EF31EC1E10091B607011B10E02D
:1011B00010C0CC2359F01F5F113009F4FCC0101788
:1011C00009F400C180E20E943968C150C23008F4BD
:1011D00067C2C23070F3F70181917F010E940F6AEC
:1011E000C250E7CF1250212F33272DCE84E10E9429
:1011F0003268EC2FFF27EE5FF94F80810E940F6A63
:101200008AE30E9439688CE0C89FC0011124912FA5
:10121000980FF60156815C1709F40EC16FEFE62EA8
:101220007091B4077C1709F404C140E2B42EE601C2
:10123000B981B43609F4C8C0E6010B811C81090FDD
:10124000111DC1E1FF240FC0CC2351F0F39431E014
:10125000F31691F0FE14A1F08B2D0E943968C15055
:10126000C23008F41DC2C23078F3F80181918F01B9
:101270000E940F6AC250E8CFEE2061F78CE3EDCFF9
:101280008EE3EBCFCF5F88E20E943268EC2FFF271E
:10129000EE5FF94F80810E940F6A8AE30E943968ED
:1012A0008CE0C89FC0011124912F980FF601068190
:1012B0000C1709F4D4C00FEFE02E1091B4071C17DF
:1012C00009F405C1C0E2BC2EE6016981643609F467
:1012D000C9C0E6010B811C81090F111DC1E1FF246A
:1012E00010C0CC2359F0F39471E0F71699F0FE1476
:1012F00009F45BC08B2D0E943968C150C23008F4DC
:10130000CFC1C23070F3F80181918F010E940F6A42
:10131000C250E7CFEE2059F78CE3EDCFCE5F8CE3E0
:101320000E943268EC2FFF27EE5FF94F80810E9408
:101330000F6A8AE30E9439688CE0C89FC0011124BB
:10134000912F980FF60136813C1709F4FBC06FEF1F
:10135000E62EF091B407FC1709F4F1C040E2B42E78
:10136000E6010981043609F4B5C0E6010B811C8150
:10137000090F111DC1E1FF240FC0CC2351F0F394DC
:1013800051E0F516A1F0FE14D9F08B2D0E943968BA
:10139000C150C23008F484C1C23078F3F8018191A1
:1013A0008F010E940F6AC250E8CF8EE3A4CFEE20D7
:1013B00051F78CE3EBCF002309F001CF8CE303CF8F
:1013C0008EE3E4CF8EE3FFCEA92FBB2736EDC32EED
:1013D00034E0D32ECA0EDB1E8D010A0F1B1F0A54E8
:1013E0001C4FC1E1FF240FC0CC2351F0F394F1E076
:1013F000FF16C9F0FE14D9F08B2D0E943968C15038
:10140000C23008F44DC1C23078F3F80141915191D6
:101410008F01852F9927F60191916F01891B0E94F9
:101420000F6AC250E1CFEE2029F78CE3E6CF8EE3BE
:10143000E4CF5DE2B52EFBCEE780E11AF1CEFF27C7
:10144000EA50FA4FC090B507AC2DBB27AA50BA4F4F
:1014500040914B0360818C910E9421289DCDE780B3
:10146000E11A2BCF892F9927B6EDCB2EB4E0DB2ED6
:10147000C80ED91E8C01080F191F0A541C4FC1E158
:10148000FF240FC0CC2351F0F39451E0F516C9F0BE
:10149000FE14D9F08B2D0E943968C150C23008F477
:1014A000FFC0C23078F3F801419151918F01852F2F
:1014B0009927F60121916F01821B0E940F6AC25089
:1014C000E1CFEE2029F78CE3E6CF8EE3E4CF1DE2F7
:1014D000B12EFACE692F772736EDC32E34E0D32E06
:1014E000C60ED71E8B01060F171F0A541C4FC1E1F1
:1014F000FF240FC0CC2351F0F39441E0F416C9F05F
:10150000FE14D9F08B2D0E943968C150C23008F406
:10151000C7C0C23078F3F801819191918F01892F72
:101520009927F60121916F01821B0E940F6AC25018
:10153000E1CFEE2029F78CE3E6CF8EE3E4CF5DE246
:10154000B52E0ECFE780E11A04CF8FEF58CD369538
:10155000279536952795422F552744CD62E3C8013C
:101560000E94D5688BE30E944A698091B6070E9469
:101570006D630E94396882E50E943968E091B60780
:10158000EE2309F06BC08FEF0E940F6A80E20E9489
:1015900039688091B4070E946D630E9439688BE4BA
:1015A0000E943968E091B407EE2309F467C02091E6
:1015B0003F03309140038091D50699278F7090703A
:1015C000029709F464C0F3E02C3F3F0708F458C0C9
:1015D0004FEF50E0FF27EE5FF94FE090B307CE2DBD
:1015E000DD27CE5FD94F608188810E9421280E942B
:1015F0000F6A80E20E94396880913A030E946D630D
:101600000E94396884E50E94396890913A039923D1
:1016100009F483CD30913903E32FFF27EE5DF94FB5
:10162000F090410330853F1508F008CDC92FDD2724
:10163000CE5DD94F409141032885421708F06DCD0A
:1016400090914103931B231B5CCD369527953695CE
:10165000279536952795422F5527C4CCFF27EA506A
:10166000FA4FC090B507AC2DBB27AA50BA4F409196
:101670004B0360818C910E94212886CF8FEFB7CFDA
:101680003695279536952795422F5527A3CF369522
:1016900027953695279536952795422F55279ACF2A
:1016A000DF91CF911F910F91FF90EF90DF90CF903E
:1016B000BF9008959FEF9093E3088093E4087093A0
:1016C000E7086093E6081092E5080895582F4091C6
:1016D000E208242F332787E290E0851B91098217C7
:1016E000930718F0242F250F01C020E02093E20873
:1016F00008959091E208981718F0981B9093E208CB
:1017000008950895809191029927FC01EE0FFF1F23
:10171000EE0FFF1FEE0FFF1FE80FF91FEE56FD4FF4
:10172000868187FD03C080689927089588E790E047
:101730000895089580E590E008958AE090E0089586
:101740001F920F920FB60F9211242F923F924F9239
:101750005F926F927F928F929F92AF92BF92CF9241
:10176000DF92EF92FF920F931F932F933F934F932C
:101770005F936F937F938F939F93AF93BF93EF93F9
:10178000FF93CF93DF93CDB7DEB72D97DEBFCDBFED
:10179000D090DA068091DC068758E82EFF24EE20F0
:1017A000E9F410916408112309F4C8C08091D608A7
:1017B000992788709070882309F0F3C120903D0329
:1017C00026FC62C23090DE06131508F4F3C1509077
:1017D000DD06511609F0C1C010936408CC2446B54B
:1017E00057B580904F08909050082CB53DB5309378
:1017F000500820934F082815390508F495C08091AA
:101800005108909152082417350708F40197AA2728
:10181000BB278C01FF24EE24CA01AA27BB27E82A94
:10182000F92A0A2B1B2B7090D70876FCC5C1409172
:101830005508509156086091570870915808370123
:101840004801641A750A860A970AE0925508F092D0
:10185000560800935708109358084D2C55244A8277
:101860005B8241FC7DC0A82CAA2009F475C18FEFD2
:10187000A82EB82E1982D0906408609169087091E2
:101880006A086C837D831B0136942794D7FCD4C4EB
:101890003091DC063E83E091DA062E2F3327C90112
:1018A00096958795969587959695879561E070E0D2
:1018B00086279727AC014623572380FFA8C14C8178
:1018C0005D814A155B0538F42501441A550A241434
:1018D000350408F4D9C281E090E09927009709F413
:1018E00077C1019709F4D3C3E091BA08F091BB081E
:1018F0003196F093BB08E093BA087FEF70936408C9
:1019000080E090E0282F80917208882309F45AC162
:1019100081508093720890915803A22EBB24A1FCA1
:1019200033C08091E00632C08091510890915208F6
:101930000196909352088093510865CF8091D60804
:10194000992784709070882309F025C160903D0329
:1019500066FC92C11091DE06115010936408ADC66A
:1019600060924703709248038092490390924A0321
:1019700060913C03616060933C0321E090915803C7
:10198000A22EBB24A1FECDCF8091E106890F9091BC
:10199000E406891708F0891B80935803A0FE9EC0B7
:1019A000E0926B08F0926C0800936D0810936E083B
:1019B000A091C008B091C1081196B093C108A0933E
:1019C000C00820913D03822F992783FDC7C080FD69
:1019D00009C0E091C608F091C7083196F093C70896
:1019E000E093C60880917108882309F4DAC1815018
:1019F0008093710820933D0330903D0330FC04C078
:101A00000091DB0604FD6AC0F7016091530340902A
:101A10005B0350905C037091E906872F807F9927C4
:101A2000009709F452C18037910509F489C385E014
:101A300090E080935303E1E0CE2E0E940943F090A2
:101A40003B03F1FE2FC160913B036F7C60933B032E
:101A500040903B0341FE04C0B0904106B4FC5CC220
:101A6000E0915D08EE2309F426C29E2F91509093D9
:101A70005D08E6E09E9FD0011124A659BC4F4D9110
:101A80005C9111974115510539F1FD0102811381D6
:101A9000E0904F08F0905008692F6295607FE92F21
:101AA000FF27E256FC4F2081822F80957BB378235D
:101AB0007BBB9AB3922B9ABBC701840F951FFD0184
:101AC000848395830417150708F0D9C2C701800FD6
:101AD000911F675F0E94017071E0C72EA091960868
:101AE000B09197081196B0939708A09396081A8121
:101AF00012FF23C0082D0929002329F188E893E16A
:101B00008C01A1FE02C01695079580914F08909117
:101B1000500862E0800F911F0E940170812F992769
:101B2000892B11F431E0C32EB7B7BF7DB7BFCC20EE
:101B300009F4C3C50E947D77C0C5F0E2F6BFCC2092
:101B400009F4BBC5F7CFC3019695879503E18938A2
:101B50009007A0F6CC97D4CF53018CCE277F10915D
:101B6000EA06110F110F195F109371089091590334
:101B700020FF13C120905803291609F43BCF9093FE
:101B800058038091C4089091C50801969093C508A8
:101B90008093C4082FCF61E08AE99BE80E94A12AC4
:101BA000D5CE212F40E050E061E082E89BE80E9422
:101BB0003F3104CE11500BCE62E085E99FE20E94D6
:101BC0006F3135CEE0913D03E77AE0933D03D6CE09
:101BD0005090DB0654FE5BC160913D0366FF45C239
:101BE00030913D033F7B30933D038E2F992785FF36
:101BF0006BC32D2D2450E0915303EE2321F4A091CB
:101C0000EA06A0935A03DD2492E099834AC125FF96
:101C1000CAC0AC81BD81AA16BB0608F4EEC1909182
:101C20001707B5012C813D81621B730B9F70905F7C
:101C3000290155274427499E9001599E300D411D89
:101C40001124DA01C901F4E0569547953795279597
:101C5000FA95D1F744E1B695A795979587954A955A
:101C6000D1F7882309F037C3C9016817790708F449
:101C700032CE8FEF90E031CE20913D032F7B209329
